:020000040000FA
:04070000F2EFE2F042
:08070800056ED8CF06F0E0CF2A
:1007100007F00001E9CF0DF0EACF08F0E1CF09F0D2
:10072000E2CF0AF0D9CF0BF0DACF0CF0F3CF14F010
:10073000F4CF15F0FACF16F0FBCF17F000C00FF092
:1007400001C010F002C011F003C012F004C013F099
:100750009DAAAEEF03F09EBA83EF26F0F2AAB4EFA3
:1007600003F0F2B4E8EF23F0A3AABAEF03F0A4BABF
:10077000AAEF26F09DA0C0EF03F09EB0D5EF22F0C7
:10078000F0AAC6EF03F0F0B4AEEF22F0F0A8CCEF81
:1007900003F0F0B28CEF22F0F0A6D2EF03F0F0B04D
:1007A0009DEF22F0F2A8D8EF03F0F2B27BEF22F037
:1007B000A0A2DEEF03F0A1B2F2EF24F00FC000F030
:1007C00010C001F011C002F012C003F013C004F019
:1007D0000E8E0DC0E9FF08C0EAFF09C0E1FF0AC0A4
:1007E000E2FF0BC0D9FF0CC0DAFF14C0F3FF15C045
:1007F000F4FF16C0FAFF17C0FBFF055007C0E0FF6B
:1008000006C0D8FF1000F2CF0EF0F29EF76A240F58
:10081000F66E080EF722000EF86E0900F5500EBEB7
:10082000F28E1200280C0106F2CF0EF0F29EF76A4B
:10083000460FF66E080EF722000EF86E0900F5500E
:100840000EBEF28E12000000F2CF0EF0F29EF76A9A
:10085000660FF66E080EF722000EF86E0900F550CE
:100860000EBEF28E1200536F6E79204556492D440C
:1008700033302020202020202000F2CF0EF0F29EE6
:10088000F76A980FF66E080EF722000EF86E090050
:10089000F5500EBEF28E1200536F6E792045564908
:1008A0002D4433302F44333120202000F2CF0EF07E
:1008B000F29EF76ACA0FF66E080EF722000EF86E67
:1008C0000900F5500EBEF28E120056616464696F25
:1008D000204164642D612D43616D20202000F2CF02
:1008E0000EF0F29EF76AFC0FF66E080EF722000E6D
:1008F000F86E0900F5500EBEF28E1200536F6E793D
:10090000204556492D443130302020202020200021
:10091000F2CF0EF0F29EF76A2E0FF66E090EF72256
:10092000000EF86E0900F5500EBEF28E1200536FE5
:100930006E79204556492D44373020202020202034
:100940002000F2CF0EF0F29EF76A600FF66E090EED
:10095000F722000EF86E0900F5500EBEF28E12005E
:10096000536F6E79204252432D33303020202020A7
:1009700020202000F2CF0EF0F29EF76A920FF66E62
:10098000090EF722000EF86E0900F5500EBEF28E29
:100990001200536F6E79204252432D483730302079
:1009A000202020202000F2CF0EF0F29EF76AC40F24
:1009B000F66E090EF722000EF86E0900F5500EBE15
:1009C000F28E1200536F6E79204252432D5A373007
:1009D0003020202020202000F2CF0EF0F29EF76A77
:1009E000F60FF66E090EF722000EF86E0900F550AC
:1009F0000EBEF28E1200536F6E79204556492D4877
:100A000044312020202020202000F2CF0EF0F29E42
:100A1000F76A280FF66E0A0EF722000EF86E09002C
:100A2000F5500EBEF28E120056616464696F204369
:100A300065696C696E67564945572000F2CF0EF024
:100A4000F29EF76A5A0FF66E0A0EF722000EF86E43
:100A50000900F5500EBEF28E120043616E6E6F6E8D
:100A60002056432D43353069202020202000F2CF2E
:100A70000EF0F29EF76A8C0FF66E0A0EF722000E49
:100A8000F86E0900F5500EBEF28E12004E6F742003
:100A9000466F756E6420202020202020202020001A
:100AA000F2CF0EF0F29EF76ABE0FF66E0A0EF72234
:100AB000000EF86E0900F5500EBEF28E1200457859
:100AC0007420507265736574733A2043616D3120F0
:100AD000312D31322C2043616D32204E6F6E650016
:100AE000F2CF0EF0F29EF76AFE0FF66E0A0EF722B4
:100AF000000EF86E0900F5500EBEF28E1200457819
:100B00007420507265736574733A2043616D3120AF
:100B1000312D362C2043616D3220312D3600F2CF3D
:100B20000EF0F29EF76A3C0FF66E0B0EF722000EE7
:100B3000F86E0900F5500EBEF28E12005A6F6F6DFE
:100B400020446972656374696F6E3A20496E7665F8
:100B500072740000F2CF0EF0F29EF76A720FF66E1A
:100B60000B0EF722000EF86E0900F5500EBEF28E45
:100B700012005A6F6F6D20446972656374696F6EFD
:100B80003A204E6F726D616C0000F2CF0EF0F29E53
:100B9000F76AA80FF66E0B0EF722000EF86E09002A
:100BA000F5500EBEF28E12004578742050726573B7
:100BB000657420696E332D362044697265637469EB
:100BC0006F6E3A204F75747075740000F2CF0EF09E
:100BD000F29EF76AEA0FF66E0B0EF722000EF86E21
:100BE0000900F5500EBEF28E120045787420507246
:100BF0006573657420696E332D36204469726563B0
:100C000074696F6E3A20496E70757400F2CF0EF001
:100C1000F29EF76A2A0FF66E0C0EF722000EF86E9F
:100C20000900F5500EBEF28E1200486F7374205307
:100C3000657269616C20496E7075743A20456E6109
:100C4000626C65640000F2CF0EF0F29EF76A640FEA
:100C5000F66E0C0EF722000EF86E0900F5500EBE6F
:100C6000F28E1200486F73742053657269616C20B4
:100C7000496E7075743A2044697361626C656400F2
:100C8000F2CF0EF0F29EF76A9E0FF66E0C0EF72270
:100C9000000EF86E0900F5500EBEF28E120053657C
:100CA0007269616C204563686F3A20456E61626CC1
:100CB00065640000F2CF0EF0F29EF76AD20FF66E76
:100CC0000C0EF722000EF86E0900F5500EBEF28EE3
:100CD000120053657269616C204563686F3A204465
:100CE000697361626C656400F2CF0EF0F29EF76A80
:100CF000060FF66E0D0EF722000EF86E0900F55085
:100D00000EBEF28E120043616D2053656C20466F5B
:100D10006C6C6F777320507265766965773A204501
:100D20006E61626C65640000F2CF0EF0F29EF76AAD
:100D3000460FF66E0D0EF722000EF86E0900F55004
:100D40000EBEF28E120043616D2053656C20466F1B
:100D50006C6C6F777320507265766965773A2044C2
:100D6000697361626C656400F2CF0EF0F29EF76AFF
:100D7000860FF66E0D0EF722000EF86E0900F55084
:100D80000EBEF28E120053797374656D204D6F6440
:100D9000653A204175746F00F2CF0EF0F29EF76A4B
:100DA000B60FF66E0D0EF722000EF86E0900F55024
:100DB0000EBEF28E120053797374656D204D6F6410
:100DC000653A204D616E75616C00F2CF0EF0F29EB7
:100DD000F76AE80FF66E0D0EF722000EF86E0900A6
:100DE000F5500EBEF28E1200566964656F204D6F8D
:100DF00064653A2050414C00F2CF0EF0F29EF76A43
:100E0000160FF66E0E0EF722000EF86E0900F55062
:100E10000EBEF28E1200566964656F204D6F6465D8
:100E20003A204E5453430000F2CF0EF0F29EF76A80
:100E3000460FF66E0E0EF722000EF86E0900F55002
:100E40000EBEF28E1200446961676E6F737469633F
:100E5000204D6F64653A204F6E00F2CF0EF0F29E87
:100E6000F76A780FF66E0E0EF722000EF86E090084
:100E7000F5500EBEF28E1200446961676E6F737496
:100E80006963204D6F64653A204F66660000F2CFBB
:100E90000EF0F29EF76AAC0FF66E0E0EF722000E01
:100EA000F86E0900F5500EBEF28E1200536572699D
:100EB000616C20496E666F3A204F6E00F2CF0EF0E3
:100EC000F29EF76ADA0FF66E0E0EF722000EF86E3B
:100ED0000900F5500EBEF28E120053657269616C06
:100EE00020496E666F3A204F66660000F2CF0EF022
:100EF000F29EF76A0A0FF66E0F0EF722000EF86EDA
:100F00000900F5500EBEF28E12004F7574707574A4
:100F10002027436F6C6F72204261727327204F6EDF
:100F2000204E6F20496E70757420536F7572636523
:100F30000000F2CF0EF0F29EF76A500FF66E0F0E21
:100F4000F722000EF86E0900F5500EBEF28E120068
:100F50004F75747075742027426C616E6B27204F3B
:100F60006E204E6F20496E70757420536F757263DA
:100F70006500F2CF0EF0F29EF76A900FF66E0F0E3C
:100F8000F722000EF86E0900F5500EBEF28E120028
:100F9000506F776572207570205072657365743A72
:100FA000205072657365742031320000F2CF0EF06C
:100FB000F29EF76ACA0FF66E0F0EF722000EF86E59
:100FC0000900F5500EBEF28E1200506F7765722048
:100FD0007570205072657365743A20486F6D652096
:100FE00043616D00F2CF0EF0F29EF76A020FF66ECB
:100FF000100EF722000EF86E0900F5500EBEF28EAC
:101000001200504320457870616E646572204D6F08
:1010100064653A20532D566964656F00F2CF0EF077
:10102000F29EF76A3A0FF66E100EF722000EF86E77
:101030000900F5500EBEF28E120050432045787024
:10104000616E646572204D6F64653A204E6F6E6507
:101050000000F2CF0EF0F29EF76A700FF66E100EDF
:10106000F722000EF86E0900F5500EBEF28E120047
:10107000504320457870616E646572204D6F6465E1
:101080003A20436F6D706F7369746500F2CF0EF094
:10109000F29EF76AAA0FF66E100EF722000EF86E97
:1010A0000900F5500EBEF28E120050726573657421
:1010B000204C6F636174696F6E3A20312D36204980
:1010C0006E43616D2C362D3132204C6F63616C00A4
:1010D000F2CF0EF0F29EF76AEE0FF66E100EF722C8
:1010E000000EF86E0900F5500EBEF28E120050721E
:1010F00065736574204C6F636174696F6E3A20315B
:101100002D3132204C6F63616C00F2CF0EF0F29EF5
:10111000F76A280FF66E110EF722000EF86E09001E
:10112000F5500EBEF28E1200446F46696E64416344
:10113000746976655072657365747320506F72744C
:10114000202564206261640A0D00F2CF0EF0F29E49
:10115000F76A680FF66E110EF722000EF86E09009E
:10116000F5500EBEF28E1200202020537973746564
:101170006D204D656E7520202000F2CF0EF0F29E9E
:10118000F76A980FF66E110EF722000EF86E09003E
:10119000F5500EBEF28E1200202053657269616C0C
:1011A00020496E70757420202000F2CF0EF0F29E60
:1011B000F76AC80FF66E110EF722000EF86E0900DE
:1011C000F5500EBEF28E1200202053657269616CDC
:1011D000204563686F2020202000F2CF0EF0F29EA1
:1011E000F76AF80FF66E110EF722000EF86E09007E
:1011F000F5500EBEF28E12002020436C6561722005
:101200004D656D6F727920202000F2CF0EF0F29EB6
:10121000F76A280FF66E120EF722000EF86E09001C
:10122000F5500EBEF28E12002020436C65617220D4
:1012300050726573657473202000F2CF0EF0F29E39
:10124000F76A580FF66E120EF722000EF86E0900BC
:10125000F5500EBEF28E1200202020536572696197
:101260006C20496E666F20202000F2CF0EF0F29EB7
:10127000F76A880FF66E120EF722000EF86E09005C
:10128000F5500EBEF28E1200202049646C65204499
:101290006973706C617920202000F2CF0EF0F29E0D
:1012A000F76AB80FF66E120EF722000EF86E0900FC
:1012B000F5500EBEF28E12002020506F776572201E
:1012C00055702050726573657400F2CF0EF0F29E77
:1012D000F76AE80FF66E120EF722000EF86E09009C
:1012E000F5500EBEF28E12002020507265736574A8
:1012F000204C6F636174696F6E00F2CF0EF0F29E46
:10130000F76A180FF66E130EF722000EF86E09003A
:10131000F5500EBEF28E12002020202050432045B2
:101320007870616E646572202000F2CF0EF0F29E3C
:10133000F76A480FF66E130EF722000EF86E0900DA
:10134000F5500EBEF28E1200202052657475726E3A
:1013500020746F204D61696E2000F2CF0EF0F29E76
:10136000F76A780FF66E130EF722000EF86E09007A
:10137000F5500EBEF28E120020202050616E2044E7
:101380006972204D656E75202000F2CF0EF0F29E3E
:10139000F76AA80FF66E130EF722000EF86E09001A
:1013A000F5500EBEF28E12002020202020416C6CE1
:1013B00020506F72747320202000F2CF0EF0F29E46
:1013C000F76AD80FF66E130EF722000EF86E0900BA
:1013D000F5500EBEF28E1200202020202020506FEB
:1013E00072742030312020202000F2CF0EF0F29EC7
:1013F000F76A080FF66E140EF722000EF86E090059
:10140000F5500EBEF28E1200202020202020506FBA
:1014100072742030322020202000F2CF0EF0F29E95
:10142000F76A380FF66E140EF722000EF86E0900F8
:10143000F5500EBEF28E1200202020202020506F8A
:1014400072742030332020202000F2CF0EF0F29E64
:10145000F76A680FF66E140EF722000EF86E090098
:10146000F5500EBEF28E1200202020202020506F5A
:1014700072742030342020202000F2CF0EF0F29E33
:10148000F76A980FF66E140EF722000EF86E090038
:10149000F5500EBEF28E1200202020202020506F2A
:1014A00072742030352020202000F2CF0EF0F29E02
:1014B000F76AC80FF66E140EF722000EF86E0900D8
:1014C000F5500EBEF28E1200202020202020506FFA
:1014D00072742030362020202000F2CF0EF0F29ED1
:1014E000F76AF80FF66E140EF722000EF86E090078
:1014F000F5500EBEF28E1200202054696C74204408
:101500006972204D656E75202000F2CF0EF0F29EBC
:10151000F76A280FF66E150EF722000EF86E090016
:10152000F5500EBEF28E12002020205265736361CA
:101530006E2043616D6572617300F2CF0EF0F29E12
:10154000F76A580FF66E150EF722000EF86E0900B6
:10155000F5500EBEF28E12002020204465666175A3
:101560006C742043616D65726100F2CF0EF0F29EE3
:10157000F76A880FF66E150EF722000EF86E090056
:10158000F5500EBEF28E1200202020446566617573
:101590006C742050726573657400F2CF0EF0F29E89
:1015A000F76AB80FF66E150EF722000EF86E0900F6
:1015B000F5500EBEF28E120020202050616E536551
:1015C0006E736974697669747900F2CF0EF0F29ED9
:1015D000F76AE80FF66E150EF722000EF86E090096
:1015E000F5500EBEF28E1200202054696C745365C3
:1015F0006E736974697669747900F2CF0EF0F29EA9
:10160000F76A180FF66E160EF722000EF86E090034
:10161000F5500EBEF28E120020202044656620494F
:10162000646C652052746E202000F2CF0EF0F29EA2
:10163000F76A480FF66E160EF722000EF86E0900D4
:10164000F5500EBEF28E1200202020202050616E38
:1016500020537065656420202000F2CF0EF0F29ECA
:10166000F76A780FF66E160EF722000EF86E090074
:10167000F5500EBEF28E12002020202054696C74AA
:1016800020537065656420202000F2CF0EF0F29E9A
:10169000F76AA80FF66E160EF722000EF86E090014
:1016A000F5500EBEF28E1200202020202020537410
:1016B00061727400F2CF0EF0F29EF76AD20FF66EEE
:1016C000160EF722000EF86E0900F5500EBEF28ECF
:1016D0001200202020202020205965730000F2CF26
:1016E0000EF0F29EF76AFC0FF66E160EF722000E51
:1016F000F86E0900F5500EBEF28E12002020202058
:10170000202020204E6F0000F2CF0EF0F29EF76AEC
:10171000260FF66E170EF722000EF86E0900F55030
:101720000EBEF28E12002020202020204E6F726DFF
:10173000616C0000F2CF0EF0F29EF76A520FF66E67
:10174000170EF722000EF86E0900F5500EBEF28E4D
:101750001200202020202020496E7665727400003F
:10176000F2CF0EF0F29EF76A7E0FF66E170EF7229A
:10177000000EF86E0900F5500EBEF28E1200202009
:101780002020202020496E7075740000F2CF0EF0EA
:10179000F29EF76AAA0FF66E170EF722000EF86E89
:1017A0000900F5500EBEF28E1200202020202020CD
:1017B0004F75747075740000F2CF0EF0F29EF76AE8
:1017C000D60FF66E170EF722000EF86E0900F550D0
:1017D0000EBEF28E12002020362043616D3120367D
:1017E0002043616D3200F2CF0EF0F29EF76A040FD3
:1017F000F66E180EF722000EF86E0900F5500EBEB8
:10180000F28E1200202020416C6C20313220436186
:101810006D310000F2CF0EF0F29EF76A320FF66ED5
:10182000180EF722000EF86E0900F5500EBEF28E6B
:101830001200202020202020204F66660000F2CFDA
:101840000EF0F29EF76A5C0FF66E180EF722000E8D
:10185000F86E0900F5500EBEF28E120020202020F6
:101860002020204F6E200000F2CF0EF0F29EF76A8B
:10187000860FF66E180EF722000EF86E0900F5506E
:101880000EBEF28E12002020202020426C61636B7D
:10189000202020200000F2CF0EF0F29EF76AB40F55
:1018A000F66E180EF722000EF86E0900F5500EBE07
:1018B000F28E12002020202020436F6C6F72204295
:1018C00061727300F2CF0EF0F29EF76AE20FF66ECD
:1018D000180EF722000EF86E0900F5500EBEF28EBB
:1018E00012002020202020486F6D652043616D6527
:1018F00072612000F2CF0EF0F29EF76A120FF66EC0
:10190000190EF722000EF86E0900F5500EBEF28E89
:10191000120020202020205072657365742031321F
:1019200020202000F2CF0EF0F29EF76A420FF66EF2
:10193000190EF722000EF86E0900F5500EBEF28E59
:1019400012002020202020416C6C204C6F63616CC1
:1019500020202000F2CF0EF0F29EF76A720FF66E92
:10196000190EF722000EF86E0900F5500EBEF28E29
:10197000120020203620496E43616D2036204C6FC6
:1019800063616C00F2CF0EF0F29EF76AA20FF66E62
:10199000190EF722000EF86E0900F5500EBEF28EF9
:1019A0001200202020202020204E4F4E45202020B5
:1019B00020202000F2CF0EF0F29EF76AD20FF66ED2
:1019C000190EF722000EF86E0900F5500EBEF28EC9
:1019D00012002020202020532D566964656F20209E
:1019E00020202000F2CF0EF0F29EF76A020FF66E72
:1019F0001A0EF722000EF86E0900F5500EBEF28E98
:101A0000120020202020436F6D706F736974652071
:101A100020202000F2CF0EF0F29EF76A320FF66E11
:101A20001A0EF722000EF86E0900F5500EBEF28E67
:101A300012002050432D457870616E64657220530A
:101A40002D566900F2CF0EF0F29EF76A620FF66E25
:101A50001A0EF722000EF86E0900F5500EBEF28E37
:101A600012002050432D457870616E6465722043EA
:101A70006F6D7000F2CF0EF0F29EF76A920FF66E65
:101A80001A0EF722000EF86E0900F5500EBEF28E07
:101A900012000D0A20576169745F50435F457870EA
:101AA000616E646572526573706F6E736520256C2C
:101AB0006420286D73290D0A0000F2CF0EF0F29E0B
:101AC000F76AD80FF66E1A0EF722000EF86E0900AC
:101AD000F5500EBEF28E12000D0A20576169745F38
:101AE00050435F457870616E646572526573706FC4
:101AF0006E7365200000F2CF0EF0F29EF76A140FAD
:101B0000F66E1B0EF722000EF86E0900F5500EBEA1
:101B1000F28E1200496E7075742053656C656374A3
:101B20002025630A0D00F2CF0EF0F29EF76A440FF3
:101B3000F66E1B0EF722000EF86E0900F5500EBE71
:101B4000F28E1200536561726368696E6720666F7A
:101B5000722041747461636865642043616D6572CD
:101B600061730D0A0000F2CF0EF0F29EF76A840F47
:101B7000F66E1B0EF722000EF86E0900F5500EBE31
:101B8000F28E1200506F72742025643A20200000FB
:101B9000F2CF0EF0F29EF76AAE0FF66E1B0EF72232
:101BA000000EF86E0900F5500EBEF28E1200504382
:101BB0002D457870616E6465722044657465637448
:101BC00065640D0A0000F2CF0EF0F29EF76AE40F92
:101BD000F66E1B0EF722000EF86E0900F5500EBED1
:101BE000F28E1200205063457870616E6465722039
:101BF000506F72743600F2CF0EF0F29EF76A140F37
:101C0000F66E1C0EF722000EF86E0900F5500EBE9F
:101C1000F28E1200204E6F2043616D202020205054
:101C20006F7274203000F2CF0EF0F29EF76A440F0C
:101C3000F66E1C0EF722000EF86E0900F5500EBE6F
:101C4000F28E12002056432D43353069202020505B
:101C50006F7274203000F2CF0EF0F29EF76A740FAC
:101C6000F66E1C0EF722000EF86E0900F5500EBE3F
:101C7000F28E120043616E6F6E204465746563746A
:101C800065640D0A0000F2CF0EF0F29EF76AA40F11
:101C9000F66E1C0EF722000EF86E0900F5500EBE0F
:101CA000F28E12000D0A2057616974466565644220
:101CB00061636B2054696D656F757420323030300C
:101CC00020286D73290D0A00F2CF0EF0F29EF76AFC
:101CD000E60FF66E1C0EF722000EF86E0900F550A6
:101CE0000EBEF28E12000D0A2057616974466565BA
:101CF000644261636B200000F2CF0EF0F29EF76A3F
:101D0000160FF66E1D0EF722000EF86E0900F55044
:101D10000EBEF28E12000A0D2043616D6572615491
:101D2000797065200000F2CF0EF0F29EF76A440F42
:101D3000F66E1D0EF722000EF86E0900F5500EBE6D
:101D4000F28E120054696D656F75740A0D200000E3
:101D5000F2CF0EF0F29EF76A6E0FF66E1D0EF722AE
:101D6000000EF86E0900F5500EBEF28E12000D0A3C
:101D7000536F6E79204556492D4433302F3331202F
:101D80000D0A0000F2CF0EF0F29EF76AA20FF66E77
:101D90001D0EF722000EF86E0900F5500EBEF28EF1
:101DA0001200204556492D4433302F3331506F7285
:101DB00074203000F2CF0EF0F29EF76AD20FF66E6A
:101DC0001D0EF722000EF86E0900F5500EBEF28EC1
:101DD00012000D0A536F6E79204556492D44333059
:101DE0000D0A0000F2CF0EF0F29EF76A020FF66EB7
:101DF0001E0EF722000EF86E0900F5500EBEF28E90
:101E00001200204556492D443330202020506F7257
:101E100074203000F2CF0EF0F29EF76A320FF66EA9
:101E20001E0EF722000EF86E0900F5500EBEF28E5F
:101E300012000D0A56616464696F204164642D418B
:101E40002D43616D0D0A0000F2CF0EF0F29EF76A8D
:101E5000660FF66E1E0EF722000EF86E0900F550A2
:101E60000EBEF28E1200204164642D412D43616D3F
:101E700020506F7274203000F2CF0EF0F29EF76A9D
:101E8000960FF66E1E0EF722000EF86E0900F55042
:101E90000EBEF28E12000D0A536F6E792045564920
:101EA0002D443130300D0A00F2CF0EF0F29EF76A69
:101EB000C60FF66E1E0EF722000EF86E0900F550E2
:101EC0000EBEF28E1200204556492D44313030208E
:101ED00020506F7274203000F2CF0EF0F29EF76A3D
:101EE000F60FF66E1E0EF722000EF86E0900F55082
:101EF0000EBEF28E12000D0A536F6E7920455649C0
:101F00002D4437300D0A0000F2CF0EF0F29EF76A32
:101F1000260FF66E1F0EF722000EF86E0900F55020
:101F20000EBEF28E1200204556492D443730202037
:101F300020506F7274203000F2CF0EF0F29EF76ADC
:101F4000560FF66E1F0EF722000EF86E0900F550C0
:101F50000EBEF28E12000D0A536F6E79204252436C
:101F6000482D3730300D0A00F2CF0EF0F29EF76A9E
:101F7000860FF66E1F0EF722000EF86E0900F55060
:101F80000EBEF28E120020425243482D37303020D0
:101F900020506F7274203000F2CF0EF0F29EF76A7C
:101FA000B60FF66E1F0EF722000EF86E0900F55000
:101FB0000EBEF28E12000D0A456C6D6F2043616DEE
:101FC0006572610D0A00F2CF0EF0F29EF76AE40F1F
:101FD000F66E1F0EF722000EF86E0900F5500EBEC9
:101FE000F28E120020456C6D6F20202020202050A2
:101FF0006F7274203000F2CF0EF0F29EF76A140F69
:10200000F66E200EF722000EF86E0900F5500EBE97
:10201000F28E12000D0A536F6E79204252432D3317
:1020200030300D0A0000F2CF0EF0F29EF76A440F36
:10203000F66E200EF722000EF86E0900F5500EBE67
:10204000F28E1200204252432D3330302020205097
:102050006F7274203000F2CF0EF0F29EF76A740FA8
:10206000F66E200EF722000EF86E0900F5500EBE37
:10207000F28E12000D0A536F6E79204252432D5A90
:102080003730300D0A00F2CF0EF0F29EF76AA40F3F
:10209000F66E200EF722000EF86E0900F5500EBE07
:1020A000F28E1200204252432D5A373030202050F9
:1020B0006F7274203000F2CF0EF0F29EF76AD40FE8
:1020C000F66E200EF722000EF86E0900F5500EBED7
:1020D000F28E12000D0A536F6E79204556492D4835
:1020E00044310D0A0000F2CF0EF0F29EF76A040FA1
:1020F000F66E210EF722000EF86E0900F5500EBEA6
:10210000F28E1200204556492D484431202020509F
:102110006F7274203000F2CF0EF0F29EF76A340F27
:10212000F66E210EF722000EF86E0900F5500EBE75
:10213000F28E12000D0A56616464696F204365696E
:102140006C696E67564945570D0A0000F2CF0EF0D4
:10215000F29EF76A6A0FF66E210EF722000EF86EF5
:102160000900F5500EBEF28E12002043562F435642
:102170004D50202020506F7274203000F2CF0EF0AE
:10218000F29EF76A9A0FF66E210EF722000EF86E95
:102190000900F5500EBEF28E1200496E76616C6930
:1021A000642043616D6572610D0A0000F2CF0EF08C
:1021B000F29EF76ACA0FF66E210EF722000EF86E35
:1021C0000900F5500EBEF28E120020496E76616C49
:1021D00069642043616D65726100F2CF0EF0F29E7A
:1021E000F76AF80FF66E210EF722000EF86E09005E
:1021F000F5500EBEF28E12000D0A536F6E79204517
:1022000056492D4433302872290D0A00F2CF0EF0C2
:10221000F29EF76A2A0FF66E220EF722000EF86E73
:102220000900F5500EBEF28E1200204556492D448D
:102230003330287229506F7274203000F2CF0EF0C4
:10224000F29EF76A5A0FF66E220EF722000EF86E13
:102250000900F5500EBEF28E12000A0D2041542FD7
:102260004D445F4D6F6465496E712000F2CF0EF0F2
:10227000F29EF76A8A0FF66E220EF722000EF86EB3
:102280000900F5500EBEF28E12002054696D656F84
:1022900075740A0D2000F2CF0EF0F29EF76AB40FAB
:1022A000F66E220EF722000EF86E0900F5500EBEF3
:1022B000F28E12000D0A2057616974536F6E7941D6
:1022C000636B2054696D656F757420256C642028DC
:1022D0006D73290D0A00F2CF0EF0F29EF76AF40F2B
:1022E000F66E220EF722000EF86E0900F5500EBEB3
:1022F000F28E12000D0A2057616974536F6E794196
:10230000636B2000F2CF0EF0F29EF76A220FF66E9A
:10231000230EF722000EF86E0900F5500EBEF28E65
:1023200012000D0A2057616974536F6E7920546949
:102330006D656F757420256C6420286D73290D0AF6
:102340000000F2CF0EF0F29EF76A600FF66E230ED9
:10235000F722000EF86E0900F5500EBEF28E120044
:102360000D0A2057616974536F6E79200000F2CF17
:102370000EF0F29EF76A8C0FF66E230EF722000E17
:10238000F86E0900F5500EBEF28E12002054696DF1
:10239000656F757420256C6420286D73290D0A0003
:1023A000F2CF0EF0F29EF76ABE0FF66E230EF72202
:1023B000000EF86E0900F5500EBEF28E12000A0DE6
:1023C0002042616420436F6D6D616E640A0D0000F0
:1023D000F2CF0EF0F29EF76AEE0FF66E230EF722A2
:1023E000000EF86E0900F5500EBEF28E12000D0AB6
:1023F000205761697443616E6F6E2054696D656F1B
:10240000757420256C6420286D73290D0A00F2CFA5
:102410000EF0F29EF76A2C0FF66E240EF722000ED5
:10242000F86E0900F5500EBEF28E12000D0A20570C
:1024300061697443616E6F6E2000F2CF0EF0F29E00
:10244000F76A580FF66E240EF722000EF86E090098
:10245000F5500EBEF28E12000D0A205761697443CA
:10246000616E6F6E41636B2054696D656F7574208A
:10247000256C6420286D73290D0A0000F2CF0EF040
:10248000F29EF76A9A0FF66E240EF722000EF86E8F
:102490000900F5500EBEF28E12000D0A2057616938
:1024A0007443616E6F6E41636B200000F2CF0EF0DB
:1024B000F29EF76ACA0FF66E240EF722000EF86E2F
:1024C0000900F5500EBEF28E120057616974436127
:1024D0006E6F6E41636B202532782C253278202870
:1024E000253278290D0A0000F2CF0EF0F29EF76A2D
:1024F000060FF66E250EF722000EF86E0900F55055
:102500000EBEF28E1200446F5570646174654361B3
:102510006D65726153746174653A205374617465BA
:10252000466C61673D202532582C204C6173743D08
:102530002532582C204163746976653D2532580A4E
:102540000D3E0000F2CF0EF0F29EF76A620FF66EBB
:10255000250EF722000EF86E0900F5500EBEF28E21
:102560001200446F55706461746543616D657261FA
:1025700053746174653A20446966666572656E637A
:10258000653D2532780A0D00F2CF0EF0F29EF76A13
:10259000A60FF66E250EF722000EF86E0900F55014
:1025A0000EBEF28E1200446F557064617465436113
:1025B0006D65726153746174653A20546F20417582
:1025C000746F0A0D3E00F2CF0EF0F29EF76AE40F30
:1025D000F66E250EF722000EF86E0900F5500EBEBD
:1025E000F28E1200446F55706461746543616D65CD
:1025F000726153746174653A205265736574204248
:1026000072696768746E657320746F2064656661B3
:10261000756C740A0D3E0000F2CF0EF0F29EF76A60
:10262000360FF66E260EF722000EF86E0900F550F2
:102630000EBEF28E1200446F557064617465436182
:102640006D65726153746174653A20546F204D61F9
:102650006E75616C0A0D3E00F2CF0EF0F29EF76AC5
:10266000760FF66E260EF722000EF86E0900F55072
:102670000EBEF28E12000A0D50726F6475637420E4
:102680004E616D653A20257325730A0D0000F2CF67
:102690000EF0F29EF76AAC0FF66E260EF722000ED1
:1026A000F86E0900F5500EBEF28E12002020202098
:1026B000436F6D70696C65643A20257320617420E6
:1026C00025730A0D0000F2CF0EF0F29EF76AE40FB8
:1026D000F66E260EF722000EF86E0900F5500EBEBB
:1026E000F28E120031342D4D61792D303800F2CF49
:1026F0000EF0F29EF76A0C0FF66E270EF722000E10
:10270000F86E0900F5500EBEF28E120031303A33E9
:10271000333A30360000F2CF0EF0F29EF76A340FF3
:10272000F66E270EF722000EF86E0900F5500EBE69
:10273000F28E12000D0A53797374656D205365741F
:1027400074696E67733A0A0D0A0D44656661756CAB
:10275000742043616D6572613A2025640A0D4465F9
:102760006661756C74205072657365743A202564D7
:102770000A0D0000F2CF0EF0F29EF76A920FF66E8D
:10278000270EF722000EF86E0900F5500EBEF28EED
:1027900012000D0A54696C745370656564202050F2
:1027A000616E5370656564202049646C65205265D4
:1027B0007475726E202050616E656C204C6967687C
:1027C00074730A0D0000F2CF0EF0F29EF76AE40F68
:1027D000F66E270EF722000EF86E0900F5500EBEB9
:1027E000F28E12002020202564202020202020208E
:1027F0002020256420202020202020202025642047
:10280000202020202020202020202025640A0D0ABE
:102810000D00F2CF0EF0F29EF76A300FF66E280E22
:10282000F722000EF86E0900F5500EBEF28E12006F
:102830000D0A4A6F79737469636B2053656E73690F
:10284000746976697479202050616E202054696C17
:1028500074202049646C65205A6F6E650A0D000073
:10286000F2CF0EF0F29EF76A7E0FF66E280EF72278
:10287000000EF86E0900F5500EBEF28E12002020F8
:102880002020202020202020202020202020202048
:1028900020202020256420202020256420202020A6
:1028A000202025640A0D0A0D0000F2CF0EF0F29EE2
:1028B000F76AC80FF66E280EF722000EF86E0900B0
:1028C000F5500EBEF28E12002050616E20446972E7
:1028D000656374696F6E20627920506F72743A205C
:1028E00031203220332034203520360A0D00F2CF3B
:1028F0000EF0F29EF76A0C0FF66E290EF722000E0C
:10290000F86E0900F5500EBEF28E12002020202035
:1029100020202020202020202020202020202020B7
:102920002020202025632025632025632025632087
:1029300025632025630A0D00F2CF0EF0F29EF76AA0
:10294000560FF66E290EF722000EF86E0900F550AC
:102950000EBEF28E12000D0A54696C742044697226
:10296000656374696F6E20627920506F72743A20CB
:1029700031203220332034203520360A0D00F2CFAA
:102980000EF0F29EF76A9C0FF66E290EF722000EEB
:10299000F86E0900F5500EBEF28E12000A0D50724C
:1029A00065736574733A0A0D0A0D0000F2CF0EF0DC
:1029B000F29EF76ACA0FF66E290EF722000EF86E25
:1029C0000900F5500EBEF28E120043616D20507268
:1029D00065204D6F64656C20202020202020202061
:1029E000202020202020202050616E2020205469AB
:1029F0006C7420205A6F6F6D20466F6375732020B2
:102A00004272696768746E6573730000F2CF0EF0EE
:102A1000F29EF76A2A0FF66E2A0EF722000EF86E63
:102A20000900F5500EBEF28E1200205B42726967FB
:102A300068742C466F6375732C4157422C424C438B
:102A40005D0A0D0A0D00F2CF0EF0F29EF76A640FD8
:102A5000F66E2A0EF722000EF86E0900F5500EBE33
:102A6000F28E12002025642020202532642025319A
:102A7000387320253258254C582020254C582020CA
:102A8000254C582020254C582020202020254C580B
:102A90000000F2CF0EF0F29EF76AB00FF66E2A0E2B
:102AA000F722000EF86E0900F5500EBEF28E1200ED
:102AB0002020202020202000F2CF0EF0F29EF76A86
:102AC000D60FF66E2A0EF722000EF86E0900F550AA
:102AD0000EBEF28E12004F6E20202020202000001B
:102AE000F2CF0EF0F29EF76AFE0FF66E2A0EF72274
:102AF000000EF86E0900F5500EBEF28E12004F6601
:102B00006620202020200000F2CF0EF0F29EF76A0F
:102B1000260FF66E2B0EF722000EF86E0900F55008
:102B20000EBEF28E12004F6E202020200000F2CF49
:102B30000EF0F29EF76A4C0FF66E2B0EF722000E87
:102B4000F86E0900F5500EBEF28E12004F66662038
:102B500020200000F2CF0EF0F29EF76A720FF66EA0
:102B60002B0EF722000EF86E0900F5500EBEF28E05
:102B700012004F6E20202000F2CF0EF0F29EF76A76
:102B8000960FF66E2B0EF722000EF86E0900F55028
:102B90000EBEF28E12004F6666202000F2CF0EF0BD
:102BA000F29EF76ABA0FF66E2B0EF722000EF86E41
:102BB0000900F5500EBEF28E12004F6E0000F2CFEB
:102BC0000EF0F29EF76ADC0FF66E2B0EF722000E67
:102BD000F86E0900F5500EBEF28E12004F666600C8
:102BE000F2CF0EF0F29EF76AFE0FF66E2B0EF72272
:102BF000000EF86E0900F5500EBEF28E12000A0D9E
:102C0000436F6D6D616E6420436F6D706C657465AC
:102C10000A0D3E00F2CF0EF0F29EF76A320FF66E0A
:102C20002C0EF722000EF86E0900F5500EBEF28E43
:102C300012000A0D43616D204D6F64656C0A0D0032
:102C4000F2CF0EF0F29EF76A5E0FF66E2C0EF722B0
:102C5000000EF86E0900F5500EBEF28E120020250F
:102C60006420204E6F2043616D6572610A0D000083
:102C7000F2CF0EF0F29EF76A8E0FF66E2C0EF72250
:102C8000000EF86E0900F5500EBEF28E12003E25C1
:102C900073204E6F7420466F756E640A0D3E0000FF
:102CA000F2CF0EF0F29EF76ABE0FF66E2C0EF722F0
:102CB000000EF86E0900F5500EBEF28E12000A0DDD
:102CC0003E2043616D657261202564204E6F742043
:102CD000617661696C61626C650A0D3E2000F2CF1D
:102CE0000EF0F29EF76AFC0FF66E2C0EF722000E25
:102CF000F86E0900F5500EBEF28E12000A0D3E204D
:102D00004A6F79737469636B204E65757472616C78
:102D1000205A6F6E65202564200A0D3E2000F2CFF8
:102D20000EF0F29EF76A3C0FF66E2D0EF722000EA3
:102D3000F86E0900F5500EBEF28E12000A0D3E200C
:102D4000446973706C617920436F6C6F7242617279
:102D500073206F6E2049646C6520446973706C61E8
:102D6000790A0D3E2000F2CF0EF0F29EF76A840F32
:102D7000F66E2D0EF722000EF86E0900F5500EBE0D
:102D8000F28E12000A0D3E20446973706C61792046
:102D9000426C61636B206F6E2049646C65204469EE
:102DA00073706C61790A0D3E2000F2CF0EF0F29E36
:102DB000F76AC80FF66E2D0EF722000EF86E0900A6
:102DC000F5500EBEF28E1200566964656F204D6F8D
:102DD0006465206973200000F2CF0EF0F29EF76A5E
:102DE000F60FF66E2D0EF722000EF86E0900F55064
:102DF0000EBEF28E12004F6E2043616D657261202F
:102E0000496E69742C2073656E6420486F6D65206F
:102E1000636F6D6D616E640A0D3E2000F2CF0EF09F
:102E2000F29EF76A3A0FF66E2E0EF722000EF86E3B
:102E30000900F5500EBEF28E12004F6E2043616DF8
:102E400065726120496E69742C2073656E64205030
:102E5000726573657420313220636F6D6D616E64CD
:102E60002073657175656E63650A0D3E2000F2CFB3
:102E70000EF0F29EF76A8C0FF66E2E0EF722000E01
:102E8000F86E0900F5500EBEF28E12000A0D3E20BB
:102E90004A6F79737469636B2050616E2053656E5D
:102EA0007369746976697479202564200A0D3E205F
:102EB0000000F2CF0EF0F29EF76AD00FF66E2E0EE3
:102EC000F722000EF86E0900F5500EBEF28E1200C9
:102ED0000A0D3E53657444656661756C7420256403
:102EE000200A0D3E2000F2CF0EF0F29EF76A040F8A
:102EF000F66E2F0EF722000EF86E0900F5500EBE8A
:102F0000F28E12000A0D3E44656661756C74436171
:102F10006D202564200A0D3E2000F2CF0EF0F29EB7
:102F2000F76A380FF66E2F0EF722000EF86E0900C2
:102F3000F5500EBEF28E12000A0D3E204A6F7973D4
:102F40007469636B2054696C742053656E73697483
:102F50006976697479202564200A0D3E2000F2CF3D
:102F60000EF0F29EF76A7C0FF66E2F0EF722000E1F
:102F7000F86E0900F5500EBEF28E120050726F63AB
:102F80006573732055313320254C5820254C580A41
:102F90000D00F2CF0EF0F29EF76AB00FF66E2F0E14
:102FA000F722000EF86E0900F5500EBEF28E1200E8
:102FB00050726F636573732055313420254C58204F
:102FC000254C580A0D00F2CF0EF0F29EF76AE40F7E
:102FD000F66E2F0EF722000EF86E0900F5500EBEA9
:102FE000F28E120020202050726576696577496E56
:102FF000205043200000F2CF0EF0F29EF76A140F2B
:10300000F66E300EF722000EF86E0900F5500EBE77
:10301000F28E120020202050726576696577496E25
:1030200020302000F2CF0EF0F29EF76A420FF66ECB
:10303000300EF722000EF86E0900F5500EBEF28E2B
:10304000120050726576696577496E2025640A0D15
:103050003E00F2CF0EF0F29EF76A700FF66E300E61
:10306000F722000EF86E0900F5500EBEF28E120027
:1030700020202020205043204F757470757420202C
:103080002000F2CF0EF0F29EF76AA00FF66E300E1F
:10309000F722000EF86E0900F5500EBEF28E1200F7
:1030A00020202020204D61696E496E203020202094
:1030B0002000F2CF0EF0F29EF76AD00FF66E300EBF
:1030C000F722000EF86E0900F5500EBEF28E1200C7
:1030D0004D61696E496E2025640A0D3E0000F2CFF5
:1030E0000EF0F29EF76AFC0FF66E300EF722000E1D
:1030F000F86E0900F5500EBEF28E1200202020203E
:103100002043616D2053656C203020202000F2CFD9
:103110000EF0F29EF76A2C0FF66E310EF722000EBB
:10312000F86E0900F5500EBEF28E120043616D6517
:1031300072612025640A0D3E0000F2CF0EF0F29E6F
:10314000F76A580FF66E310EF722000EF86E09007E
:10315000F5500EBEF28E12002043616D2053656C57
:103160002030204E6F2043616D00F2CF0EF0F29EB2
:10317000F76A880FF66E310EF722000EF86E09001E
:10318000F5500EBEF28E120050726F63657373209D
:1031900055313520254C5820254C580A0D00F2CFCA
:1031A0000EF0F29EF76ABC0FF66E310EF722000E9B
:1031B000F86E0900F5500EBEF28E120020496E2006
:1031C00043616D2053746F72652030300000F2CF80
:1031D0000EF0F29EF76AEC0FF66E310EF722000E3B
:1031E000F86E0900F5500EBEF28E1200496E436172
:1031F0006D2053746F72652025640A0D3E00F2CF76
:103200000EF0F29EF76A1C0FF66E320EF722000ED9
:10321000F86E0900F5500EBEF28E120020205265A5
:103220006164696E672043616D6572610000F2CF71
:103230000EF0F29EF76A4C0FF66E320EF722000E79
:10324000F86E0900F5500EBEF28E12002020537465
:103250006F72696E67205072657365740000F2CFFB
:103260000EF0F29EF76A7C0FF66E320EF722000E19
:10327000F86E0900F5500EBEF28E12002053746FE6
:103280007265203030205072657365740000F2CF93
:103290000EF0F29EF76AAC0FF66E320EF722000EB9
:1032A000F86E0900F5500EBEF28E120053746F7264
:1032B000652025640A0D3E00F2CF0EF0F29EF76AFB
:1032C000D60FF66E320EF722000EF86E0900F5509A
:1032D0000EBEF28E12002053746F726520303020C3
:1032E0004661696C65640000F2CF0EF0F29EF76AE9
:1032F000060FF66E330EF722000EF86E0900F55039
:103300000EBEF28E120020496E2043616D20507275
:1033100065736574203030200000F2CF0EF0F29E0D
:10332000F76A380FF66E330EF722000EF86E0900BA
:10333000F5500EBEF28E1200507265736574202532
:10334000640A0D3E0000F2CF0EF0F29EF76A640FA1
:10335000F66E330EF722000EF86E0900F5500EBE21
:10336000F28E120020204C6F6164696E67205072EB
:10337000657365740000F2CF0EF0F29EF76A940F49
:10338000F66E330EF722000EF86E0900F5500EBEF1
:10339000F28E120020202050726573657420303048
:1033A000202020200000F2CF0EF0F29EF76AC40F1A
:1033B000F66E330EF722000EF86E0900F5500EBEC1
:1033C000F28E120020202050726573657420303018
:1033D000204261640000F2CF0EF0F29EF76AF40F13
:1033E000F66E330EF722000EF86E0900F5500EBE91
:1033F000F28E12002020204E6F205072657365748B
:10340000203030200000F2CF0EF0F29EF76A240F39
:10341000F66E340EF722000EF86E0900F5500EBE5F
:10342000F28E120020202050726576696577204F59
:103430006E2020200000F2CF0EF0F29EF76A540FAB
:10344000F66E340EF722000EF86E0900F5500EBE2F
:10345000F28E1200446973706C6179205072657647
:103460006965770A0D3E0000F2CF0EF0F29EF76A12
:10347000860FF66E340EF722000EF86E0900F55036
:103480000EBEF28E1200202020507265766965779C
:10349000204F666620200000F2CF0EF0F29EF76A01
:1034A000B60FF66E340EF722000EF86E0900F550D6
:1034B0000EBEF28E1200446973706C6179204F6603
:1034C000660A0D3E0000F2CF0EF0F29EF76AE40F9E
:1034D000F66E340EF722000EF86E0900F5500EBE9F
:1034E000F28E12002020204D61696E204F6E202048
:1034F0002000F2CF0EF0F29EF76A100FF66E350E36
:10350000F722000EF86E0900F5500EBEF28E120082
:10351000446973706C6179204D61696E0A0D3E00DB
:10352000F2CF0EF0F29EF76A3E0FF66E350EF722DE
:10353000000EF86E0900F5500EBEF28E120020202B
:10354000204D61696E204F6666202000F2CF0EF09C
:10355000F29EF76A6A0FF66E350EF722000EF86ECD
:103560000900F5500EBEF28E120050726F63657343
:10357000732055313620254C5820254C580A0D0013
:10358000F2CF0EF0F29EF76A9E0FF66E350EF7221E
:10359000000EF86E0900F5500EBEF28E12002042A9
:1035A00061636B4C69676874436D70204F66660099
:1035B000F2CF0EF0F29EF76ACE0FF66E350EF722BE
:1035C000000EF86E0900F5500EBEF28E1200424C4D
:1035D00043204F66660A0D3E0000F2CF0EF0F29EC9
:1035E000F76AF80FF66E350EF722000EF86E090036
:1035F000F5500EBEF28E1200204261636B4C69677B
:103600006874436D70204F6E2000F2CF0EF0F29E72
:10361000F76A280FF66E360EF722000EF86E0900D4
:10362000F5500EBEF28E1200424C43204F6E0A0D32
:103630003E00F2CF0EF0F29EF76A500FF66E360E95
:10364000F722000EF86E0900F5500EBEF28E120041
:103650002020204D61696E20456E61626C6564209A
:103660000000F2CF0EF0F29EF76A800FF66E360E73
:10367000F722000EF86E0900F5500EBEF28E120011
:103680002020204D61696E2044697361626C65641D
:103690002000F2CF0EF0F29EF76AB00FF66E360EF3
:1036A000F722000EF86E0900F5500EBEF28E1200E1
:1036B0004D61696E496E20300A0D3E00F2CF0EF06A
:1036C000F29EF76ADA0FF66E360EF722000EF86EEB
:1036D0000900F5500EBEF28E12002020537973209F
:1036E0004D616E75616C204D6F646500F2CF0EF018
:1036F000F29EF76A0A0FF66E370EF722000EF86E8A
:103700000900F5500EBEF28E12005379734D6F64AE
:1037100065204D616E75616C0A0D3E00F2CF0EF0B2
:10372000F29EF76A3A0FF66E370EF722000EF86E29
:103730000900F5500EBEF28E12002020205379733E
:10374000204175746F204D6F64652000F2CF0EF03C
:10375000F29EF76A6A0FF66E370EF722000EF86EC9
:103760000900F5500EBEF28E12005379734D6F644E
:1037700065204175746F0A0D3E00F2CF0EF0F29E87
:10378000F76A980FF66E370EF722000EF86E0900F2
:10379000F5500EBEF28E1200506F776572204F66A4
:1037A000660A0D3E0000F2CF0EF0F29EF76AC40FDB
:1037B000F66E370EF722000EF86E0900F5500EBEB9
:1037C000F28E1200506F776572204F6E0A0D3E0028
:1037D000F2CF0EF0F29EF76AEE0FF66E370EF7227A
:1037E000000EF86E0900F5500EBEF28E1200202079
:1037F0004272696768746E6573732055702020008B
:10380000F2CF0EF0F29EF76A1E0FF66E380EF72218
:10381000000EF86E0900F5500EBEF28E12004272D4
:10382000696768742055700A0D3E0000F2CF0EF0F3
:10383000F29EF76A4A0FF66E380EF722000EF86E07
:103840000900F5500EBEF28E120020204272696708
:1038500068746E65737320446E202000F2CF0EF002
:10386000F29EF76A7A0FF66E380EF722000EF86EA7
:103870000900F5500EBEF28E12004272696768743C
:1038800020446F776E0A0D3E0000F2CF0EF0F29EDC
:10389000F76AA80FF66E380EF722000EF86E0900D0
:1038A000F5500EBEF28E12002020427269676874D5
:1038B0006E657373204175746F00F2CF0EF0F29E47
:1038C000F76AD80FF66E380EF722000EF86E090070
:1038D000F5500EBEF28E1200427269676874204184
:1038E00075746F0A0D3E0000F2CF0EF0F29EF76A7B
:1038F000060FF66E390EF722000EF86E0900F5502D
:103900000EBEF28E120020204272696768746E65E6
:103910007373204D616E2000F2CF0EF0F29EF76AB5
:10392000360FF66E390EF722000EF86E0900F550CC
:103930000EBEF28E1200427269676874204D616E8D
:1039400075616C0A0D3E0000F2CF0EF0F29EF76A30
:10395000660FF66E390EF722000EF86E0900F5506C
:103960000EBEF28E120020202020466F6375732059
:103970004E65617220202000F2CF0EF0F29EF76AB1
:10398000960FF66E390EF722000EF86E0900F5500C
:103990000EBEF28E1200466F637573204E65617223
:1039A0000A0D3E00F2CF0EF0F29EF76AC20FF66EDD
:1039B000390EF722000EF86E0900F5500EBEF28E99
:1039C000120020202020466F63757320466172200C
:1039D00020200000F2CF0EF0F29EF76AF20FF66E92
:1039E000390EF722000EF86E0900F5500EBEF28E69
:1039F0001200466F637573204661720A0D3E000027
:103A0000F2CF0EF0F29EF76A1E0FF66E3A0EF72214
:103A1000000EF86E0900F5500EBEF28E1200202046
:103A20002020466F637573204175746F202000005D
:103A3000F2CF0EF0F29EF76A4E0FF66E3A0EF722B4
:103A4000000EF86E0900F5500EBEF28E1200202016
:103A50002020466F637573204D616E75616C0000A8
:103A6000F2CF0EF0F29EF76A7E0FF66E3A0EF72254
:103A7000000EF86E0900F5500EBEF28E1200466F71
:103A8000637573204175746F0A0D3E00F2CF0EF01E
:103A9000F29EF76AAA0FF66E3A0EF722000EF86E43
:103AA0000900F5500EBEF28E1200204175746F575A
:103AB0006869746542616C204F666600F2CF0EF053
:103AC000F29EF76ADA0FF66E3A0EF722000EF86EE3
:103AD0000900F5500EBEF28E1200415742204F668B
:103AE000660A0D3E0000F2CF0EF0F29EF76A040F58
:103AF000F66E3B0EF722000EF86E0900F5500EBE72
:103B0000F28E1200204175746F57686974654261C6
:103B10006C204F6E2000F2CF0EF0F29EF76A340F49
:103B2000F66E3B0EF722000EF86E0900F5500EBE41
:103B3000F28E1200415742204F6E0A0D3E00F2CF26
:103B40000EF0F29EF76A5C0FF66E3B0EF722000E47
:103B5000F86E0900F5500EBEF28E120053746172B9
:103B6000742049646C652052657475726E205469C6
:103B70006D65720D0A00F2CF0EF0F29EF76A940F97
:103B8000F66E3B0EF722000EF86E0900F5500EBEE1
:103B9000F28E1200205072657365742050474D20DC
:103BA0004D6F64652000F2CF0EF0F29EF76AC40FED
:103BB000F66E3B0EF722000EF86E0900F5500EBEB1
:103BC000F28E1200204C6F6164696E67205072653E
:103BD000736574313200F2CF0EF0F29EF76AF40F83
:103BE000F66E3B0EF722000EF86E0900F5500EBE81
:103BF000F28E1200204E6F20507265736574313260
:103C000020466F756E640000F2CF0EF0F29E240F16
:103C1000F66E3C0EF722000EF86E0900F5500EBE4F
:103C2000F28E120000584001000003000004000062
:103C30000500000600000700000800001000001149
:103C40000000120000140000150000160202171BED
:103C50001B181B1B191F1F1A20201B060620000003
:103C600021000024000025000026FFFF273F3F28F9
:103C70001919291D1D2AFFFF2BFFFF2C0F0F2DB433
:103C8000B43000003100003300003600003800007E
:103C90003900003A151554030355FFFF56FFFF572F
:103CA000FFFF58FBFB59FFFF5A00005B80805CB8A8
:103CB000B85D3A3F5E2E2D5F2E2D607A7A615152AB
:103CC00062463F631FCB647C8A65F00966212A67E0
:103CD000AAAA68AAAA69AAAA6AAAAA6C00006D0080
:103CE000006E00006FD11470FC24719C9C726061A6
:103CF000735454745252750000760606771010788B
:103D000005057910107A0C127B032B7C40407D0056
:103D1000007E00007F000080010181FFFF82FFFF25
:103D2000831F1F90865691795F920D13930D139404
:103D30000E0F95F61896141597FAEA989DA999060C
:103D4000069A00009B00009C08089DFFFF9EFFFF55
:103D50009FFFFFA00000A10000A20707A38080A48E
:103D60008080F0EBEBF1EBEBF2EBEBF31010F410E7
:103D700010F51010F61010F71010F8EBEBF94040AA
:103D8000FA0606FB2C2CFC0000FD939300000000BB
:103D9000F2CF0EF0F29EAC0FF66E3D0EF722000E43
:103DA000F86E0900F5500EBEF28E120000101001E0
:103DB000080702C0C003303204404005D02A064F35
:103DC0004F070000085B1B0940400A7D800B4144FF
:103DD0000C40400D00000E0B0B0F0F0F100E0E11BC
:103DE000000012CFCF13808014040415111116FEA9
:103DF000FE17D8D81840401980801E40401FC0C010
:103E000023030324102A25102A2900002A80802B4E
:103E100048442C40402D00002E40402F808030BC74
:103E2000BC31DFDF32020234CDCD35CCCC363A3A6C
:103E30003803033920203A000040000041FFFF42D0
:103E4000FFFF43FFFF44FFFF45FFFF46FFFF47FF24
:103E5000FF48FFFF49FFFF4AFFFF4BFFFF4CFFFFFB
:103E60004DFFFF4EFFFF4FFFFF50FFFF51FFFF527F
:103E7000FFFF53FFFF54FFFF55FFFF56FFFF57FFA4
:103E8000FF5800005947475A06065B03035C0000D1
:103E90005D00005E00005F00006000006128256298
:103EA000FFEF63000064000065000066000067002B
:103EB0000068000080101081000082000083212132
:103EC00084202085040486454587010188E0E08F31
:103ED00003039000409108089200009300009400B2
:103EE0001295000096D0BC970202980F1A99000014
:103EF0009AF41A9B00019CD0BC9D02029EF4189F6C
:103F00000001A00101A10000A20000A48080A54042
:103F100040A64040A80000A90404AA0000AC00008C
:103F2000AD0202AE0000B00000B10404B20000B364
:103F30000404B40000B82001B92121BA0101BB0179
:103F400001BC2001BD2121BE0101BF0101C0000053
:103F5000C10808C20000C38080C43C3CC50000C644
:103F6000D0D0C70202C80000C90000CA0606CB01B3
:103F700001CCD0D0CD0202CE0606CF0101D0010186
:103F8000D10000D20000D48080D53F3FD63F3FD83B
:103F90000000D90404DA0000DC0000DD0202DE00CB
:103FA00000E00000E10404E20000E30404E4010195
:103FB000E80000E90000EA0000EB0000EC0000ED82
:103FC0000000EE0000EF0000F2CF0EF0F29EF76A64
:103FD000E60FF66E3F0EF722000EF86E0900F55060
:103FE0000EBEF28E120053797374656D20697320D2
:103FF00050414C0A0D00F2CF0EF0F29EF76A140FFA
:10400000F66E400EF722000EF86E0900F5500EBE57
:10401000F28E120053797374656D206973204E54CB
:1040200053430A0D0000F2CF0EF0F29EF76A440FE0
:10403000F66E400EF722000EF86E0900F5500EBE27
:10404000F28E1200436F6D312052656365697665AB
:10405000204572726F722873293D2532780A0D004F
:10406000F2CF0EF0F29EF76A7E0FF66E400EF72248
:10407000000EF86E0900F5500EBEF28E1200436F6E
:104080006D322052656365697665204572726F7284
:104090002873293D2532780A0D00F2CF0EF0F29EEA
:1040A000F76AB80FF66E400EF722000EF86E0900A0
:1040B000F5500EBEF28E12000C2050726F647563C4
:1040C00074696F6E566965772000F2CF0EF0F29E2C
:1040D000F76AE80FF66E400EF722000EF86E090040
:1040E000F5500EBEF28E12000A00F2CF0EF0F29ED4
:1040F000F76A080FF66E410EF722000EF86E0900FF
:10410000F5500EBEF28E1200202053746172746955
:104110006E67205570202000F2CF0EF0F29EF76AF5
:10412000360FF66E410EF722000EF86E0900F550BC
:104130000EBEF28E120043616D6572612050617394
:104140007320436F6D706C6574650A0D0000F2CFCB
:104150000EF0F29EF76A6C0FF66E410EF722000E1B
:10416000F86E0900F5500EBEF28E120043616D65C7
:104170007261205061737320496E636F6D706C655E
:1041800074650A0D0000F2CF0EF0F29EF76AA40FDC
:10419000F66E410EF722000EF86E0900F5500EBEC5
:1041A000F28E120043616D657261204E6F74204182
:1041B0007661696C61626C650A0D0000F2CF0EF0E9
:1041C000F29EF76ADA0FF66E410EF722000EF86ED5
:1041D0000900F5500EBEF28E120050726F647563C6
:1041E00074696F6E5669657725730A0D0000F2CF0A
:1041F0000EF0F29EF76A0C0FF66E420EF722000EDA
:10420000F86E0900F5500EBEF28E1200202020201C
:10421000436F6D70696C65643A202573206174206A
:1042200025730A0D3E00F2CF0EF0F29EF76A440F9E
:10423000F66E420EF722000EF86E0900F5500EBE23
:10424000F28E12002046696E64696E672043616DCC
:10425000657261730000F2CF0EF0F29EF76A740F80
:10426000F66E420EF722000EF86E0900F5500EBEF3
:10427000F28E120020436C65617220507265736586
:10428000747320200000F2CF0EF0F29EF76AA40FA4
:10429000F66E420EF722000EF86E0900F5500EBEC3
:1042A000F28E120020436C656172696E6720416C6A
:1042B0006C2020200000F2CF0EF0F29EF76AD40F9F
:1042C000F66E420EF722000EF86E0900F5500EBE93
:1042D000F28E1200446F44756D700000F2CF0EF044
:1042E000F29EF76AFA0FF66E420EF722000EF86E93
:1042F0000900F5500EBEF28E1200456E61626C65CB
:104300002053657269616C0A0D00F2CF0EF0F29EC7
:10431000F76A280FF66E430EF722000EF86E0900BA
:10432000F5500EBEF28E120020204E6F74206F6E7C
:1043300020507265736574200000F2CF0EF0F29E7B
:10434000F76A580FF66E430EF722000EF86E09005A
:10435000F5500EBEF28E1200204C6F6164696E67DC
:104360002044656661756C747300F2CF0EF0F29EA6
:10437000F76A880FF66E430EF722000EF86E0900FA
:10438000F5500EBEF28E12002020506F77657269D4
:104390006E672055702020200000F2CF0EF0F29EB4
:1043A000F76AB80FF66E430EF722000EF86E09009A
:1043B000F5500EBEF28E12000C50726F647563746D
:1043C000696F6E5669657700F2CF0EF0F29EF76A5C
:1043D000E60FF66E430EF722000EF86E0900F55058
:1043E0000EBEF28E12000A2020506F776572696E41
:1043F0006720446F776E2000C69E9E9652CDC9FFFF
:10440000020EC6BE05D09EA6FED7000EC5BC010E8C
:10441000016E000CC586C5B6FED700B0C59A00A0D7
:10442000C58AC588C5B8FED7C9CF01F0000C0D01FB
:104430004B6BC580C5B0FED70D0E006E002EFED7AB
:104440004951FE0B4C6F526F0001D6DF0D0E006E0E
:10445000002EFED74ACD52FDCFDF0D0E006E002E8E
:10446000FED7C582C5B2FED70D0E006E002EFED758
:104470000D01495101094C6F526F0001BDDF0D0E56
:10448000006E002EFED7006AC5DF01C04BFD0D0E89
:10449000006E002EFED7C584C5B4FED70F0E006E89
:1044A000002EFED700D00D014BCD01F00001000C15
:1044B0000D01456B466B476B4451FE0B486F43CD76
:1044C00049FD4A6F0001B3DF01C047FD0D014451B2
:1044D0000109486F43CD49FD4A6F0001A8DF01C0C3
:1044E00046FD0D01456B4751451345CD01F046CDC5
:1044F00002F00001000C0D01416B426B4C80400E3C
:10450000436F080E446F0001D3DF02C042FD01C0BB
:1045100041FDF292DEEF03F00D01416B426B4C82E4
:10452000440E436F080E446F0001C2DF02C042FD1B
:1045300001C041FDF092DEEF03F00D01416B426BD3
:104540004C84420E436F080E446F0001B1DF02C07D
:1045500042FD01C041FDF090DEEF03F00D01416B23
:10456000426B4C86460E436F080E446F0001A0DF7D
:1045700002C042FD01C041FDF094DEEF03F00D01E9
:104580004451016A435D03E243CD00F00CD0006A60
:10459000080E456F433700364451005CD8B0006EBA
:1045A0000136452FF7D70001000C01012151040D00
:1045B000F3500D01426B416F036A010131510D014E
:1045C0004125016E425103220150250FE96E010E73
:1045D0000320EA6EC282C2B2FED7C4CFEFFF010150
:1045E0002151040DF3500D01426B416F036A01012B
:1045F00031510D014125016E425103220150250F19
:10460000E96E010E0320EA6EEF507B0827E20101FC
:104610002151040DF3500D01456B446F036A0101F4
:1046200031510D014425016E455103220150250FE2
:10463000E96E010E0320EA6EEF5084080FE3D89074
:1046400001012135036A320FE96E010E0320EA6E83
:10465000EC6AED52800EEF6E7DD00D01D890010115
:104660002135036A320F016E010E032201C041FDA4
:1046700003C042FD01012151040DF3500D01446BB3
:10468000436F250E4325E96E010E4421EA6EEF507B
:10469000466B456F01012151040DF3500D01486B2C
:1046A000476F010E4725016E000E4821036E015031
:1046B000250FE96E010E0320EA6EEF50036A4525CF
:1046C000496F035046214A6F01012151040DF350F7
:1046D0000D014C6B4B6F020E4B25016E000E4C21F1
:1046E000036E0150250FE96E010E0320EA6EEF50B4
:1046F000036A49254D6F03504A214E6F0101215134
:10470000040DF3500D01506B4F6F030E4F25016EDA
:10471000000E5021036E0150250FE96E010E03209B
:10472000EA6EEF50036A4D25516F03504E21526FD0
:104730005231036E5131026E033202323F0E0316C4
:1047400042CDEAFF41CDE9FF03C0ECFFED5202C0CC
:10475000EFFF0101010E3125030B316F010E212501
:104760000D01426F436F030E446F000108DF00C06C
:1047700021F101012135006E0036FC0E0016C250F9
:10478000C30B0010C26E5D2E1FD05C2A5E2A1B0E6A
:104790005D6E5BA80FD00001600760530AE15B9873
:1047A0003BC18BF13CC18CF13BC18AF14A804A820A
:1047B000498C010158BE02D05BA006D05E500308B0
:1047C00003E2589E5B90458A9E900001DEEF03F065
:1047D000F294DEEF03F0C580C5B0FED70D0E006E7B
:1047E000002EFED70D014E51FE0B516F526F00018E
:1047F00003DE0D0E006E002EFED74FCD52FDFCDD08
:104800000D0E006E002EFED750CD52FDF5DD0D0EC3
:10481000006E002EFED7C584C5B4FED70F0E006E05
:10482000002EFED700D0000C0D0146510109496F42
:1048300048CD4AFD4B6B48CD4CFD4D6B45CD4EFDF3
:104840004F6F48CD50FD0001C6DF0D014651FE0BF4
:10485000496F47CD4AFD4B6B45CD4EFD4F6F47CD60
:1048600050FD0001B8DF000C0D01466B476B010ED7
:10487000455DF40F51E20C0F000192EF24F00D01A1
:10488000476B080E466F48D00D01476B040E466F0C
:1048900043D0010138A105D00D01476B010E466FD1
:1048A00004D00D01476B020E466F36D0010138A1CE
:1048B00005D00D01476B020E466F04D00D01476B0A
:1048C000010E466F29D0800E0D01476F466B24D034
:1048D000400E0D01476F466B1FD0200E0D01476F34
:1048E000466B1AD0100E0D01476F466B15D0080E9F
:1048F0000D01476F466B10D0040E0D01476F466BDC
:104900000BD0020E0D01476F466B06D0010E0D0154
:10491000476F466B01D00D0146CD01F047CD02F047
:104920000001000C0DAE03D0F2CF0EF0F29EE82491
:10493000F76AF736570FF66E490EF722000EF86E3B
:10494000FB6E0A00F550FA6E0800F5500DAE02D06D
:104950000EBEF28EF96E0C490249F848EE48E44862
:10496000DA48D048C648AC48924888487E480D018D
:10497000466B476B455102080EE3010E455D006E24
:10498000400E466F476B005205E0D89046374737D8
:10499000002EFBD721D0455104080EE3030E455DE0
:1049A000006E400E476F466B005205E0D8904637C8
:1049B0004737002EFBD710D0455106080DE3050EF2
:1049C000455D006E400E466F476B005205E0D89083
:1049D00046374737002EFBD746CD01F047CD02F0D2
:1049E0000001000C0D01416B426B436B446B58AAF4
:1049F00003D0589CA08283D1A092588C58A062D03A
:104A00004F504D14456F50504E14466F455304E1BE
:104A1000465302E158A20BD04D50FF0A006E4E5093
:104A2000FF0A036E00504F160350501604D04D502D
:104A30004F124E5050125150010A000105E0030A76
:104A40000EE0010A1CE026D04C0E0D01456F466BAE
:104A500050C048FD4FC047FD0001E6DE1DD050C0EC
:104A600045FD0D01466B50C047FD486B480E4E6F2B
:104A7000010E4F6F50C050FD0001ADDE0DD04A0E4B
:104A80000D01456F466B50C048FD4FC047FD00010A
:104A9000CBDE02D0588200D058A205D0516A506AAD
:104AA0004F6A5890589258A006D0A082589C0D0189
:104AB00026D108D0000158B406D0589C5894589676
:104AC0000D011DD1000158A607D0589458960D012C
:104AD000416B596A14D1000158A40ED15952D8B46F
:104AE0000BD10D01416B59C044FD44510C080EE33C
:104AF000036A4451CF0FE96E010E0320EA6EEF52B4
:104B000003E144CD41FD02D0442BEFD7415318E1DE
:104B1000592C01D015D0010E596E59C044FD445195
:104B20000C080EE3036A4451CF0FE96E010E032017
:104B3000EA6EEF5203E144CD41FD02D0442BEFD7A2
:104B40004153D8B475D0FF0E521A531A300E521674
:104B5000536A41515A5C02E1587801D0589858B8CC
:104B600008D041CD45FD00017FDE015052120250B8
:104B7000531285C145FD0001FADE02C043FD01C0AC
:104B800042FD0101855102081AE30D0142515614FC
:104B9000456F43515714466F45530BE1465309E1A6
:104BA000425152124351531242515612435157121D
:104BB00004D03F0E5216576A566A27D00101FF0EE5
:104BC000541A551A54500D014215456F555043154E
:104BD000466F45530AE1465308E13F0E54165516F9
:104BE000425154124351551203D03F0E54165516DC
:104BF000FF0E541A551A4A0E456F466B55C048FDB4
:104C000054C047FD000110DE0D01FF0E521A531A69
:104C10004C0E456F466B53C048FD52C047FD000126
:104C200003DE41CD5AF0010E0D014125596E5ED0D3
:104C3000592C5CD0FF0E521A531AF00E5216536ABA
:104C400085C145FD000193DE02C043FD01C042FD68
:104C500001018551020824E352500D014215456FB0
:104C600053504315466F45530AE1465308E1300E51
:104C70005216536A425152124351531203D0300E0E
:104C80005216536AFF0E521A531A4C0E456F466B5A
:104C900053C048FD52C047FD0001C6DD26D00101CA
:104CA000FF0E541A551A54500D014215456F5550B8
:104CB0004315466F45530AE1465308E13F0E54162B
:104CC0005516425154124351551203D03F0E5416FB
:104CD0005516FF0E541A551A4A0E456F466B55C0AD
:104CE00048FD54C047FD00019FDD0D0144510C08F3
:104CF00002E2010E596E0001589CA0820D01A192A2
:104D00000001DEEF03F0036A6151680FE96E000EE7
:104D10000320EA6E9EAAFED7AECFEFFF036A615171
:104D2000680FE96E000E0320EA6E6751EF5C01E147
:104D3000662B010E61253F0B616F5B9E01013ABD41
:104D400004D061C063F05B8C01D05B9C9E9A000133
:104D5000DEEF03F0036A6251A90FE96E000E032033
:104D6000EA6EA4AAFED76ECFEFFF010E62250D01F9
:104D7000426F436F780E446F000101DC00C062F0A7
:104D8000A891A49ADEEF03F0070EEA6ECE0EE96E4C
:104D9000EF500EE0050E016E006A002EFED7012EC8
:104DA000FBD72E0E006E002EFED700D0EF2EF2D7CE
:104DB000000C080EEA6E110EE96EEF500EE0050EC3
:104DC000016E006A002EFED7012EFBD72E0E006E5C
:104DD000002EFED700D0EF2EF2D7000C08011639B6
:104DE000F00B006E0F0E83140010836E00008380A2
:104DF000020E006E002EFED7000083900001000C12
:104E0000F00E956E838400008380000083380F0BC2
:104E10000801166F83900000838000D000D0833893
:104E20000F0B156F8390000E956E1639006EF00E05
:104E3000001600501511016E000121EF27F083923A
:104E4000DFD701C015F8080101AE02D00001F8D784
:104E500013A1839213B18382000083940000839096
:104E60001439156F0F0E151715C816F80001B6DFA7
:104E7000080114510F0B156F166F0001AFDF000C06
:104E8000000E956E8392839483900F0E0801116F2C
:104E900000018FDF010E0401336F335103080DE36E
:104EA000030E0801166F000199DF050E0801116F4E
:104EB00000017FDF0401332BF0D7020E0801166FCB
:104EC00000018CDF0401336B3351030814E3036AE0
:104ED0003351F2CF34F4F29E000103EC04F00401EC
:104EE00034BFF28E356F0801136B146F0001A7DF1A
:104EF0000401332BE9D70001BDEFE6F00EC810F82E
:104F00000DC80FF810C803F008010FC8E9FF10C85A
:104F1000EAFFEF5206E00F2BD8B4102B0001F2D7B6
:104F200008010D510F5D006E0E511059036E00C047
:104F300001F0026E0001000C0801102D01D003D019
:104F4000400E116F01D0116B010E0F5D1127115131
:104F50008009126F136B146F000171DF000C0801E0
:104F60000E510C0A000105E0060A0FE0020A15E0E6
:104F70001BD00801136B010E146F000160DF020EDD
:104F80000801116F000115DF17D0010E08010F6F26
:104F9000020E106F0001D0DF0FD00801136B100E4E
:104FA000146F00014CDF08D0010E0801136F0EC80A
:104FB00014F8000144DF00D0000C08010C6B0BC892
:104FC0000EF80AC80DF8000199DF02C00EF801C002
:104FD0000DF808010D5303E10E53D8B495D00BC85A
:104FE0000EF80AC80DF8000189DF02C003F0015075
:104FF000035206E1015008010C5DD8B085D00001D4
:10500000036A08010C510A25E96E0B510320EA6E70
:10501000EF50010A00010DE0030A26E0010A3FE01B
:10502000080A58E0070A5EE0060A5CE0020A5AE055
:1050300059D008010C5317E1010E0F6F106F0001DA
:105040007BDF200E08010E6F000189DF010E0801D1
:105050000F6F020E106F00016FDF200E08010E6F40
:1050600000017DDF08014ED008010C5317E1010E4D
:105070000F6F106F000160DF3E0E08010E6F000120
:105080006EDF010E08010F6F020E106F000154DF7A
:10509000200E08010E6F000162DF080133D0080105
:1050A0000C5317E1010E0F6F106F000145DF200E4A
:1050B00008010E6F000153DF010E08010F6F020E91
:1050C000106F000139DF3E0E08010E6F000147DF4F
:1050D000080118D0010E08010F6F106F00012CDFBE
:1050E000080110D0036A08010C510A25E96E0B5122
:1050F0000320EA6EEFCF0DF80DC80EF800012FDF88
:10510000080100D00C2B6BD70001000C08010B67C5
:1051100003D00C6702D007D00C2B0AC8EEFF0B2F70
:10512000FCD70C2FFAD70001000C196AF2BE198EB9
:10513000F29E67C449FD68C44AFD17EC22F019BE0F
:10514000F28E0150000C0701CEC7E9FFCFC7EAFF7E
:10515000EFCFD2F7D1C703F0D0C7E9FFD1C7EAFF3D
:10516000EF50D25D48E0CFC703F0CEC7E9FFCFC70D
:10517000EAFFEFCFD3F7D351400803E2D3515A08E7
:1051800006E2D35160084CE2D3517A0849E3D1C713
:1051900003F0D0C7E9FFD1C7EAFFEFCFD4F7D4516E
:1051A000400803E2D4515A0806E2D451600838E2BC
:1051B000D4517A0835E3CEC7E9FFCFC7EAFFEFCF76
:1051C000D5F7D1C703F0D0C7E9FFD1C7EAFF200E5A
:1051D000EF24D55D10E0D0C7E9FFD1C7EAFFEFCFDC
:1051E000D7F7CFC703F0CEC7E9FFCFC7EAFF200E3E
:1051F000EF24D75D15E1CFC703F0CEC7E9FFCFC7D6
:10520000EAFFEF5203E1000E016E1FD0CFC703F09B
:10521000CE51CE2BD8B4CF2BD02BD8B4D12B94D702
:10522000CFC703F0CEC7E9FFCFC7EAFFEFCFD2F772
:10523000D1C703F0D0C7E9FFD1C7EAFFEF50D25D75
:1052400002E2FF0E01D0010E016E0001000C500EB3
:105250000401506F410E516F4C0E526F200E536F70
:10526000546B556B040EEA6E4B0EE96E08010A6B27
:105270000C6B050E0B6F000149DF0401556B555196
:10528000030819E3036A55514B0F016E040E032204
:1052900001C056F403C057F4A00E676F55C468F4FC
:1052A000000143DF57C4EAFF56C4E9FF01C0EFFF26
:1052B0000401552BE4D7040E0701CF6F4B0ECE6FC0
:1052C000040ED16F500ED06F00013DDF01521DE181
:1052D00004014A2D15D0010139B502D0040110D0C6
:1052E0000401566B56510001E4EC1FF00401562BEB
:1052F000006E00509EA8FED7AD6E0F0E565DF2E117
:10530000010E016E1DD01CD0000104014A2D15D0E4
:10531000010139B502D0040110D00401566B565179
:105320000001FBEC1FF00401562B006E00509EA8FC
:10533000FED7AD6E100E565DF2E1000E016E00D08C
:105340000001000C0D013C513E03F3CF01F0F4CFFE
:1053500000F03F03F35000263D513E03F350002080
:10536000026E0001000C080E016E0A0E006E002E87
:10537000FED78E9C979C0A0E006E002EFED704016D
:105380006F378E9ED8B0978ED8A0979E978C85AC9D
:10539000FED7012E01D002D00001E7D70A0E006E21
:1053A000002EFED78E9C979C0000978E0A0E006EF2
:1053B000002EFED70A0E006E002EFED7978C85AC0D
:1053C000FED7016A0A0E006E002EFED785BE018050
:1053D0008E9C979C8E9E979E0001000C978E0A0EC5
:1053E000006E002EFED7978C0A0E006E002EFED7A0
:1053F0008E9E979E0A0E006E002EFED78E9C979C66
:1054000004016B51FE0B6E6F6F6F0001ACDF6CC45B
:105410006FF4A9DF6DC46FF4A6DF979E0000978C30
:1054200085ACFED70A0E006E002EFED700D000001D
:10543000978E0A0E006E002EFED71D0E006E002EF7
:10544000FED700D02BEF2AF067C46BF468C46CF46D
:1054500069C46DF4C3D7000C0401336B346B010EC7
:10546000356F4A6B0001F3DE012C02D00401352BAD
:105470000401346B336B345351E13351B3084EE3C1
:1054800034C43DFD33C43CFD0D013F6B030E3E6F44
:10549000000158DF02C037F401C036F402C003F047
:1054A00004010150F2CF38F4F29E02C0F7FF000170
:1054B000C8EC1EF0040138BFF28E396F34C43DFDD4
:1054C00033C43CFD0D013F6B030E3E6F00013ADF1C
:1054D00002C03BF401C03AF4040135510124016ECD
:1054E000000E0220036E0150F2CF3CF4F29E03C086
:1054F000F7FF0001C8EC1EF004013CBFF28E3D6FC7
:10550000400E676F39C468F46A6B3DC469F40001EA
:105510009BDF0401332BD8B4342BADD7346B336B02
:10552000345351E1335178084EE334C43DFD33C464
:105530003CFD0D013F6B030E3E6F000103DF02C017
:1055400037F401C036F402C003F004010150F2CF79
:1055500038F4F29E02C0F7FF000104EC1EF00401D3
:1055600038BFF28E396F34C43DFD33C43CFD0D01AC
:105570003F6B030E3E6F0001E5DE02C03BF401C04D
:105580003AF4040135510124016E000E0220036E2D
:105590000150F2CF3CF4F29E03C0F7FF000104EC8F
:1055A0001EF004013CBFF28E3D6F880E676F39C458
:1055B00068F46A6B3DC469F4000146DF0401332BD3
:1055C000D8B4342BADD70001B0EF2BF0196AF2BE7E
:1055D000198EF29E67C44EFD68C44FFD69C450FD2C
:1055E000EBEC23F019BEF28E000C0401336B346B2C
:1055F000010E356F4A6B00012ADE012C02D0040136
:10560000352B0401346B336B345351E13351B30800
:105610004EE334C43DFD33C43CFD0D013F6B030E2E
:105620003E6F00018FDE02C037F401C036F402C0C5
:1056300003F004010150F2CF38F4F29E02C0F7FFEC
:105640000001C8EC1EF0040138BFF28E396F34C47B
:105650003DFD33C43CFD0D013F6B030E3E6F000169
:1056600071DE02C03BF401C03AF40401355101245B
:10567000016E000E0220036E0150F2CF3CF4F29E48
:1056800003C0F7FF0001C8EC1EF004013CBFF28E1E
:105690003D6F420E676F39C468F46A6B3DC469F4AC
:1056A0000001D2DE0401332BD8B4342BADD7346BD8
:1056B000336B345351E1335178084EE334C43DFD2C
:1056C00033C43CFD0D013F6B030E3E6F00013ADE1B
:1056D00002C037F401C036F402C003F004010150E7
:1056E000F2CF38F4F29E02C0F7FF000104EC1EF086
:1056F000040138BFF28E396F34C43DFD33C43CFD24
:105700000D013F6B030E3E6F00011CDE02C03BF437
:1057100001C03AF4040135510124016E000E02204B
:10572000036E0150F2CF3CF4F29E03C0F7FF00017C
:1057300004EC1EF004013CBFF28E3D6F880E676FD3
:1057400039C468F46A6B3DC469F400013FDF0401A9
:10575000332BD8B4342BADD70001B1EF2BF07CD66E
:1057600044D7010E016EFFEFE6F0196AF2BE198E02
:10577000F29E4C0E0D01456F040E466F486B476B51
:10578000000114EC24F019BEF28E196AF2BE198ED3
:10579000F29E4C0E0D01456F060E466F486B476B2F
:1057A000000114EC24F019BEF28E196AF2BE198EB3
:1057B000F29E4C0E0D014E6F0B0E4F6F506B0001A1
:1057C000EBEC23F019BEF28E196AF2BE198EF29E2E
:1057D000480E0D01456F040E466F486B476B000184
:1057E00014EC24F019BEF28E196AF2BE198EF29EE4
:1057F000480E0D01456F060E466F486B476B000162
:1058000014EC24F019BEF28E196AF2BE198EF29EC3
:10581000480E0D014E6F0A0E4F6F506B0001EBECFE
:1058200023F019BEF28E196AF2BE198EF29E4A0E4C
:105830000D01456F040E466F486B476B000114EC79
:1058400024F019BEF28E196AF2BE198EF29E4A0E2B
:105850000D01456F060E466F486B476B000114EC57
:1058600024F019BEF28E196AF2BE198EF29E4A0E0B
:105870000D014E6F0A0E4F6F506B0001EBEC23F0E1
:1058800019BEF28E196AF2BE198EF29E4E0E0D01ED
:10589000456F040E466F486B476B000114EC24F013
:1058A00019BEF28E196AF2BE198EF29E4E0E0D01CD
:1058B000456F060E466F486BFF0E476F000114ECF4
:1058C00024F019BEF28E196AF2BE198EF29E4E0EA7
:1058D0000D014E6F0A0E4F6F506B0001EBEC23F081
:1058E00019BEF28E196AF2BE198EF29E400E0D019B
:1058F000456F040E466F486B476B000114EC24F0B3
:1059000019BEF28E196AF2BE198EF29E400E0D017A
:10591000456F060E466FFF0E486F476F000114EC8F
:1059200024F019BEF28E196AF2BE198EF29E400E54
:105930000D014E6F0A0E4F6F506B0001EBEC23F020
:1059400019BEF28E196AF2BE198EF29E440E0D0136
:10595000456F040E466F486B476B000114EC24F052
:1059600019BEF28E196AF2BE198EF29E440E0D0116
:10597000456F060E466FFF0E486F476F000114EC2F
:1059800024F019BEF28E196AF2BE198EF29E440EF0
:105990000D014E6F0A0E4F6F506B0001EBEC23F0C0
:1059A00019BEF28E196AF2BE198EF29E420E0D01D8
:1059B000456F040E466F486B476B000114EC24F0F2
:1059C00019BEF28E196AF2BE198EF29E420E0D01B8
:1059D000456F060E466FFF0E486F476F000114ECCF
:1059E00024F019BEF28E196AF2BE198EF29E420E92
:1059F0000D014E6F0A0E4F6F506B0001EBEC23F060
:105A000019BEF28E196AF2BE198EF29E460E0D0173
:105A1000456F040E466F486B476B000114EC24F091
:105A200019BEF28E196AF2BE198EF29E460E0D0153
:105A3000456F060E466FFF0E486F476F000114EC6E
:105A400024F019BEF28E196AF2BE198EF29E460E2D
:105A50000D014E6F0A0E4F6F506B0001EBEC23F0FF
:105A600019BEF28E000C04016851010A00010AE01F
:105A7000030AD8B4F6D0010AD8B4BAD1030AD8B40C
:105A80007ED27DD2010EEA6EDC0EE96EF2CF69F4B1
:105A9000F29E000EA5EC08F00A000900F550EE6E2B
:105AA0000009FBE1040169BFF28E010EEA6EEE0E01
:105AB000E96EF2CF69F4F29E000E0001BDEC08F031
:105AC0000A000900F550EE6E0009FBE1040169BF10
:105AD000F28E020EEA6EE96AF2CF69F4F29E000ECF
:105AE0000001D5EC08F00A000900F550EE6E00093F
:105AF000FBE1040169BFF28E020EEA6E120EE96E3E
:105B0000F2CF69F4F29E000E0001EDEC08F00A00FD
:105B10000900F550EE6E0009FBE1040169BFF28E49
:105B2000020EEA6E240EE96EF2CF69F4F29E000EC8
:105B3000000105EC09F00A000900F550EE6E0009BD
:105B4000FBE1040169BFF28E020EEA6E360EE96EC9
:105B5000F2CF69F4F29E000E00011DEC09F00A007C
:105B60000900F550EE6E0009FBE1040169BFF28EF9
:105B7000020EEA6E480EE96EF2CF69F4F29E000E54
:105B8000000135EC09F00A000900F550EE6E00093D
:105B9000FBE1040169BFF28E020EEA6E5A0EE96E55
:105BA000F2CF69F4F29E000E00014DEC09F00A00FC
:105BB0000900F550EE6E0009FBE1040169BFF28EA9
:105BC000020EEA6E6C0EE96EF2CF69F4F29E000EE0
:105BD000000165EC09F00A000900F550EE6E0009BD
:105BE000FBE1040169BFF28E020EEA6E7E0EE96EE1
:105BF000F2CF69F4F29E000E00017DEC09F00A007C
:105C00000900F550EE6E0009FBE1040169BFF28E58
:105C1000020EEA6E900EE96EF2CF69F4F29E000E6B
:105C2000000195EC09F00A000900F550EE6E00093C
:105C3000FBE1040169BFF28E010E0301326F036ABA
:105C400032513B0FE96E030E0320EA6E0A0EEF6E2F
:105C5000036A32513F0FE96E030E0320EA6EEF6ACA
:105C60007ED2010EEA6EDC0EE96EF2CF69F4F29E8E
:105C7000000EADEC09F00A000900F550EE6E0009C7
:105C8000FBE1040169BFF28E010EEA6EEE0EE96ED1
:105C9000F2CF69F4F29E000E0001C5EC09F00A0093
:105CA0000900F550EE6E0009FBE1040169BFF28EB8
:105CB000020EEA6EE96AF2CF69F4F29E000E00016C
:105CC000DDEC09F00A000900F550EE6E0009FBE179
:105CD000040169BFF28E020EEA6E120EE96EF2CF77
:105CE00069F4F29E000E0001F5EC09F00A000900CB
:105CF000F550EE6E0009FBE1040169BFF28E020E61
:105D0000EA6E240EE96EF2CF69F4F29E000E0001F5
:105D10000DEC0AF00A000900F550EE6E0009FBE1F7
:105D2000040169BFF28E020EEA6E360EE96EF2CF02
:105D300069F4F29E000E000125EC0AF00A00090049
:105D4000F550EE6E0009FBE1040169BFF28E020E10
:105D5000EA6E480EE96EF2CF69F4F29E000E000181
:105D60003DEC0AF00A000900F550EE6E0009FBE177
:105D7000040169BFF28E020EEA6E5A0EE96EF2CF8E
:105D800069F4F29E000E000155EC0AF00A000900C9
:105D9000F550EE6E0009FBE1040169BFF28E020EC0
:105DA000EA6E6C0EE96EF2CF69F4F29E000E00010D
:105DB00095EC09F00A000900F550EE6E0009FBE1D0
:105DC000040169BFF28E020E0301326F036A325181
:105DD0003B0FE96E030E0320EA6E080EEF6E036AB6
:105DE00032513F0FE96E030E0320EA6EEF6AB7D11E
:105DF000010EEA6EDC0EE96EF2CF69F4F29E000E3F
:105E00006DEC0AF00A000900F550EE6E0009FBE1A6
:105E1000040169BFF28E010EEA6EEE0EE96EF2CF5A
:105E200069F4F29E000E0001C5EC09F00A000900B9
:105E3000F550EE6E0009FBE1040169BFF28E020E1F
:105E4000EA6EE96AF2CF69F4F29E000E0001DDEC21
:105E500009F00A000900F550EE6E0009FBE10401AB
:105E600069BFF28E020EEA6E120EE96EF2CF69F48D
:105E7000F29E000E0001F5EC09F00A000900F55051
:105E8000EE6E0009FBE1040169BFF28E020EEA6EBC
:105E9000240EE96EF2CF69F4F29E000E00010DECC3
:105EA0000AF00A000900F550EE6E0009FBE104015A
:105EB00069BFF28E020EEA6E360EE96EF2CF69F419
:105EC000F29E000E000125EC0AF00A000900F550D0
:105ED000EE6E0009FBE1040169BFF28E020EEA6E6C
:105EE000480EE96EF2CF69F4F29E000E00013DEC1F
:105EF0000AF00A000900F550EE6E0009FBE104010A
:105F000069BFF28E020EEA6E5A0EE96EF2CF69F4A4
:105F1000F29E000E000155EC0AF00A000900F5504F
:105F2000EE6E0009FBE1040169BFF28E020EEA6E1B
:105F30006C0EE96EF2CF69F4F29E000E000195EC52
:105F400009F00A000900F550EE6E0009FBE10401BA
:105F500069BFF28E030E0301326F036A32513B0FA9
:105F6000E96E030E0320EA6E080EEF6E036A3251EB
:105F70003F0FE96E030E0320EA6EEF6AF0D0010EC8
:105F8000EA6EDC0EE96EE26A320EE16EE752E6CFAF
:105F9000EEFFFCE1010EEA6EEE0EE96EE26A200E03
:105FA000E16EE752E6CFEEFFFCE1020EEA6EE96A2F
:105FB000F2CF69F4F29E000E85EC0AF00A000900A7
:105FC000F550EE6E0009FBE1040169BFF28E020E8E
:105FD000EA6E120EE96EF2CF69F4F29E000E000135
:105FE0009DEC0AF00A000900F550EE6E0009FBE195
:105FF000040169BFF28E020EEA6E240EE96EF2CF42
:1060000069F4F29E000E0001B5EC0AF00A000900E6
:10601000F550EE6E0009FBE1040169BFF28E020E3D
:10602000EA6E360EE96EF2CF69F4F29E000E0001C0
:10603000CDEC0AF00A000900F550EE6E0009FBE114
:10604000040169BFF28E020EEA6E480EE96EF2CFCD
:1060500069F4F29E000E0001E5EC0AF00A00090066
:10606000F550EE6E0009FBE1040169BFF28E020EED
:10607000EA6E5A0EE96EF2CF69F4F29E000E00014C
:10608000FDEC0AF00A000900F550EE6E0009FBE194
:10609000040169BFF28E020EEA6E6C0EE96EF2CF59
:1060A00069F4F29E000E000115EC0BF00A000900E5
:1060B000F550EE6E0009FBE1040169BFF28E020E9D
:1060C000EA6E7E0EE96EF2CF69F4F29E000E0001D8
:1060D000ADEC09F00A000900F550EE6E0009FBE195
:1060E000040169BFF28E020EEA6E900EE96EF2CFE5
:1060F00069F4F29E000E00012DEC0BF00A0009007D
:10610000F550EE6E0009FBE1040169BFF28E020E4C
:10611000EA6EA20EE96EF2CF69F4F29E000E000163
:106120006DEC0AF00A000900F550EE6E0009FBE183
:10613000040169BFF28E0301326B036A32513B0FD7
:10614000E96E030E0320EA6E110EEF6E036A325100
:106150003F0FE96E030E0320EA6EEF6A00D00001E4
:10616000000C0BC810F80AC80FF808010E5324E001
:106170000DC803F00CC8E9FF0DC8EAFFEF521CE0A0
:1061800010C803F00F510F2BD8B4102B116F03C0A0
:1061900012F80DC803F00C510C2BD8B40D2BE96E7E
:1061A00003C0EAFFEFCF13F812C8EAFF11C8E9FFF6
:1061B00013C8EFFF0E07DAD70E530CE010C803F038
:1061C0000F510F2BD8B4102BE96E03C0EAFFEF6A12
:1061D0000E07F2D70AC801F00BC802F00001000C4C
:1061E000A8B362D0070EEA6EE40EE96E08010A6BEE
:1061F0000C6B130E0B6F000186EC28F0A8A936D0AB
:10620000040119A304D019A502D000012FD0010167
:1062100038A516D0070EEA6EE40EE96EF2CF0AF842
:10622000F29E000E00010AEC0DF00A000900F55084
:10623000EE6E0009FBE108010ABFF28E15D00101E4
:10624000070EEA6EE40EE96EF2CF0AF8F29E000E37
:10625000000122EC0DF00A000900F550EE6E000975
:10626000FBE108010ABFF28E0ED00001070E080103
:106270000B6FE40E0A6F010E0D6FDC0E0C6F120E29
:106280000E6F00016EDF0C0E0701E46F070E0801B0
:106290000B6FE40E0A6F0001DDEC27F0050E08011C
:1062A000116F0001D9EC26F0070EEA6EF70EE96EC9
:1062B00008010A6B0C6B130E0B6F000186EC28F0C3
:1062C000070E08010B6FF70E0A6FE3C70DF8E2C760
:1062D0000CF8120E0E6F000144DF0A0E0701F76F73
:1062E000070E08010B6FF70E0A6F0001DDEC27F0B7
:1062F000000C040148C4E9FF49C4EAFFEFCF4CF4A5
:106300004BC403F04AC4E9FF4BC4EAFFEF504C5DB5
:1063100015E149C403F048C4E9FF03C0EAFFEF52A6
:1063200003E1000E016E1FD049C403F04851482B11
:10633000D8B4492B4A2BD8B44B2BDCD749C403F033
:1063400048C4E9FF49C4EAFFEFCF4CF44BC403F063
:106350004AC4E9FF4BC4EAFFEF504C5D02E2FF0E76
:1063600001D0010E016E0001F9EF31F00401336B31
:10637000346B356B200E366F376F386F396F3A6F6D
:106380003B6F3C6F3D6F3E6F3F6F406F416F426FA1
:10639000436F446F456F466F476B030E356FE70ED3
:1063A000346F336B335111081BE3036A3351360FDB
:1063B000E96E040E0320EA6EF2CF4AF4F29E35C471
:1063C000AAFF34C4A9FFA69CA69EA680A8504ABFD7
:1063D000F28EEF6E010E3427000E3523332BE2D7F9
:1063E000040E496F360E486F4B6B320E4A6F000138
:1063F00080D7015204E1010E016E04D003D0000EDB
:10640000016E00D0B6EFE8F004014C6B4D6B4E6BA3
:10641000F2CF4FF4F29E030EAA6EFF0EA96EA69C59
:10642000A69EA680A8504FBFF28E4E6F4D6B4C6B50
:106430004D5103081CE34DC4AAFF4CC4A9FFFF0E35
:10644000A86EA69CA69EA684F2CF00F0F29E0F0135
:10645000550EA76EAA0EA76EA682A6B2FED7A69468
:106460000050F21204014C2BD8B44D2BE1D74E5101
:10647000010819E3030EAA6EFF0EA96E4EC4A8FF11
:10648000A69CA69EA684F2CF00F0F29E0F01550EA8
:10649000A76EAA0EA76EA682A6B2FED7A69400503B
:1064A000F21217D00401030EAA6EFF0EA96EA86A9D
:1064B000A69CA69EA684F2CF00F0F29E0F01550E78
:1064C000A76EAA0EA76EA682A6B2FED7A69400500B
:1064D000F2120001BEEF32F00401606B616B626B7F
:1064E000636B646B616B200E606F626B62510508B9
:1064F0002DE3636B63510B0827E3646B64510B0856
:1065000021E361C403F06051602BD8B4612B656F47
:1065100003C066F403C0AAFFA96EA86AA69CA69E43
:10652000A684F2CF00F0F29E0F01550EA76EAA0EC0
:10653000A76EA682A6B2FED7A6940050F21204015E
:10654000642BDCD7632BD6D7622BD0D7626B62511A
:106550000C080AE3036A6251CF0FE96E010E0320B3
:10656000EA6EEF6A622BF3D70001000C0401476B5F
:10657000486B496B4A6B4B6B000146D7AA6AA96A04
:10658000010EA86EA69CA69EA684F2CF00F0F29EF5
:106590000F01550EA76EAA0EA76EA682A6B2FED751
:1065A000A6940050F212AA6A010EA96EA86EA69CCB
:1065B000A69EA684F2CF00F0F29E550EA76EAA0EFC
:1065C000A76EA682A6B2FED7A6940050F212AA6ABF
:1065D000020EA96E0F0EA86EA69CA69EA684F2CFF0
:1065E00000F0F29E550EA76EAA0EA76EA682A6B266
:1065F000FED7A6940050F212AA6A030EA96E120EDC
:10660000A86EA69CA69EA684F2CF00F0F29E550E20
:10661000A76EAA0EA76EA682A6B2FED7A6940050B9
:10662000F212AA6A040EA96EA86EA69CA69EA68463
:10663000F2CF00F0F29E550EA76EAA0EA76EA682AC
:10664000A6B2FED7A6940050F212AA6A050EA96E51
:106650000A0EA86EA69CA69EA684F2CF00F0F29E1B
:10666000550EA76EAA0EA76EA682A6B2FED7A69456
:106670000050F212AA6A060EA96E600EA86EA69CC1
:10668000A69EA684F2CF00F0F29E550EA76EAA0E2B
:10669000A76EA682A6B2FED7A6940050F212AA6AEE
:1066A000070EA96EA86AA69CA69EA684F2CF00F04B
:1066B000F29E550EA76EAA0EA76EA682A6B2FED7B0
:1066C000A6940050F212F2CF4CF4F29E030EAA6E82
:1066D000FF0EA96EA69CA69EA680A85004014CBFE2
:1066E000F28E4D6FAA6A080EA96E4DC4A8FFA69C33
:1066F000A69EA684F250006EF29E0F01550EA76E64
:10670000AA0EA76EA682A6B2FED7A6940050F212D9
:10671000AA6A090EA96E190EA86EA69CA69EA6844A
:10672000F2CF00F0F29E550EA76EAA0EA76EA682BB
:10673000A6B2FED7A6940050F212AA6A0A0EA96E5B
:10674000180EA86EA69CA69EA684F2CF00F0F29E1C
:10675000550EA76EAA0EA76EA682A6B2FED7A69465
:106760000050F212AA6A0B0EA96E180EA86EA69C13
:10677000A69EA684F2CF00F0F29E550EA76EAA0E3A
:10678000A76EA682A6B2FED7A6940050F212AA6AFD
:106790000D0EA96EA86AA69CA69EA684F2CF00F054
:1067A000F29E550EA76EAA0EA76EA682A6B2FED7BF
:1067B000A6940050F212AA6A0E0EA96EA86AA69CB0
:1067C000A69EA684F2CF00F0F29E550EA76EAA0EEA
:1067D000A76EA682A6B2FED7A6940050F212AA6AAD
:1067E0000C0EA96E0E0EA86EA69CA69EA684F2CFD5
:1067F00000F0F29E550EA76EAA0EA76EA682A6B254
:10680000FED7A6940050F212000166DE030E0401CA
:10681000486FE70E476F4B6B4B51110827E3036A34
:106820004B51320FE96E000E0320EA6EEFCF4CF4AD
:1068300048C4AAFF47C4A9FF4CC4A8FFA69CA69EB3
:10684000A684F2CF00F0F29E0F01550EA76EAA0E9D
:10685000A76EA682A6B2FED7A6940050F212010E31
:1068600004014727000E48234B2BD6D74A6B496BB0
:106870004B6B4B51110843E3036A4B51200FE96EF8
:10688000000E0320EA6EEFCF4CF44C512F0803E2C8
:106890004C51390802E2000E01D0010E01082DE131
:1068A0004A532BE14951050828E3036A4B51200F55
:1068B000E96E000E0320EA6EEFCF4CF448C4AAFF45
:1068C00047C4A9FF4CC4A8FFA69CA69EA684F2CFED
:1068D00000F0F29E0F01550EA76EAA0EA76EA682BB
:1068E000A6B2FED7A6940050F2120401492BD8B4E8
:1068F0004A2B010E4727000E48234B2BBAD7000125
:10690000000C0401776B786B796B755303E075515C
:10691000060804E2000E016E6BD108D0765303E046
:1069200076510C0803E2000E016E62D1786B900E76
:10693000776F010E755D036A7A6F03C07BF478C4CC
:106940003DFD77C43CFD03C03FFDE8CF3EFD0001A7
:10695000A2EC29F002C078F401C077F4200E040103
:106960007727000E7823010E765D0C0DF350036A35
:106970007727035078237851036E7751772BD8B45B
:10698000782B7A6F03C07BF4F2CF7CF4F29E7BC449
:10699000AAFF7AC4A9FFA69CA69EA680A8507CBF89
:1069A000F28E796F7951F00BD8B41FD17951F00B79
:1069B0007B6F01014851F00B04017B5DD8A415D118
:1069C00079C448F17851036E7751772BD8B4782B7E
:1069D0007A6F03C07BF4F2CF7CF4F29E7BC4AAFFF3
:1069E0007AC4A9FFA69CA69EA680A8507CBFF28E62
:1069F0000101496F04017851036E7751772BD8B4A8
:106A0000782B7A6F03C07BF4F2CF7CF4F29E7BC4C8
:106A1000AAFF7AC4A9FFA69CA69EA680A8507CBF08
:106A2000F28E01014B6F4A6B04017851036E77516E
:106A3000772BD8B4782B7A6F03C07BF4F2CF7CF439
:106A4000F29E7BC4AAFF7AC4A9FFA69CA69EA6803C
:106A5000A8507CBFF28E01014A1304017851036EE5
:106A60007751772BD8B4782B7A6F03C07BF4F2CFB1
:106A70007CF4F29E7BC4AAFF7AC4A9FFA69CA69EC2
:106A8000A680A8507CBFF28E01014D6F4C6B0401B3
:106A90007851036E7751772BD8B4782B7A6F03C077
:106AA0007BF4F2CF7CF4F29E7BC4AAFF7AC4A9FFE8
:106AB000A69CA69EA680A8507CBFF28E01014C1316
:106AC00004017851036E7751772BD8B4782B7A6F05
:106AD00003C07BF4F2CF7CF4F29E7BC4AAFF7AC49D
:106AE000A9FFA69CA69EA680A8507CBFF28E01019D
:106AF0004F6F4E6B04017851036E7751772BD8B4EA
:106B0000782B7A6F03C07BF4F2CF7CF4F29E7BC4C7
:106B1000AAFF7AC4A9FFA69CA69EA680A8507CBF07
:106B2000F28E01014E1304017851036E7751772BD9
:106B3000D8B4782B7A6F03C07BF4F2CF7CF4F29E4A
:106B40007BC4AAFF7AC4A9FFA69CA69EA680A850D3
:106B50007CBFF28E0101516F506B04017851036EBE
:106B60007751772BD8B4782B7A6F03C07BF4F2CFB0
:106B70007CF4F29E7BC4AAFF7AC4A9FFA69CA69EC1
:106B8000A680A8507CBFF28E0101501304017851F9
:106B9000036E7751772BD8B4782B7A6F03C07BF4D0
:106BA000F2CF7CF4F29E7BC4AAFF7AC4A9FFA69C14
:106BB000A69EA680A8507CBFF28E0101536F526B37
:106BC000F2CF7AF4F29E78C4AAFF77C4A9FFA69CFC
:106BD000A69EA680A85004017ABFF28E010152132E
:106BE000010E016E040104D003D0000E016E00D02E
:106BF0000001000CF2CF4AF4F29EAA6AA96AA69C90
:106C0000A69EA680A85004014ABFF28E01013B6FE8
:106C1000F2CF4AF4F29EAA6A010EA96EA69CA69E25
:106C2000A680A85004014ABFF28E01013C6FF2CF4A
:106C30004AF4F29EAA6A020EA96EA69CA69EA6809F
:106C4000A85004014ABFF28E01013D6FF2CF4AF411
:106C5000F29EAA6A030EA96EA69CA69EA680A850C4
:106C600004014ABFF28E01013E6FF2CF4AF4F29E58
:106C7000AA6A040EA96EA69CA69EA680A85004012E
:106C80004ABFF28E0101416FF2CF4AF4F29EAA6A26
:106C9000050EA96EA69CA69EA680A85004014ABF18
:106CA000F28E0101436FF2CF4AF4F29EAA6A060EF9
:106CB000A96EA69CA69EA680A85004014ABFF28E8B
:106CC00001013A6FF2CF4AF4F29EAA6A070EA96E4A
:106CD000A69CA69EA680A85004014ABFF28E010180
:106CE000396FF2CF4AF4F29EAA6A080EA96EA69CEA
:106CF000A69EA680A85004014ABFF28E0101386FFB
:106D0000F2CF4AF4F29EAA6A0D0EA96EA69CA69E28
:106D1000A680A85004014ABFF28E01013F6FF2CF56
:106D20004AF4F29EAA6A0E0EA96EA69CA69EA680A2
:106D3000A85004014ABFF28E0101406FF2CF4AF41D
:106D4000F29EAA6A090EA96EA69CA69EA680A850CD
:106D500004014ABFF28E0101446FF2CF4AF4F29E61
:106D6000AA6A0A0EA96EA69CA69EA680A850040137
:106D70004ABFF28E0101456FF2CF4AF4F29EAA6A31
:106D80000B0EA96EA69CA69EA680A85004014ABF21
:106D9000F28E0101466FF2CF4AF4F29EAA6A0C0EFF
:106DA000A96EA69CA69EA680A85004014ABFF28E9A
:106DB0000101476F4751280802E2280E476F4551ED
:106DC000180802E2180E456F4651180802E2180E24
:106DD000466F3BC175F43CC176F4000192DD010EB3
:106DE000016E55EF64F0036A6551A90FE96E000E5C
:106DF0000320EA6EEFCF0EF80801010E00016525B1
:106E00000801106F196AF2BE198EF29EE8CF43FD99
:106E1000780E0D01446F0001BFEC22F019BEF28E16
:106E200000C065F06551625D01E1A88108010EC8EE
:106E300001F00001000C080113BF10D00F0E006E0E
:106E4000123900160A0E005C03E2300E002602D052
:106E50001351002600509EA8FED7AD6E0F0E1217DC
:106E60000A0E125D02E2300E02D0139F1351122758
:106E700012519EA8FED7AD6E0001000C640E0801F1
:106E8000116F0001D9EC26F0010139A508D00D0ED3
:106E90009EA8FED7AD6E0A0E9EA8FED7AD6E00016D
:106EA0006551625D1AE09FDF01C04BF4010139A515
:106EB0000DD04BC412F8570E0801136F0001BBDF51
:106EC000200E9EA8FED7AD6E07D00101320E08013C
:106ED000116F0001D9EC26F0E3D7000C200E07015A
:106EE000EAA9300EEB6FE9C700F0E9AF07D0001E4A
:106EF000002A00C0E9F72D0EEB6FEA8F0150196AE6
:106F0000F2BE198EF29EE9C743FD640E0D01446F77
:106F10000001BFEC22F019BEF28E00C0E9F7300E7E
:106F200001240701EC6F196AF2BE198EF29EE9C7BF
:106F300043FD0A0E0D01446F0001BFEC22F019BEA3
:106F4000F28E300E00240701EE6F300E0124ED6F3B
:106F5000EBC700F0EAA702D0EAAFEA95EAB90BD096
:106F6000EAAF22D0EAB520D000C0ECF7EAB31CD0DB
:106F700000C0EDF719D0300EEC5D16E100C0ECF763
:106F8000200EEB6FEAA704D0EA95EA83EAAFEA9312
:106F9000300EED5D09E100C0EDF7200EEC6FEAA7C1
:106FA000F7D7EA93EAAFEA91EAA504D0EB519EA89D
:106FB000FED7AD6EEAA304D0EC519EA8FED7AD6E0D
:106FC000EAA104D0ED519EA8FED7AD6EEE519EA869
:106FD000FED7AD6E0001000C08010F6B106B0DC8E1
:106FE000E9FF0EC8EAFFEFCF10F8105340E00101AF
:106FF00039A508D00D0E9EA8FED7AD6E0A0E9EA82C
:10700000FED7AD6E010E08010F6F0F51105D2FE31B
:10701000010139A516D0036A08010F510D25E96E4B
:107020000E510320EA6EEFCF11F811C812F8570E77
:10703000136F000100DF200E9EA8FED7AD6E07D0B3
:107040000101010E0801116F0001D9EC26F0036A5D
:1070500008010F510D25E96E0E510320EA6EEFCFA6
:1070600011F81151A4A8FED76D6E0F2BCED70001D9
:10707000000CEACF08F8E9CF07F8080101AF08D003
:10708000078F07A9072B001F011F002BD8B4012B66
:107090000139F009036F0327E20F046F320F066F07
:1070A00001510F0B042704270627E90F056F052759
:1070B000052700390F0B0527062705370637061F5A
:1070C000063700510F0B06270337070E026F0A0E13
:1070D00005070627FDE304070527FDE3030704274B
:1070E000FDE302070327FDE3080EEA6E020EE96ED8
:1070F000070E0715079DE906071507E107B9E92AF5
:1071000007B903D0200E006E1CD0E926060EE95CFC
:10711000D8B4078DEF50006E08E107BD06D007B95F
:1071200014D007B702D0200E0BD007AF06D02D0E1B
:10713000006EED50079D079F04D007870799300E1A
:10714000002600509EA8FED7AD6EEE5007ADDED7EC
:107150000001000C0701FA6BFB6BFC6BFD6BFE91F1
:107160000001A8A159D0FDC73DFDFCC73CFD0D01A4
:107170003F6B320E3E6F0001A2EC29F002C000F816
:1071800001C0FFF70701ED510801025C3AE308E195
:107190000701EC51FF5DD8B002D0080132D00801E0
:1071A000010139A52AD00701FF6BFF5100014BEC0B
:1071B00011F00701FF2B006E00509EA8FED7AD6EA8
:1071C000170EFF5DF2E1100EE96EEDC701F8ECC796
:1071D00000F800014EDF1A0E0801006F0051000197
:1071E0004BEC11F00801002B006E00509EA8FED75A
:1071F000AD6E210E005DF2E10101000E016EEDD0D9
:107200000801320E116F0001D9EC26F00701FC2BAA
:10721000D8B4FD2BA5D70001070EEA6EEE0EE96E7D
:1072200008010A6B0C6B0C0E0B6F000186EC28F04A
:10723000010139A510D00701FF6BFF5100016BEC74
:1072400011F00701FF2B006E00509EA8FED7AD6E17
:107250000F0EFF5DF2E10001A8B1BED0C4DD01C098
:10726000FAF70701FEA169D0FA3D37D0010139A52F
:107270000CD0FAC712F8370E0801136F0001DBDDDE
:10728000200E9EA8FED7AD6E01010701EF51410807
:1072900003E0EF51420806E1010E016E01019DD0AD
:1072A0001AD00701EF51510803E0EF5152080FE1E6
:1072B000070EEA6EEE0EE96E08010A6B0C6B0C0EFF
:1072C0000B6F000186EC28F00701FE9105D0000E3F
:1072D000016E010182D007012FD0036AFB51EE0F2E
:1072E000E96E070E0320EA6EFAC7EFFF010139A528
:1072F00017D0036A0701FB51EE0FE96E070E03205A
:10730000EA6EEFCFFFF7FFC712F8370E0801136FD1
:10731000000191DD200E9EA8FED7AD6E07D00101C1
:10732000320E0801116F0001D9EC26F00701FB2B8A
:10733000FB510B0801E2FE9148D0FA51900826E17A
:10734000FB6B036AFB51EE0FE96E070E0320EA6E3A
:10735000FAC7EFFF010139A515D0036A0701FB51F8
:10736000EE0FE96E070E0320EA6EEFCFFFF7FFC7BF
:1073700012F8370E0801136F00015DDD200E9EA884
:10738000FED7AD6E0701FB2BFE811FD0010139A591
:1073900015D05B0E9EA8FED7AD6EFAC712F8370E59
:1073A0000801136F000147DD5D0E9EA8FED7AD6E8C
:1073B000200E9EA8FED7AD6E07D00101320E080147
:1073C000116F0001D9EC26F00701320E0801116F90
:1073D0000001D9EC26F040D701010001000C0801A2
:1073E0000D6B0001A8B104D0FEDC01C00DF8FAD786
:1073F000000C060E0701D86F810ED96F010EDA6FEF
:10740000040EDB6F070EDC6FDD6BFF0EDE6F090E07
:10741000DF6F810EE06F010EE16F060EE26F010E6D
:10742000E36FE46BE56B030EE66FE76FFF0EE86F4B
:10743000D5517F0BE96FD6517F0BEA6FD7517F0B88
:10744000EB6FE95305E1010EE96F030EE66F09D01A
:10745000D551800B800803E1010EE66F02D0020EC9
:10746000E66FE9C7E4F7EA5305E1010EEA6F030EA0
:10747000E76F09D0D651800B800803E1010EE76F5A
:1074800002D0020EE76FEAC7E5F701014839006E46
:107490000F0E001600500A083EE00701E6510308EF
:1074A00003E1E751030822E001015483070E0801BC
:1074B0000E6FDF0E0D6F00018FDD01014839006E88
:1074C0000F0E00160050010807E04839006E0F0E3D
:1074D00000160050050808E1030E0701ED6FE80EE5
:1074E000EC6F000137DE010114D00701010154A344
:1074F00010D05493070E08010E6FDF0E0D6F0001C0
:107500006BDD030E0701ED6FE80EEC6F000122DE6C
:107510000101000164DF0701EB5302E1DD6B0DD0D7
:10752000D751800B800805E1EB51070B2009DD6F77
:1075300004D0EB51070B3009DD6FDD5321E0070E5E
:1075400008010E6FD80E0D6F000146DD0101548158
:107550004839006E0F0E00160050010807E0483948
:10756000006E0F0E00160050050808E1030E07011B
:10757000ED6FE80EEC6F0001EDDD010114D00701A5
:10758000010154A110D05491070E08010E6FD80EBE
:107590000D6F000121DD030E0701ED6FE80EEC6FAA
:1075A0000001D8DD010100011ADF000C08011051B3
:1075B000090805E3300E1025016E05D004D0370E02
:1075C0001025016E00D00001000C080E0701D86FD5
:1075D000FF0ED96F300EDA6FDB6FDC6B600EDD6F84
:1075E000300EDE6FDF6FEF0EE06F070EE16FFF0E04
:1075F000E26F300EE36FE46FE56BA20EE66F300EC4
:10760000E76FEF0EE86F090EE96FFF0EEA6F300EBD
:10761000EB6FEC6FED6B500EEE6FEF6BF06BF16B91
:10762000EF0EF26F090EF36FFF0EF46F300EF56F71
:10763000F66FF76B510EF86FF96BFA6BFB6BEF0E91
:10764000FC6F080EFD6FFF0EFE6F300EFF6F08011E
:10765000006F016BB40E026F310E036F046BEF0EFF
:10766000056F0701D5517F0B0801066F0701D65141
:107670007F0B0801076F0701D7517F0B0801086FC7
:10768000085315E10301DA513008D8A402D00801EB
:107690000ED00001A4DE070E08010E6FE10E0D6F83
:1076A00000019ADCE7C7DAF301015491080106539F
:1076B0001CE107531AE10301D851300806E1D95102
:1076C0003008D8A402D0080110D0000188DE070ECF
:1076D00008010E6FD80E0D6F00017EDCDEC7D8F3F7
:1076E000DFC7D9F3010154930801065305E107539D
:1076F00003E1085301E145D1065305E1300E0701CE
:10770000DE6F0BD008010701D551800B800803E123
:10771000320EDE6F02D0310EDE6F0801075305E135
:10772000300E0701DF6F0BD008010701D651800B27
:10773000800803E1310EDF6F02D0320EDF6F036A83
:1077400007C80DF803C00EF80D013D6B1E0E3C6F0F
:1077500003C03FFD07C83EFD0001A2EC29F0080E62
:1077600008010124096F000E02200A6F036A06C88F
:107770000DF803C00EF80D013D6B210E3C6F03C0E8
:107780003FFD06C83EFD0001A2EC29F0080E0801ED
:1077900001240B6F000E02200C6F0C5306E10B51FD
:1077A000090803E30C6B0A0E0B6F0C51020809E287
:1077B000FF0A03E10B51200804E2030E0C6F200EB8
:1077C0000B6F0A5306E10951090803E30A6B0A0E1D
:1077D000096F0A51010809E2FF0A03E109516E0825
:1077E00004E2020E0A6F6E0E096F0C510F0B0E6F42
:1077F000106F0001DBDE01C0EFF708010BC800F0DD
:10780000003A0F0E001600500F0B0F6F106F0001A3
:10781000CDDE01C0F0F708010B510F0B0E6F106F9A
:107820000001C4DE01C0F1F708010A510F0B0E6F11
:10783000106F0001BBDE01C0F9F7080109C800F0B4
:10784000003A0F0E001600500F0B0F6F106F000163
:10785000ADDE01C0FAF7080109510F0B0E6F106F72
:107860000001A4DE01C0FBF7080106531CE007017C
:10787000DE513008D8A402D0080115D0010154838C
:10788000080106510101555D0DE006C855F10001E2
:10789000A6DD070E08010E6FE90E0D6F0001ECEC7E
:1078A00037F00101080107531CE00701DF513008E0
:1078B000D8A402D0080115D0010154830801075152
:1078C0000101565D0DE007C856F1000188DD070E85
:1078D00008010E6FF30E0D6F0001ECEC37F00101A3
:1078E00008010701DF510301D95D05E10701DE5100
:1078F0000301D85D0EE0DEC7D8F3DFC7D9F300017E
:107900006EDD070E08010E6FD80E0D6F0001ECEC56
:1079100037F00801085335E00701D751800B800884
:1079200003E1320EE76F02D0310EE76F010154819F
:10793000080108510101575D11E008C857F108011D
:107940000851070B3009046F000149DD070E0801DB
:107950000E6FFD0E0D6F0001ECEC37F00701E751E3
:107960000301DA5D0DE0E7C7DAF3000138DD070E49
:1079700008010E6FE10E0D6F0001ECEC37F0030112
:1079800008010001000C6B50060B2DE0010139A528
:1079900021D004016A6B6A51000130EC20F004012F
:1079A0006A2B006E00509EA8FED7AD6E160E6A5D63
:1079B000F2E16BCF12F8570E0801136F00011BECB8
:1079C00037F00A0E9EA8FED7AD6E0D0E9EA8FED70C
:1079D000AD6E01016B6A010E0701CE6F0001C4ECB0
:1079E00026F0900E6B6E2DEF3DF001014839006ED0
:1079F0000F0E00160050FF0FF20F14E20E0F0001E1
:107A000061EF3DF00701D56BD66BD76B0001F1DC60
:107A1000010108D00701D56BD66BD76B0001D5DD0E
:107A2000010100D0040169B102D08D9601D08D868C
:107A3000969669B302D08D9801D08D88969869B5D5
:107A400002D08D9A01D08D8A969A050E0801116F89
:107A50000001D9EC26F0C3DC96D769C485F1036A2E
:107A600004016951200F016E000E03220150380FEE
:107A7000E96E010E0320EA6EEFCF48F10101D890C4
:107A800004016935036A350F016E000E03220150AF
:107A9000380FE96E010E0320EA6EECCF03F0ED52D1
:107AA000EFCF52F1010103C053F1496B4B6B4A6BAD
:107AB0004D6B4C6B4F6B4E6B516B506B546B0001AD
:107AC000000CF2CF0EF0F29EE824F76AF736ED0FC5
:107AD000F66E7A0EF722000EF86EFB6E0A00F55075
:107AE000FA6E0800F5500EBEF28EF96E047A047A32
:107AF000047A047A047A047A047A047A047A047A96
:107B0000247A147A247A047A050E04016C6F5B0ED1
:107B10006D6F490E6E6F4E0E6F6F300E706F5D0E93
:107B2000716F6A510301D65D46E06AC4D6F3040161
:107B30006BB102D08D9601D08D8696966BB302D034
:107B40008D9801D08D8896986BB502D08D9A01D012
:107B50008D8A969A050E0801116F0001D9EC26F066
:107B60006AC470F4040E08010E6F6C0E0D6F0001F4
:107B7000ECEC37F0050E0801116F0001D9EC26F08E
:107B80002EDC010185B102D08D9601D08D869696AE
:107B900085B302D08D9801D08D88969885B502D096
:107BA0008D9A01D08D8A969A050E0801116F0001F9
:107BB000D9EC26F003010001000C11DC0401692D51
:107BC00014D0010138A708D0300E04016A6F060EE8
:107BD0006B6F000199DF07D0310E04016A6F060E4A
:107BE0006B6F000191DF07D00401330E6A6F060E40
:107BF0006B6F000189DF000C04017F6B806B816B70
:107C0000826BFF0E836F84910001A8A154D082C4BF
:107C10003DFD81C43CFD0D013F6B320E3E6F000106
:107C2000A2EC29F002C086F401C085F404016A5177
:107C3000025C35E303E16951855D31E3010139A55A
:107C40002BD00401856B855100013AEC0DF0040145
:107C5000852B006E00509EA8FED7AD6E1C0E855D74
:107C6000F2E1100EE96E6AC401F869C400F800017F
:107C700039EC38F01F0E0401866F865100013AEC92
:107C80000DF00401862B006E00509EA8FED7AD6E4D
:107C9000260E865DF2E10101FF0E016EDDD0320E8F
:107CA0000801116F0001D9EC26F00401812BD8B432
:107CB000822BAAD70001040EEA6E6B0EE96E080152
:107CC0000A6B0C6B140E0B6F000186EC28F001019F
:107CD00039A510D00401856B855100015DEC0DF0D4
:107CE0000401852B006E00509EA8FED7AD6E1C0EC1
:107CF000855DF2E10401806BFF0E836F0001A8B186
:107D000099D0F3EC36F001C07FF4040184B135D092
:107D1000806B7F515B081AE1036A80516B0FE96E3B
:107D2000040E0320EA6E7FC4EFFF802B84810101E3
:107D300039A50AD004017F519EA8FED7AD6E200E52
:107D40009EA8FED7AD6E010116D00401010139A530
:107D500012D0280E9EA8FED7AD6E04017F519EA8BA
:107D6000FED7AD6E290E9EA8FED7AD6E200E9EA842
:107D7000FED7AD6E01015CD00401036A80516B0F28
:107D8000E96E040E0320EA6E7FC4EFFF010139A5FE
:107D900009D004017F519EA8FED7AD6E200E9EA88B
:107DA000FED7AD6E04017F515D083BE16C5149087F
:107DB00029E16D514E0826E16F515D0823E16EC443
:107DC00083F4010139A51CD00401856B85510001A4
:107DD0007BEC0DF00401852B006E00509EA8FED7B1
:107DE000AD6E0D0E855DF2E183519EA8FED7AD6E9E
:107DF0000A0E9EA8FED7AD6E0D0E9EA8FED7AD6EE4
:107E0000000118D0010139A508D00A0E9EA8FED79E
:107E1000AD6E0D0E9EA8FED7AD6E0401806B8491F1
:107E200007D0802B8051130803E2000103D0040126
:107E3000040164D7010139A508D00A0E9EA8FED717
:107E4000AD6E0D0E9EA8FED7AD6E0001EFEC39F0C1
:107E5000040183C401F00101000161EF3FF0080E4D
:107E60000401606F5B0E616F530E626F540E636F9F
:107E7000410E646F540E656F550E666F530E676F3B
:107E80005D0E686F010E696F000197DE640E0801D8
:107E9000116F0001D9EC26F0040E08010E6F600E80
:107EA0000D6F0001ECEC37F0320E0801116F00018C
:107EB000D9EC26F0030E04016A6FE80E696F000129
:107EC0009BD60150DDEF5FF00501D76BD86BD96B06
:107ED000DA91050EEA6ECA0EE96E08010A6B0C6BA8
:107EE0000D0E0B6F000186EC28F0A8A154D0D9C567
:107EF0003DFDD8C53CFD0D013F6B190E3E6F0001E5
:107F0000A2EC29F002C0DCF501C0DBF50501C95186
:107F1000025C35E303E1C851DB5D31E3010139A5C2
:107F20002BD00501DB6BDB510001E8EC11F0050102
:107F3000DB2B006E00509EA8FED7AD6E150EDB5DEC
:107F4000F2E1100EE96EC9C501F8C8C500F80001DC
:107F500039EC38F0180E0501DC6FDC510001E8EC5B
:107F600011F00501DC2B006E00509EA8FED7AD6E0F
:107F70001F0EDC5DF2E10101000E016EACD0190EA6
:107F80000801116F0001D9EC26F00501D82BD8B4F7
:107F9000D92B0001AAD7010139A510D00501DB6B4F
:107FA000DB51000107EC12F00501DB2B006E0050E5
:107FB0009EA8FED7AD6E0D0EDB5DF2E10001A8B10B
:107FC00087D0036A0501D751CA0F016E050E03223F
:107FD00001C0DBF503C0DCF50001F3EC36F0DCC5D5
:107FE000EAFFDBC5E9FF01C0EFFF010139A516D0AB
:107FF000036A0501D751CA0FE96E050E0320EA6E28
:10800000EFCFDBF5DBC512F8370E0801136F000167
:108010001BEC37F0200E9EA8FED7AD6E0501DAB13D
:1080200017D0036AD751CA0FE96E050E0320EA6E16
:10803000EF50FE080CE1036AD751CA0FE96E050E36
:108040000320EA6EEFCFCAF5DA81010ED76F36D082
:10805000036AD751CA0FE96E050E0320EA6EEF508E
:10806000EF081EE1010139A508D00D0E9EA8FED72C
:10807000AD6E0A0E9EA8FED7AD6E0501CD5130083B
:1080800009E1CE51300806E1010E016E010123D055
:1080900005D00501000E016E01011DD007D00501BC
:1080A000320E0801116F0001D9EC26F00501D751FD
:1080B0000B0802E3D72B02D0D76BDA910001A8A1FD
:1080C00006D0320E0801116F0001D9EC26F077D7E7
:1080D000000E016E01010001000C0401C26BC36BB4
:1080E000060EC46FFF0EC56F300EC66FC76FC86B2C
:1080F000860EC96FEF0ECA6F060ECB6FFF0ECC6FE8
:10810000300ECD6FCE6FCF6B860ED06FEF0ED16F6E
:10811000060ED26FFF0ED36F300ED46FD56FD66BB5
:10812000860ED76FEF0ED86F060ED96FFF0EDA6F7F
:10813000300EDB6FDC6FDD6B860EDE6FEF0EDF6FF8
:10814000060EE06FFF0EE16F300EE26FE36FE46B3F
:10815000860EE56FEF0EE66F060EE76FFF0EE86F17
:10816000300EE96FEA6FEB6B860EEC6FEF0EED6F82
:10817000070EEE6FFF0EEF6F300EF06FF16FF26BC8
:10818000A50EF36F3C0EF46FEF0EF56F070EF66F52
:10819000FF0EF76F300EF86FF96FFA6BB40EFB6FCE
:1081A000300EFC6FEF0EFD6F060EFE6FFF0EFF6FC1
:1081B000300E0501006F016F026B630E036FEF0E4F
:1081C000046F070E056FFF0E066F300E076F086F06
:1081D000096BB10E0A6F300E0B6FEF0E0C6F070EAE
:1081E0000D6FFF0E0E6F300E0F6F106F116B900E34
:1081F000126F300E136FEF0E146F070E156FFF0E18
:10820000166F300E176F186F196BA00E1A6F310EA4
:108210001B6FEF0E1C6F070E1D6FFF0E1E6F300ED3
:108220001F6F206F216BA00E226F300E236FEF0E99
:10823000246F070E256FFF0E266F300E276F286FF5
:10824000296BA50E2A6F310E2B6FEF0E2C6F070EC8
:108250002D6FFF0E2E6F300E2F6F306F316BA50E0E
:10826000326F300E336FEF0E346F070E356FFF0E27
:10827000366F300E376F386F396BA70E3A6F300E8E
:108280003B6FEF0E3C6F070E3D6FFF0E3E6F300EE3
:108290003F6F406F416BA70E426F310E436FEF0E81
:1082A000446F070E456FFF0E466F300E476F486FE5
:1082B000496BA70E4A6F310E4B6FEF0E4C6F070ED6
:1082C0004D6FFF0E4E6F300E4F6F506F516BA50EFE
:1082D000526F320E536FEF0E546F070E556FFF0E35
:1082E000566F300E576F586F596BA50E5A6F320E7E
:1082F0005B6FEF0E5C6F090E5D6FFF0E5E6F300EF1
:108300005F6F606F616BA50E626F3B0E636F646B96
:10831000656BEF0E666F090E676FFF0E686F300EAC
:10832000696F6A6F6B6BA50E6C6F340E6D6F300EDC
:108330006E6FEF0E6F6F706B070E716FFF0E726FC7
:10834000300E736F746F756BA10E766F300E776F92
:10835000EF0E786F070E796FFF0E7A6F300E7B6F1E
:108360007C6F7D6BA10E7E6F310E7F6FEF0E806F85
:10837000070E816FFF0E826F300E836F846F856BE7
:10838000A10E866F330E876FEF0E886F070E896F11
:10839000FF0E8A6F300E8B6F8C6F8D6BA10E8E6F00
:1083A000320E8F6FEF0E906F070E916FFF0E926F70
:1083B000300E936F946F956BA10E966F310E976F81
:1083C000EF0E986F090E996FFF0E9A6F300E9B6F2C
:1083D0009C6FB00E9D6F9E6B9F6BA06BA16BEF0EA1
:1083E000A26F060EA36FFF0EA46F300EA56FA66FCF
:1083F000A76B570EA86FEF0EA96F070EAA6FFF0E9F
:10840000AB6F300EAC6FAD6FAE6B580EAF6F310E01
:10841000B06FEF0EB16F090EB26FFF0EB36F300E7B
:10842000B46FB56FB66B500EB76F310EB86FB96FD2
:10843000BA6FEF0EBB6F090EBC6FFF0EBD6F300E33
:10844000BE6FBF6FC06B890EC16FC26BEF0EC36F83
:10845000C46BC56BC66BC76B0401C051330A000106
:10846000D8B497D0320AD8B49DD0030AD8B4A3D0D8
:10847000010AD8B4A9D0070AD8B4AFD0010AD8B439
:10848000B5D0030AD8B4BBD00E0AD8B4C1D0010A03
:10849000D8B4C7D0030AD8B4CDD00D0AD8B4D3D03D
:1084A0000A0AD8B4D8D0030AD8B4DED0010AD8B4A6
:1084B000E4D01F0AD8B4EAD0010AD8B4F0D0030A35
:1084C000D8B4F6D0010AD8B4FCD0260AD8B402D168
:1084D000010AD8B410D1020AD8B41ED12C0AD8B4DB
:1084E0002CD1030AD8B435D10D0AD8B43ED1010A33
:1084F000D8B444D1030AD8B45BD1010AD8B45ED150
:108500000F0AD8B461D1030AD8B49BD1070AD8B4F2
:10851000A1D1010AD8B4A7D1030AD8B4ADD1010AB8
:10852000D8B4B3D13F0AD8B4B9D1030AD8B406D26B
:10853000070AD8B410D2010AD8B41AD2030AD8B4A0
:108540001FD2010AD8B425D20F0AD8B42FD2010AFB
:10855000D8B435D2030AD8B440D2010AD8B446D22E
:10856000070AD8B457D2010AD8B463D2030AD8B4E0
:108570006FD2010AD8B476D21E0AD8B47BD2030ACD
:10858000D8B481D20A0AD8B487D2010AD8B4F4D2B6
:1085900063D3050E08010E6F0D0E0D6F0001ECEC9C
:1085A00037F05ED3040E08010E6FC40E0D6F00018C
:1085B000ECEC37F055D3040E08010E6FCB0E0D6FA7
:1085C0000001ECEC37F04CD3040E08010E6FD20E14
:1085D0000D6F0001ECEC37F043D3040E08010E6F71
:1085E000D90E0D6F0001ECEC37F03AD3040E080100
:1085F0000E6FE00E0D6F0001ECEC37F031D3040E7E
:1086000008010E6FE70E0D6F0001ECEC37F028D378
:10861000040E08010E6FEE0E0D6F0001ECEC37F04A
:108620001FD3040E08010E6FF60E0D6F0001ECEC67
:1086300037F016D3040E08010E6FFE0E0D6F000109
:10864000ECEC37F00DD3050E08010E6F0D6F000135
:10865000ECEC37F005D3050E08010E6F150E0D6F0B
:108660000001ECEC37F0FCD2050E08010E6F1D0E78
:108670000D6F0001ECEC37F0F3D2050E08010E6F20
:10868000250E0D6F0001ECEC37F0EAD2050E080163
:108690000E6F2D0E0D6F0001ECEC37F0E1D2050EE0
:1086A00008010E6F350E0D6F0001ECEC37F0D8D2DB
:1086B000050E08010E6F3D0E0D6F0001ECEC37F05A
:1086C000CFD2050E08010E6F450E0D6F0001ECECC8
:1086D00037F0C6D2010186510F0B30090501C26F78
:1086E0008A0EC16F050E08010E6FBC0E0D6F0001E2
:1086F000ECEC37F0B5D2010186510F0B30090501C2
:10870000C26F890EC16F050E08010E6FBC0E0D6F92
:108710000001ECEC37F0A4D2010186510F0B3009B7
:108720000501C26F8B0EC16F050E08010E6FBC0EE6
:108730000D6F0001ECEC37F093D2300E05016E6F37
:10874000050E08010E6F670E0D6F0001ECEC37F09F
:1087500087D2310E05016E6F050E08010E6F670E90
:108760000D6F0001ECEC37F07BD2050E08010E6FA7
:10877000550E0D6F0001ECEC37F072D2050E0801BA
:108780000E6F4D0E0D6F0001ECEC37F0640E08011A
:10879000116F0001D9EC26F0300E05016E6F050E49
:1087A00008010E6F670E0D6F0001ECEC37F058D228
:1087B000020E01015227000E532300010101525104
:1087C000D8B45307520700010101535307E1525136
:1087D0000F0804E3536B100E526F06D0535100087C
:1087E00003E2536BFF0E526F53C1C7F552C1C6F57A
:1087F0000501C731C96FC631C86FC933C833C93322
:10880000C833C933C8330F0EC917C8C510F80001E3
:10881000D6EC3AF001C064F50501C6510F0BC86FE4
:10882000C96BE8CF10F80001D6EC3AF001C065F54D
:10883000050E08010E6F5D0E0D6F0001ECEC37F0B8
:108840000FD2050E08010E6F710E0D6F0001ECECDA
:1088500037F006D2050E08010E6F790E0D6F00017C
:10886000ECEC37F0FDD1050E08010E6F810E0D6F97
:108870000001ECEC37F0F4D1050E08010E6F890E03
:108880000D6F0001ECEC37F0EBD1050E08010E6F17
:10889000910E0D6F0001ECEC37F0E2D151C1C7F53C
:1088A00050C1C6F50501C86BC751F00BC96FC93976
:1088B000CA6FCB6B0F0ECA17CAC510F80001D6ECF1
:1088C0003AF001C09EF50501C86BC7510F0BC96F87
:1088D000CA6FCB6BE8CF10F80001D6EC3AF001C0BC
:1088E0009FF50501C651F00BC86FC96BC931CB6F3D
:1088F000C831CA6FCB33CA33CB33CA33CB33CA3355
:108900000F0ECB17CAC510F80001D6EC3AF001C023
:10891000A0F50501C6510F0BC86FC96BE8CF10F861
:108920000001D6EC3AF001C0A1F5050E08010E6F6A
:10893000990E0D6F0001ECEC37F092D1010141511D
:1089400088090501C86F0701D56BD66BD76F000189
:10895000E5EC3AF085D10101415108090501C86FE4
:108960000701D56BD66BD76F0001E5EC3AF078D1F3
:108970000701D56BD66BD76B0001E5EC3AF070D1EF
:108980000701D56BD66B41C1D7F70001E5EC3AF092
:1089900067D101013D5180090501C86F0701D56B01
:1089A000D66FD76B0001E5EC3AF05AD10701D56BD1
:1089B0003DC1D6F7D76B0001E5EC3AF051D101018A
:1089C0003E5180090501C86FE8CFD5F70701D66B86
:1089D000D76B0001E5EC3AF043D13EC1D5F7070172
:1089E000D66BD76B0001E5EC3AF03AD101013E516C
:1089F00080090501C86F01013D5180090501C96F5A
:108A0000C8C5D5F7E8CFD6F70701D76B0001E5EC6D
:108A10003AF026D101013D5180090501C86F3EC1E0
:108A2000D5F7E8CFD6F70701D76B0001E5EC3AF0B0
:108A300017D101013E5180090501C86FE8CFD5F774
:108A40003DC1D6F70701D76B0001E5EC3AF008D13C
:108A50003EC1D5F73DC1D6F70701D76B0001E5EC64
:108A60003AF0FED00701D56BD66BD76B0001E5EC71
:108A70003AF0F6D0050E08010E6FA30E0D6F00013F
:108A8000ECEC37F0EDD0050E08010E6FAA0E0D6F5D
:108A90000001ECEC37F0E4D0036A3EC1C8F503C036
:108AA000C9F50D013D6B210E3C6F03C03FFD3EC17A
:108AB0003EFD0001A2EC29F0080E0501012404018D
:108AC000C26F000E050102200401C36FC35307E10A
:108AD000C251070804E3C36B080EC26F0CD0C35128
:108AE000020809E2FF0A03E1C251200804E2030E72
:108AF000C36F200EC26F500E0501B76FC86B040123
:108B0000C3510F0B0501C96FCA6FCB6BE8CF10F8CB
:108B10000001D6EC3AF001C0B8F50401C251F00BE7
:108B20000501C86FC96BC931CB6FC831CA6FCB3370
:108B3000CA33CB33CA33CB33CA330F0ECB17CAC5B4
:108B400010F80001D6EC3AF001C0B9F50401C251A9
:108B50000F0B0501C86FC96BE8CF10F80001D6EC08
:108B60003AF001C0BAF5050E08010E6FB20E0D6F96
:108B70000001ECEC37F074D0036A3DC1C8F503C0C6
:108B8000C9F50D013D6B1A0E3C6F03C03FFD3DC1A1
:108B90003EFD0001A2EC29F0080E050101240401AC
:108BA000C26F000E050102200401C36FC35307E129
:108BB000C251070804E3C36B080EC26F0CD0C35147
:108BC000010809E2FF0A03E1C2516E0804E2020E45
:108BD000C36F6E0EC26F510E0501B76FC86B0401F3
:108BE000C3510F0B0501C96FCA6FCB6BE8CF10F8EB
:108BF0000001D6EC3AF001C0B8F50401C251F00B07
:108C00000501C86FC96BC931CB6FC831CA6FCB338F
:108C1000CA33CB33CA33CB33CA330F0ECB17CAC5D3
:108C200010F80001D6EC3AF001C0B9F50401C251C8
:108C30000F0B0501C86FC96BE8CF10F80001D6EC27
:108C40003AF001C0BAF5050E08010E6FB20E0D6FB5
:108C50000001ECEC37F004D0000E016E0FD000D014
:108C60000401C12D09D0070E0501C96FD00EC86FD0
:108C7000000164EC3FF00401010E016E0001000CE4
:108C80000401606B716BFE0E726F736B746B00018D
:108C9000A8A13BD074C43DFD73C43CFD0D013F6BE6
:108CA000320E3E6F0001A2EC29F002C076F401C042
:108CB00075F40401025006081CE2FF0A03E1755135
:108CC000CF0817E2010139A511D00401756B755168
:108CD000000143EC0EF00401752B006E00509EA8BD
:108CE000FED7AD6E230E755DF2E10101000E016E3F
:108CF00087D0320E0801116F0001D9EC26F0040173
:108D0000732BD8B4742BC3D70001040EEA6E610E26
:108D1000E96E08010A6B0C6B100E0B6F000186ECFC
:108D200028F0010139A511D00401756B75510001BE
:108D300064EC0EF00401752B006E00509EA8FED767
:108D4000AD6E100E755DF2E101010001A8B13DD0DC
:108D5000040171510F08D8B002D0000136D00001D3
:108D6000F3EC36F001C060F40A0E0801116F000147
:108D7000D9EC26F0010139A50ED060C412F8370EE7
:108D80000801136F00011BEC37F0200E9EA8FED7E0
:108D9000AD6E07D00101320E0801116F0001D9EC50
:108DA00026F004017251605D04E1716B60C461F4EE
:108DB0000AD0712B036A7151610FE96E040E032012
:108DC000EA6E60C4EFFF0101C0D704016151FE08E3
:108DD00013E1036A7151610FE96E040E0320EA6E1C
:108DE000EF50EF0809E17151050806E1010E016E2F
:108DF000010106D005D00401000E016E010100D072
:108E0000000168EF60F00501B26BB36BB46BB56B3A
:108E1000B691B6930001A8A154D0B5C53DFDB4C527
:108E20003CFD0D013F6B320E3E6F0001A2EC29F0BC
:108E300002C0B8F501C0B7F50501A551025C35E3E4
:108E400003E1A451B75D31E3010139A52BD0050140
:108E5000B76BB751000182EC11F00501B72B006E22
:108E600000509EA8FED7AD6E140EB75DF2E1100E55
:108E7000E96EA5C501F8A4C500F8000139EC38F089
:108E8000170E0501B86FB851000182EC11F0050111
:108E9000B82B006E00509EA8FED7AD6E1E0EB85DBA
:108EA000F2E10101000E016E3AD2320E0801116F9B
:108EB0000001D9EC26F00501B42BD8B4B52BAAD704
:108EC0000001050EEA6EA60EE96E08010A6B0C6B36
:108ED0000C0E0B6F000186EC28F0010139A510D0B3
:108EE0000501B76BB7510001A1EC11F00501B72BDB
:108EF000006E00509EA8FED7AD6E0C0EB75DF2E17D
:108F00000001A8B10BD2F3EC36F001C0B2F50501B7
:108F1000B6A3ADD1B23D42D1010139A50DD0B2C544
:108F200012F8370E0801136F00011BEC37F0200E0A
:108F30009EA8FED7AD6E01010501A651880803E089
:108F4000A651810810E1010139A508D00D0E9EA897
:108F5000FED7AD6E0A0E9EA8FED7AD6E010E016E55
:108F6000DED11AD10501A751510804E0A7515208DA
:108F7000D8A490D0010139A508D00D0E9EA8FED727
:108F8000AD6E0A0E9EA8FED7AD6E0501B6A106D045
:108F9000010E016E0101C3D17BD00501010139A58C
:108FA00011D00501B76BB7510001A1EC11F005011B
:108FB000B72B006E00509EA8FED7AD6E0C0EB75DAD
:108FC000F2E10101050EEA6EA60EE96E08010A6BD8
:108FD0000C6B0C0E0B6F000186EC28F00501B693AC
:108FE0000001A8A154D0B5C53DFDB4C53CFD0D019F
:108FF0003F6B320E3E6F0001A2EC29F002C0B8F5C3
:1090000001C0B7F50501A551025C35E303E1A451A8
:10901000B75D31E3010139A52BD00501B76BB7511D
:109020000001B7EC11F00501B72B006E00509EA8AF
:10903000FED7AD6E090EB75DF2E1100EE96EA5C563
:1090400001F8A4C500F8000139EC38F00C0E050158
:10905000B86FB8510001B7EC11F00501B82B006EE4
:1090600000509EA8FED7AD6E130EB85DF2E101016F
:10907000000E016E54D1320E0801116F0001D9ECBF
:1090800026F00501B42BD8B4B52BAAD700010101F5
:1090900083D00501A751410804E0A7514208D8A494
:1090A00079D0B681010139A511D00501B76BB7514F
:1090B0000001A1EC11F00501B72B006E00509EA835
:1090C000FED7AD6E0C0EB75DF2E10101050EEA6E42
:1090D000A60EE96E08010A6B0C6B0C0E0B6F0001FB
:1090E00086EC28F00501B6930001A8A154D0B5C5BF
:1090F0003DFDB4C53CFD0D013F6B320E3E6F0001DE
:10910000A2EC29F002C0B8F501C0B7F50501A551E0
:10911000025C35E303E1A451B75D31E3010139A5F8
:109120002BD00501B76BB7510001B7EC11F0050169
:10913000B72B006E00509EA8FED7AD6E090EB75D2E
:10914000F2E1100EE96EA5C501F8A4C500F8000112
:1091500039EC38F00C0E0501B86FB8510001B7ECCE
:1091600011F00501B82B006E00509EA8FED7AD6E21
:10917000130EB85DF2E10101000E016ED0D0320E87
:109180000801116F0001D9EC26F00501B42BD8B409
:10919000B52BAAD70001010168D00501036AB351BC
:1091A000A60FE96E050E0320EA6EB2C5EFFF0101BE
:1091B00039A518D0036A0501B351A60FE96E050E53
:1091C0000320EA6EEFCFB7F5B7C512F8370E0801E6
:1091D000136F00011BEC37F0200E9EA8FED7AD6E7A
:1091E00007D00101320E0801116F0001D9EC26F001
:1091F0000501B32BB3510B0802E2B69335D0A6514B
:10920000900832E1B35102082FE1A751410A000151
:109210000FE0030A0DE0120A0BE0010A09E0030A5D
:1092200007E0320A05E0010A03E0030A01E001D089
:109230001AD00501B693010139A510D00501B76B0D
:10924000B7510001D0EC11F00501B72B006E0050B2
:109250009EA8FED7AD6E100EB75DF2E10501B56BAD
:10926000B46B000100D00501010151D00501B251DC
:10927000900806E0B251810803E0B251880827E166
:10928000B36B036AB351A60FE96E050E0320EA6EB5
:10929000B2C5EFFF010139A516D0036A0501B3512C
:1092A000A60FE96E050E0320EA6EEFCFB7F5B7C53E
:1092B00012F8370E0801136F00011BEC37F0200E77
:1092C0009EA8FED7AD6E0501B32BB68320D0010159
:1092D00039A516D05B0E9EA8FED7AD6EB2C512F8AA
:1092E000370E0801136F00011BEC37F05D0E9EA8CE
:1092F000FED7AD6E200E9EA8FED7AD6E07D0010141
:10930000320E0801116F0001D9EC26F00501320E72
:109310000801116F0001D9EC26F0F3D5010100011D
:10932000000C050E0401C26F810EC36F090EC46FDD
:10933000040EC56FC66BFF0EC76F050EC86F810E9A
:10934000C96F090ECA6FCB6B020ECC6FFF0ECD6FCB
:10935000050ECE6F810ECF6F090ED06F040ED16F48
:10936000330ED26FFF0ED36F050ED46F810ED56F03
:10937000090ED66F040ED76F480ED86FFF0ED96F47
:10938000050EDA6F810EDB6F090EDC6F040EDD6FE8
:109390003E0EDE6FFF0EDF6F050EE06F810EE16F98
:1093A000090EE26F040EE36F380EE46FFF0EE56FF7
:1093B000050EE66F810EE76F090EE86F040EE96F88
:1093C0004E0EEA6FFF0EEB6F050EEC6F810EED6F28
:1093D000090EEE6F040EEF6F470EF06FFF0EF16F88
:1093E000050EF26F810EF36F090EF46F060EF56F26
:1093F000120EF66FFF0EF76F050EF86F810EF96F04
:10940000090EFA6F040EFB6F480EFC6FFF0EFD6F26
:10941000090EFE6F810EFF6F010E0501006F040E35
:10942000016F4E0E026F036B046B056B066BFF0E34
:10943000076F060E086FFF0E096F880E0A6F010E88
:109440000B6F0C6B0D6FFF0E0E6F060E0F6F810E04
:10945000106F010E116F060E126F136F020E146F54
:10946000FF0E156F060E166F810E176F010E186F27
:10947000060E196F1A6F030E1B6FFF0E1C6F060E80
:109480001D6F810E1E6F010E1F6F040E206F216B6A
:10949000020E226FFF0E236F060E246F810E256FC2
:1094A000010E266F040E276F286B030E296FFF0E27
:1094B0002A6F060E2B6F810E2C6F010E2D6F040E7E
:1094C0002E6F330E2F6F020E306FFF0E316F060EB0
:1094D000326F810E336F010E346F040E356F330E11
:1094E000366F030E376FFF0E386F060E396F810E21
:1094F0003A6F010E3B6F040E3C6F350E3D6F3E6BB5
:10950000FF0E3F6F060E406F810E416F010E426FDE
:10951000040E436F350E446F030E456FFF0E466F0A
:10952000060E476F810E486F010E496F040E4A6F99
:109530003E0E4B6F020E4C6FFF0E4D6F060E4E6FC0
:10954000810E4F6F010E506F040E516F3E0E526F21
:10955000030E536FFF0E546F060E556F810E566F3C
:10956000010E576F040E586F380E596F020E5A6F66
:10957000FF0E5B6F060E5C6F810E5D6F010E5E6FFE
:10958000040E5F6F380E606F030E616FFF0E626F27
:10959000060E636F810E646F010E656F040E666FB9
:1095A000080E676F210E686FFF0E696F060E6A6FF7
:1095B000810E6B6F010E6C6F040E6D6F080E6E6F77
:1095C000310E6F6FFF0E706F060E716F810E726F2E
:1095D000010E736F040E746F080E756F766BFF0EBD
:1095E000776F050E786F810E796F010E7A6F060E18
:1095F0007B6F040E7C6FFF0E7D6F050E7E6F810EFC
:109600007F6F010E806F060E816F050E826FFF0E59
:10961000836F070E846F810E856F010E866F040EB7
:10962000876F3F0E886F010E896F8A6BFF0E8B6FFD
:10963000050E8C6F810E8D6F010E8E6F040E8F6F75
:10964000080E906FFF0E916F050E926F810E936F53
:10965000010E946F040E956F480E966FFF0E976F74
:10966000050E986F890E996F010E9A6F9B6F030E0E
:109670009C6FFF0E9D6F050E9E6F810E9F6F090EF2
:10968000A06F070EA16F220EA26FFF0EA36F040141
:10969000C051010A0001D8B49DD0030AD8B4A3D0A8
:1096A000010AD8B4A9D0070AD8B4AFD0010AD8B4F7
:1096B000B5D0030AD8B4BBD00E0AD8B4C1D0010AC1
:1096C000D8B4C7D0030AD8B4CDD00D0AD8B4D3D0FB
:1096D0000C0AD8B4D9D0070AD8B4DFD00C0AD8B451
:1096E000E5D00D0AD8B4EBD0030AD8B4F1D0010A02
:1096F000D8B4F7D01F0AD8B4FDD0010AD8B403D12A
:10970000020AD8B409D1070AD8B40FD1010AD8B4D3
:1097100023D1030AD8B437D1010AD8B43AD10F0AF9
:10972000D8B43DD1030AD8B46AD1070AD8B470D1ED
:10973000010AD8B476D1030AD8B48BD1010AD8B4BF
:10974000A0D13F0AD8B4A6D1170AD8B4ACD1020A26
:10975000D8B4B2D1010AD8B4C0D1020AD8B4CED19B
:109760000E0AD8B4DBD1010AD8B4DED11A0AD8B4B3
:10977000E1D1070AD8B4EBD1010AD8B4F5D1030A74
:10978000D8B4FAD1010AD8B400D20F0AD8B40AD298
:10979000010AD8B410D2030AD8B41BD2010AD8B433
:1097A00021D2070AD8B432D2010AD8B43ED2030A71
:1097B000D8B44AD2010AD8B451D21F0AD8B456D26A
:1097C000010AD8B45CD2030AD8B462D2080AD8B469
:1097D00068D270D2040E08010E6FC20E0D6F000128
:1097E000ECEC37F06DD2040E08010E6FC80E0D6F51
:1097F0000001ECEC37F064D2040E08010E6FCE0EBF
:109800000D6F0001ECEC37F05BD2040E08010E6F17
:10981000D40E0D6F0001ECEC37F052D2040E0801AB
:109820000E6FDA0E0D6F0001ECEC37F049D2040E2A
:1098300008010E6FE00E0D6F0001ECEC37F040D226
:10984000040E08010E6FE60E0D6F0001ECEC37F010
:1098500037D2040E08010E6FEC0E0D6F0001ECEC18
:1098600037F02ED2040E08010E6FF20E0D6F0001BC
:10987000ECEC37F025D2040E08010E6FF80E0D6FD8
:109880000001ECEC37F01CD2050E08010E6F0F0E34
:109890000D6F0001ECEC37F013D2050E08010E6FCE
:1098A000160E0D6F0001ECEC37F00AD2050E080120
:1098B0000E6F080E0D6F0001ECEC37F001D2050EB3
:1098C00008010E6F1D0E0D6F0001ECEC37F0F8D1A2
:1098D000050E08010E6F240E0D6F0001ECEC37F041
:1098E000EFD1050E08010E6F2B0E0D6F0001ECEC91
:1098F00037F0E6D1050E08010E6F320E0D6F000134
:10990000ECEC37F0DDD1050E08010E6F390E0D6F4E
:109910000001ECEC37F0D4D1050E08010E6F400EBB
:109920000D6F0001ECEC37F0CBD101014839006E2E
:109930000F0E0016005006080AE0050E08010E6F13
:10994000470E0D6F0001ECEC37F005D00101010E60
:10995000016EC5D10001B4D101014839006E0F0E6E
:109960000016005006080AE0050E08010E6F4E0EA4
:109970000D6F0001ECEC37F005D00101010E016E16
:10998000AED100019DD1020E01015227000E5323DA
:10999000000101015251D8B45307520700010101DF
:1099A000535307E15251010804E3536B010E526F08
:1099B00008D0535303E152510D0803E2536B0E0ECE
:1099C000526F5331036E5231026E03320232033250
:1099D0000232033202320F0E031602C005F50501F2
:1099E000010152510F0BE8CF06F50501040E0801E5
:1099F0000E6FFE0E0D6F0001ECEC37F061D1050E1D
:109A000008010E6F550E0D6F0001ECEC37F058D1C8
:109A1000050E08010E6F5C0E0D6F0001ECEC37F0C7
:109A20004FD101014839006E0F0E00160050060894
:109A300004E1020E0501686F03D0200E0501686F76
:109A4000050E08010E6F630E0D6F0001ECEC37F090
:109A500037D101014839006E0F0E0016005006087C
:109A600004E1030E05016F6F03D0300E05016F6F27
:109A7000050E08010E6F6A0E0D6F0001ECEC37F059
:109A80001FD1050E08010E6F710E0D6F0001ECEC79
:109A900037F016D1050E08010E6F8C0E0D6F000108
:109AA000ECEC37F00DD1050E08010E6F980E0D6F1E
:109AB0000001ECEC37F004D1010E0101865D0F0BC3
:109AC00005018A6F020E896F050E08010E6F840E64
:109AD0000D6F0001ECEC37F0F3D0010E0101865D53
:109AE0000F0B05018A6F010E896F050E08010E6FBD
:109AF000840E0D6F0001ECEC37F0E2D0010E010195
:109B0000865D0F0B05018A6F896B050E08010E6FCC
:109B1000840E0D6F0001ECEC37F0D2D0010E016E17
:109B20000101DDD00001CCD0010E016E0101D7D0C2
:109B30000001C6D00101415188090501A46F070148
:109B4000D56BD66BD76F0001F9EC39F0B9D00101B4
:109B5000415108090501A46F0701D56BD66BD76F7A
:109B60000001F9EC39F0ACD00701D56BD66BD76B9F
:109B70000001F9EC39F0A4D00701D56BD66B41C1D7
:109B8000D7F70001F9EC39F09BD001013D51800974
:109B90000501A46F0701D56BD66FD76B0001F9ECF7
:109BA00039F08ED00701D56B3DC1D6F7D76B0001D8
:109BB000F9EC39F085D001013E5180090501A46F0F
:109BC000E8CFD5F70701D66BD76B0001F9EC39F078
:109BD00077D03EC1D5F70701D66BD76B0001F9EC02
:109BE00039F06ED001013E5180090501A46F0101D9
:109BF0003D5180090501A56FA4C5D5F7E8CFD6F77B
:109C00000701D76B0001F9EC39F05AD001013D5141
:109C100080090501A46F3EC1D5F7E8CFD6F707014B
:109C2000D76B0001F9EC39F04BD001013E518009AE
:109C30000501A46FE8CFD5F73DC1D6F70701D76B73
:109C40000001F9EC39F03CD03EC1D5F73DC1D6F763
:109C50000701D76B0001F9EC39F032D00701D56B61
:109C6000D66BD76B0001F9EC39F02AD0050E08014C
:109C70000E6F920E0D6F0001ECEC37F021D0050E47
:109C800008010E6F780E0D6F0001ECEC37F018D064
:109C9000050E08010E6F7E0E0D6F0001ECEC37F023
:109CA0000FD0050E08010E6F9E0E0D6F0001ECEC3B
:109CB00037F006D0000E016E010111D0000100D076
:109CC0000401C12D09D0070E0501A56FD00EA46FA8
:109CD000000103EC47F00401010E016E01010001D7
:109CE000000C04018F6B906B916BA26B900EA36FB5
:109CF0000D0EC06F010EC16F000191EC49F0040E12
:109D0000EA6E920EE96E08010A6B0C6B100E0B6F77
:109D1000000186EC28F03A0E0401C06FC16B00010F
:109D200091EC49F0010139A510D00401A46BA451B4
:109D300000011EEC11F00401A42B006E00509EA83F
:109D4000FED7AD6E110EA45DF2E10001A8A143D0D3
:109D500090C43DFD8FC43CFD0D013F6B320E3E6F44
:109D60000001A2EC29F002C0A5F401C0A4F4040192
:109D7000A55303E1A451C70821E2010139A510D080
:109D80000401A46BA451000136EC11F00401A42BD2
:109D9000006E00509EA8FED7AD6E0B0EA45DF2E1E2
:109DA00004018E5308E10E0EC06F010EC16F000159
:109DB00091EC49F00401000E016E6AD0320E0801E8
:109DC000116F0001D9EC26F004018F2BD8B4902B31
:109DD0000101BBD70001A8B135D00401A25103088D
:109DE000D8B002D000012ED00001F3EC36F001C053
:109DF00091F40A0E0801116F0001D9EC26F004015C
:109E0000A351915D04E1A26B91C492F40AD0A22BFC
:109E1000036AA251920FE96E040E0320EA6E91C408
:109E2000EFFF010139A50CD091C412F8570E0801BB
:109E3000136F00011BEC37F0200E9EA8FED7AD6E0D
:109E40000001C9D7010139A508D00A0E9EA8FED786
:109E5000AD6E0D0E9EA8FED7AD6E0401A251030893
:109E60000BE1953D09D09351500806E19451020849
:109E700003E3010E016E0CD08E5308E10E0EC06F8D
:109E8000010EC16F000191EC49F00401000E016E5A
:109E90000001000C010148390401BF6F0F0EBF170C
:109EA000010EBF5DF20F15E20E0F00016BEF4FF0D8
:109EB000BDC4C0F4BEC4C1F491EC49F0040109D0A2
:109EC000BDC4C0F4BEC4C1F46DEC40F0040101D0C7
:109ED00004010001000CF2CF0EF0F29EE824F76AB4
:109EE000F736010FF66E9F0EF722000EF86EFB6E2E
:109EF0000A00F550FA6E0800F5500EBEF28EF96EAB
:109F0000B09EB09EB09EB09EB09EB09EB09EB09EE1
:109F1000B09EB09ED09EC09ED09EB09E0401656B48
:109F2000666B676B786B900E796F040EEA6E7A0E33
:109F3000E96E08010A6B0C6B140E0B6F000186ECC6
:109F400028F0040EEA6E680EE96E08010A6B0C6BCD
:109F5000100E0B6F000186EC28F0020E0401C06F9A
:109F6000C16B000191EC49F0010139A510D0040149
:109F70008E6B8E5100017CEC0EF004018E2B006E76
:109F800000509EA8FED7AD6E0E0E8E5DF2E1000170
:109F9000A8A138D066C43DFD65C43CFD0D013F6BF2
:109FA000320E3E6F0001A2EC29F002C08FF401C016
:109FB0008EF404018F5303E18E51C70816E20101AC
:109FC00039A511D004018E6B8E51000193EC0EF077
:109FD00004018E2B006E00509EA8FED7AD6E0A0EB7
:109FE0008E5DF2E10101CCEF53F0320E0801116FEA
:109FF0000001D9EC26F00401652BD8B4662B0101D1
:10A00000C6D70001A8B135D0040178510F08D8B0E7
:10A0100002D000012ED00001F3EC36F001C067F44D
:10A020000A0E0801116F0001D9EC26F004017951E4
:10A03000675D04E1786B67C468F40AD0782B036A23
:10A040007851680FE96E040E0320EA6E67C4EFFFD3
:10A05000010139A50CD067C412F8570E0801136F1F
:10A0600000011BEC37F0200E9EA8FED7AD6E00015C
:10A07000C9D7010139A508D00A0E9EA8FED7AD6E3A
:10A080000D0E9EA8FED7AD6E040178510408D8B01D
:10A0900007D36AC462F46BC461F46CC464F46DC425
:10A0A00063F463C400F064C403F0040E645D06E16D
:10A0B000020E005C0001D8B464D00401080E035CF9
:10A0C00005E100520001D8B4C6D00401040E035CBF
:10A0D00006E10D0E005C0001D8B4FBD00401040EB3
:10A0E000035C06E10E0E005C0001D8B428D1040127
:10A0F000050E035C06E1030E005C0001D8B456D1E6
:10A100000401050E035C06E1010E005C0001D8B4F9
:10A110004DD10401040E035C06E10F0E005C00014A
:10A12000D8B4B0D10401050E035C06E1050E005C55
:10A130000001D8B4DDD10401050E035C06E1040E74
:10A14000005C0001D8B40BD20401040E035C06E1EC
:10A150002C0E005C0001D8B438D20401200E035C40
:10A1600006E1010E005C0001D8B42FD20401040EF8
:10A17000035C06E12D0E005C0001D8B426D2040178
:10A180005BD20101486B010E04018E6F0001A9DD55
:10A19000012C2CD0600E0101481339A511D0040107
:10A1A0008E6B8E510001A8EC0EF004018E2B006E18
:10A1B00000509EA8FED7AD6E140E8E5DF2E1010137
:10A1C000040EEA6E7A0EE96EF2CF8EF4F29E000E65
:10A1D0000001C2EC0EF00A000900F550EE6E000915
:10A1E000FBE104018EBFF28E2AD0000101014889F3
:10A1F00039A511D004018E6B8E510001DAEC0EF0FE
:10A2000004018E2B006E00509EA8FED7AD6E100E7E
:10A210008E5DF2E10101040EEA6E7A0EE96EF2CF74
:10A220008EF4F29E000E0001F2EC0EF00A0009001E
:10A23000F550EE6E0009FBE104018EBFF28E605115
:10A2400030098A6F040E0701E36F7A0EE26F000196
:10A25000F0EC30F023D20101486B500E481339A5C1
:10A2600011D004018E6B8E5100010AEC0FF0040135
:10A270008E2B006E00509EA8FED7AD6E140E8E5D24
:10A28000F2E10101040EEA6E7A0EE96EF2CF8EF46D
:10A29000F29E000E000124EC0FF00A000900F550B8
:10A2A000EE6E0009FBE104018EBFF28E60513009B1
:10A2B0008A6F040E0701E36F7A0EE26F0001F0EC83
:10A2C00030F0370E0401BD6F010EBE6F0001E2DDFC
:10A2D000E5D10101486B488B39A511D004018E6B83
:10A2E0008E5100013CEC0FF004018E2B006E0050EB
:10A2F0009EA8FED7AD6E110E8E5DF2E10101040E37
:10A30000EA6E7A0EE96EF2CF8EF4F29E000E000134
:10A3100054EC0FF00A000900F550EE6E0009FBE165
:10A3200004018EBFF28E605130098A6F040E07015E
:10A33000E36F7A0EE26F0001F0EC30F0AFD1010173
:10A34000486B300E481339A511D004018E6B8E5125
:10A3500000016CEC0FF004018E2B006E00509EA8E3
:10A36000FED7AD6E100E8E5DF2E10101040EEA6EB5
:10A370007A0EE96EF2CF8EF4F29E000E000184ECAC
:10A380000FF00A000900F550EE6E0009FBE1040130
:10A390008EBFF28E605130098A6F040E0701E36FA1
:10A3A0007A0EE26F0001F0EC30F078D10401632DF9
:10A3B00033D06451050830E1612D2ED062532CE179
:10A3C0000101486B900E481339A511D004018E6B22
:10A3D0008E5100019CEC0FF004018E2B006E00509A
:10A3E0009EA8FED7AD6E110E8E5DF2E10101040E46
:10A3F000EA6E7A0EE96EF2CF8EF4F29E000E000144
:10A40000B4EC0FF00A000900F550EE6E0009FBE114
:10A4100004018EBFF28E2AD00101486B488939A50C
:10A4200011D004018E6B8E510001CCEC0FF00401B1
:10A430008E2B006E00509EA8FED7AD6E0F0E8E5D67
:10A44000F2E10101040EEA6E7A0EE96EF2CF8EF4AB
:10A45000F29E000E0001E3EC0FF00A000900F55037
:10A46000EE6E0009FBE104018EBFF28E60513009EF
:10A470008A6F040E0701E36F7A0EE26F0001F0ECC1
:10A4800030F00CD10101486B488F39A511D004017F
:10A490008E6B8E510001FBEC0FF004018E2B006ED1
:10A4A00000509EA8FED7AD6E100E8E5DF2E1010148
:10A4B000040EEA6E7A0EE96EF2CF8EF4F29E000E72
:10A4C000000113EC10F00A000900F550EE6E0009CF
:10A4D000FBE104018EBFF28E605130098A6F040ED9
:10A4E0000701E36F7A0EE26F0001F0EC30F0D6D096
:10A4F0000101486B700E481339A511D004018E6B11
:10A500008E5100012BEC10F004018E2B006E0050D8
:10A510009EA8FED7AD6E110E8E5DF2E10101040E14
:10A52000EA6E7A0EE96EF2CF8EF4F29E000E000112
:10A5300043EC10F00A000900F550EE6E0009FBE153
:10A5400004018EBFF28E605130098A6F040E07013C
:10A55000E36F7A0EE26F0001F0EC30F09FD0010162
:10A56000486B488D39A511D004018E6B8E510001C6
:10A570005BEC10F004018E2B006E00509EA8FED7FD
:10A58000AD6E100E8E5DF2E10101040EEA6E7A0EE0
:10A59000E96EF2CF8EF4F29E000E000173EC10F023
:10A5A0000A000900F550EE6E0009FBE104018EBFC0
:10A5B000F28E605130098A6F040E0701E36F7A0E44
:10A5C000E26F0001F0EC30F069D00101486BA00EA1
:10A5D000481339A511D004018E6B8E5100018BEC0C
:10A5E00010F004018E2B006E00509EA8FED7AD6EB9
:10A5F000160E8E5DF2E10101040EEA6E7A0EE96E2E
:10A60000F2CF8EF4F29E000E0001A6EC10F00A00CC
:10A610000900F550EE6E0009FBE104018EBFF28ED9
:10A62000605130098A6F040E0701E36F7A0EE26F02
:10A630000001F0EC30F032D0010139A511D0040155
:10A640008E6B8E510001BEEC10F004018E2B006E5B
:10A6500000509EA8FED7AD6E100E8E5DF2E1010196
:10A66000486B040EEA6E7A0EE96EF2CF8EF4F29E1B
:10A67000000E0001D6EC10F00A000900F550EE6E55
:10A680000009FBE104018EBFF28E040E0701E36FA7
:10A690007A0EE26F0001F0EC30F000D07CD00401C3
:10A6A0007851030847E16B3D45D06951600803E0EC
:10A6B000695161083FE18E6B000171EC4EF0012C95
:10A6C00039D00101486B600E481339A511D004013F
:10A6D0008E6B8E510001EDEC10F004018E2B006E9C
:10A6E00000509EA8FED7AD6E130E8E5DF2E1010103
:10A6F000040EEA6E7A0EE96EF2CF8EF4F29E000E30
:10A70000000106EC11F00A000900F550EE6E000998
:10A71000FBE104018EBFF28E605130098A6F040E96
:10A720000701E36F7A0EE26F0001F0EC30F00101F7
:10A7300033D00001010139A511D004018E6B8E5177
:10A740000001BEEC10F004018E2B006E00509EA89C
:10A75000FED7AD6E100E8E5DF2E10101486B040E66
:10A76000EA6E7A0EE96EF2CF8EF4F29E000E0001D0
:10A77000D6EC10F00A000900F550EE6E0009FBE17E
:10A7800004018EBFF28E040E0701E36F7A0EE26FB2
:10A790000001F0EC30F001010001BBEF60F00701B7
:10A7A000E36BE46BE56BE66BE76BE25303E0E251CE
:10A7B00006082AE2E86BE851000185EC08F0070181
:10A7C000E82B006E00509EA8FED7AD6E190EE85D16
:10A7D000F2E1E2C7E9F71F0EEA6F00016EEC37F015
:10A7E0001B0E0701E96FE951000185EC08F0070134
:10A7F000E92B006E00509EA8FED7AD6E210EE95DDC
:10A80000F2E1000E016E7CD0E2C7CFF1E66B010EE3
:10A81000E56FE65375E1E5510C0872E3E46B900EC9
:10A82000E36F010EE25D036AE86F03C0E9F7E4C776
:10A830003DFDE3C73CFD03C03FFDE8CF3EFD000109
:10A84000A2EC29F002C0E4F701C0E3F7200E0701F3
:10A85000E327000EE423010EE55DE86F000EE659E4
:10A86000E96FE8CF3DFDE8C73CFD0D013F6B0C0EE5
:10A870003E6F0001A2EC29F001500701E3270250CE
:10A88000E423F2CFE8F7F29EE4C7AAFFE3C7A9FFEB
:10A89000A69CA69EA680A850E8BFF28EE76FE7515F
:10A8A000F00B09E0CF0EE525E96E010EE621EA6E18
:10A8B000FF0EEF6E07D0CF0EE525E96E010EE62103
:10A8C000EA6EEF6A010139A516D0CF0E0701E52522
:10A8D000E96E010EE621EA6EEFCFE8F7E8C712F85D
:10A8E000570E0801136F00011BEC37F0200E9EA8D5
:10A8F000FED7AD6E01010701E52BD8B4E62B89D751
:10A900000001000C0F0E0401756F810E766F010EB1
:10A91000776F060E786F020E796F7A6B7B6B7C6BAC
:10A920007D6B7E6B7F6B806B816B826B836BFF0EAD
:10A93000846F856F090E866F810E876F010E886F99
:10A94000040E896F470E8A6F8B6B8C6B8D6B8E6BD1
:10A95000FF0E8F6F090E906F810E916F010E926F37
:10A96000040E936F480E946F956B966B976B986B74
:10A97000FF0E996F090E9A6F810E9B6F010E9C6FEF
:10A98000040E9D6F4E0E9E6F9F6BA06BA16BA26B12
:10A99000FF0EA36F070EA46F01014839006E0F0E62
:10A9A000001600500A08D8B4CCD03EC17AF43DC19C
:10A9B0007BF44839006E0F0E0016005008080EE0B8
:10A9C0004839006E0F0E00160050070807E048399E
:10A9D000006E0F0E00160050090811E10401752BDE
:10A9E000036AA451750FE96E040E0320EA6E01019B
:10A9F00049510F0BEF6E0401A42B7B6B0101036A1D
:10AA00000401A451750FE96E040E0320EA6E0101E2
:10AA10004B390401A76F0F0EA717A7510F0BEF6E4D
:10AA2000010EA425036A750FE96E040E0320EA6E79
:10AA30004BC1A8F4A8510F0BEF6E020EA425036AB8
:10AA4000750FE96E040E0320EA6E01014B3104011B
:10AA5000A96F01014A310401A86FA933A833A933B2
:10AA6000A833A933A8330F0EA917A8510F0BEF6E07
:10AA7000030EA425036A750FE96E040E0320EA6E27
:10AA800001014A510F0BEF6E040E0401A425036A65
:10AA9000750FE96E040E0320EA6E01014D390401C1
:10AAA000A86F0F0EA817A8510F0BEF6E050EA42567
:10AAB000036A750FE96E040E0320EA6E4DC1A8F417
:10AAC000A8510F0BEF6E060EA425036A750FE96EF1
:10AAD000040E0320EA6E01014D310401A96F01014A
:10AAE0004C310401A86FA933A833A933A833A93383
:10AAF000A8330F0EA917A8510F0BEF6E070EA42550
:10AB0000036A750FE96E040E0320EA6E01014C51D1
:10AB10000F0BEF6E040E08010E6F750E0D6F000126
:10AB2000ECEC37F04E0E0501A56F200EA46F00016E
:10AB300003EC47F0012C01D003D0000E016E2DD1A3
:10AB400001014F390401A56F0F0EA517A5510F0B79
:10AB50008B6F4FC1A5F4A5510F0B8C6F01014F31C5
:10AB60000401A66F01014E310401A56FA633A53380
:10AB7000A633A533A633A5330F0EA617A5510F0B89
:10AB80008D6F01014E510F0BE8CF8EF40401040EBE
:10AB900008010E6F860E0D6F0001ECEC37F0070E0A
:10ABA0000501A56FD00EA46F000103EC47F0012C46
:10ABB00001D003D0000E016EF0D0010148A70AD0E9
:10ABC0001B0E0401BD6F010EBE6F00014AEC4FF079
:10ABD00046D001011C0E0401BD6F010EBE6F0001C5
:10ABE0004AEC4FF0010151390401A56F0F0EA51772
:10ABF000A5510F0B956F51C1A5F4A5510F0B966F81
:10AC0000010151310401A66F010150310401A56F0A
:10AC1000A633A533A633A533A633A5330F0EA61747
:10AC2000A5510F0B976F010150510F0BE8CF98F40E
:10AC30000401040E08010E6F900E0D6F0001ECEC84
:10AC400037F0030E0501A56FE80EA46F000103ECB9
:10AC500047F0012C01D003D0000E016E9ED00101FF
:10AC600048A542D0140E0401BD6F010EBE6F000155
:10AC70004AEC4FF00101536B070E526FD8908535A7
:10AC8000036A350F016E000E03220150380FE96E82
:10AC9000010E0320EA6E53C1ECFFED5252C1EFFFEB
:10ACA00004019F6BA06BA16B010152510F0BE8CF08
:10ACB000A2F40401040E08010E6F9A0E0D6F00013C
:10ACC000ECEC37F0030E0501A56FE80EA46F000150
:10ACD00003EC47F0150E0401BD6F010EBE6F0001BD
:10ACE0004AEC4FF046D00101140E0401BD6F010E75
:10ACF000BE6F00014AEC4FF0010153390401A56F0A
:10AD00000F0EA517A5510F0B9F6F53C1A5F4A551A9
:10AD10000F0BA06F010153310401A66F01015231E5
:10AD20000401A56FA633A533A633A533A633A533F7
:10AD30000F0EA617A5510F0BA16F010152510F0B5A
:10AD4000E8CFA2F40401040E08010E6F9A0E0D6FF5
:10AD50000001ECEC37F0030E0501A56FE80EA46FBF
:10AD6000000103EC47F0012C01D003D0000E016E6E
:10AD700014D0010148A109D00F0E0401BD6F010ECE
:10AD8000BE6F00014AEC4FF008D0100E0401BD6FF9
:10AD9000010EBE6F00014AEC4FF03FEF5DF0040181
:10ADA000CC6BCD6BCE6BCF91040EEA6EBF0EE96E0D
:10ADB00008010A6B0C6B0D0E0B6F000186EC28F07E
:10ADC000A8A154D0CEC43DFDCDC43CFD0D013F6BC8
:10ADD000190E3E6F0001A2EC29F002C0D1F401C0AF
:10ADE000D0F40401BE51025C35E303E1BD51D05DF6
:10ADF00031E3010139A52BD00401D06BD051000102
:10AE00001DEC12F00401D02B006E00509EA8FED75E
:10AE1000AD6E180ED05DF2E1100EE96EBEC401F801
:10AE2000BDC400F8000139EC38F01B0E0401D16FED
:10AE3000D15100011DEC12F00401D12B006E005025
:10AE40009EA8FED7AD6E220ED15DF2E10101FF0E8C
:10AE5000016EF6D0190E0801116F0001D9EC26F031
:10AE60000401CD2BD8B4CE2B0001AAD7010139A5FE
:10AE700010D00401D06BD05100013EEC12F004015F
:10AE8000D02B006E00509EA8FED7AD6E100ED05D88
:10AE9000F2E10001A8B1D1D0036A0401CC51BF0F87
:10AEA000016E040E032201C0D0F403C0D1F40001EE
:10AEB000F3EC36F0D1C4EAFFD0C4E9FF01C0EFFFE4
:10AEC000010139A516D0036A0401CC51BF0FE96E08
:10AED000040E0320EA6EEFCFD0F4D0C412F8370E80
:10AEE0000801136F00011BEC37F0200E9EA8FED75F
:10AEF000AD6E0401CFB117D0036ACC51BF0FE96E1C
:10AF0000040E0320EA6EEF50FE080CE1036ACC51F8
:10AF1000BF0FE96E040E0320EA6EEFCFBFF4CF81BE
:10AF2000010ECC6F80D0036ACC51BF0FE96E040EC6
:10AF30000320EA6EEF50EF0868E1010139A508D05F
:10AF40000D0E9EA8FED7AD6E0A0E9EA8FED7AD6E62
:10AF500039A54BD00401C2510F0B006E0038D16FE0
:10AF6000F00ED117C3510F0BD111D26FD36BD35148
:10AF7000000156EC12F00401D32B006E00509EA885
:10AF8000FED7AD6E0D0ED35DF2E1C2C412F8570EBE
:10AF90000801136F00011BEC37F02C0E9EA8FED7A2
:10AFA000AD6EC3C412F8570E0801136F00011BECFD
:10AFB00037F0200E9EA8FED7AD6E280E9EA8FED7B5
:10AFC000AD6ED2C412F8570E0801136F00011BECCE
:10AFD00037F0290E9EA8FED7AD6E0D0E9EA8FED7A7
:10AFE000AD6E0A0E9EA8FED7AD6E0401C2510F0BC6
:10AFF000006E0038D16FF00ED117C3510F0BD11175
:10B00000016E01011DD007D00401320E0801116F3D
:10B010000001D9EC26F00401CC510B0802E3CC2B43
:10B0200002D0CC6BCF910001A8A106D0320E08014E
:10B03000116F0001D9EC26F02DD7EE0E016E010143
:10B040000001000C0E0E0401756FFF0E766F300EBE
:10B05000776F786F796B620E7A6F7B6B7C6B7D6B31
:10B060007E6B7F6B806B816B826BEF0E836F0A0E42
:10B07000846FFF0E856F300E866F876F886BB30EFF
:10B08000896F8A6B8B6B8C6B8D6BEF0E8E6F0A0EDC
:10B090008F6FFF0E906F300E916F926F936BB00EAB
:10B0A000946F956B966B976B986BEF0E996F090E7B
:10B0B0009A6FFF0E9B6F300E9C6F9D6F9E6B500EB4
:10B0C0009F6FA06BA16BA26BEF0EA36F090EA46F15
:10B0D000FF0EA56F300EA66FA76FA86B510EA96F5C
:10B0E000AA6BAB6BAC6BEF0EAD6F080EAE6FFF0EC5
:10B0F000AF6F300EB06FB16FB26BB40EB36F310E75
:10B10000B46FB56BEF0EB66FB76BB86BB96BBA6B4C
:10B11000BB6BBC6B036A3EC1BDF403C0BEF40D0142
:10B120003D6B210E3C6F03C03FFD3EC13EFD000163
:10B13000A2EC29F0080E04010124B96F000E0220D0
:10B14000BA6FBA5306E1B951090803E3BA6B0A0EA4
:10B15000B96FBA51020809E2FF0A03E1B9512008A8
:10B1600004E2030EBA6F200EB96FBA510F0BBE6F17
:10B17000E8CF10F80001D6EC3AF001C0A0F40401C9
:10B18000B9C400F0003A0F0E001600500F0BBF6F4D
:10B19000E8CF10F80001D6EC3AF001C0A1F40401A8
:10B1A000B9510F0BBE6FE8CF10F80001D6EC3AF0A2
:10B1B00001C0A2F4040E08010E6F9A0E0D6F00017B
:10B1C000ECEC37F0030E0401BE6FE80EBD6F00011A
:10B1D000E6DD01C0BCF40401BC5330E0BC511008F2
:10B1E00003E0BC51500824E1020EBD6FFA0E0801C5
:10B1F000116F0001D9EC26F00401BD2FF7D7040E22
:10B2000008010E6F9A0E0D6F0001ECEC37F0030E83
:10B210000501C96FE80EC86F000164EC3FF0012C16
:10B2200001D004D0000E016E1DEF5DF006D00401C8
:10B23000000E016E00011DEF5DF00401036A3DC1C7
:10B24000BDF403C0BEF40D013D6B1E0E3C6F03C088
:10B250003FFD3DC13EFD0001A2EC29F0080E0401B6
:10B260000124B76F000E0220B86FB85306E1B75142
:10B27000070803E3B86B080EB76FB851010809E27D
:10B28000FF0A03E1B7516E0804E2020EB86F6E0EBA
:10B29000B76FB8510F0BBE6FE8CF10F80001D6ECB6
:10B2A0003AF001C0AAF40401B7C400F0003A0F0E4E
:10B2B000001600500F0BBF6FE8CF10F80001D6EC5E
:10B2C0003AF001C0ABF40401B7510F0BBE6FE8CFE9
:10B2D00010F80001D6EC3AF001C0ACF4040E0801FD
:10B2E0000E6FA40E0D6F0001ECEC37F0030E04019D
:10B2F000BE6FE80EBD6F000152DD01C0BCF4040159
:10B30000BC532DE0BC51100803E0BC51500823E1B0
:10B31000020EBD6FFA0E0801116F0001D9EC26F084
:10B320000401BD2FF7D7040E08010E6FA40E0D6F98
:10B330000001ECEC37F0030E0501C96FE80EC86F91
:10B34000000164EC3FF0012C01D003D0000E016E2F
:10B3500074D305D00401000E016E00016ED301010B
:10B360004B390401BD6FBE6B0F0EBD17BD510F0BE6
:10B37000006E036ABF6FE8CF10F80001D6EC3AF018
:10B3800001C07BF44BC1BDF40401BE6BBD510F0B7A
:10B39000006E036ABF6FE8CF10F80001D6EC3AF0F8
:10B3A00001C07CF401014B310401BE6F01014A313F
:10B3B0000401BD6FBE33BD33BE33BD33BE33BD33B9
:10B3C0000F0EBE17BD510F0B006E036ABF6FE8CFA3
:10B3D00010F80001D6EC3AF001C07DF401014A51A9
:10B3E0000F0B006E036AE8CFBDF4E8CF10F8000140
:10B3F000D6EC3AF001C07EF401014D390401BD6F75
:10B40000BE6B0F0EBD17BD510F0B006E036ABF6FF1
:10B41000E8CF10F80001D6EC3AF001C07FF44DC13E
:10B42000BDF40401BE6BBD510F0B006E036ABF6F0C
:10B43000E8CF10F80001D6EC3AF001C080F4010129
:10B440004D310401BE6F01014C310401BD6FBE33AB
:10B45000BD33BE33BD33BE33BD330F0EBE17BD513A
:10B460000F0B006E036ABF6FE8CF10F80001D6EC37
:10B470003AF001C081F401014C510F0B006E036AD8
:10B48000E8CFBDF4E8CF10F80001D6EC3AF001C0E7
:10B4900082F4040E08010E6F750E0D6F0001ECECC6
:10B4A00037F0170E0401BE6F700EBD6F000177DC20
:10B4B00001C0BCF40401BC532EE0BC51100803E0F1
:10B4C000BC51500823E1080EBD6FFA0E0801116F40
:10B4D0000001D9EC26F00401BD2FF7D7040E0801B6
:10B4E0000E6F750E0D6F0001ECEC37F0070E0501C5
:10B4F000C96FD00EC86F000164EC3FF0012C01D081
:10B5000003D0000E016E99D205D00401000E016E29
:10B51000000193D20401BB5301E1BB6BBB5107088F
:10B5200002E2070EBB6F370EB56F040E08010E6FF7
:10B53000AE0E0D6F0001ECEC37F0030E0401BE6F90
:10B54000E80EBD6F00012BDC01C0BCF40401BC534C
:10B550002DE0BC51100803E0BC51500823E1020E5D
:10B56000BD6FFA0E0801116F0001D9EC26F004013D
:10B57000BD2FF7D7040E08010E6FAE0E0D6F000140
:10B58000ECEC37F0030E0501C96FE80EC86F00013F
:10B5900064EC3FF0012C01D003D0000E016E4DD2BF
:10B5A00005D00401000E016E000147D201014F39A0
:10B5B0000401BD6FBE6B0F0EBD17BD510F0B006EAA
:10B5C000036ABF6FE8CF10F80001D6EC3AF001C073
:10B5D0008AF44FC1BDF40401BE6BBD510F0B006E68
:10B5E000036ABF6FE8CF10F80001D6EC3AF001C053
:10B5F0008BF401014F310401BE6F01014E31040192
:10B60000BD6FBE33BD33BE33BD33BE33BD330F0E4E
:10B61000BE17BD510F0B006E036ABF6FE8CF10F865
:10B620000001D6EC3AF001C08CF401014E510F0B31
:10B63000006E036AE8CFBDF4E8CF10F80001D6EC45
:10B640003AF001C08DF4040E08010E6F840E0D6FE8
:10B650000001ECEC37F0030E0401BE6FE80EBD6F85
:10B660000001CFEC56F001C0BCF40401BC5328E04B
:10B67000BC51100803E0BC51500822E1080EBD6F18
:10B68000FA0E0801116F0001D9EC26F00401BD2F5C
:10B69000F7D7040E08010E6F840E0D6F0001ECEC5D
:10B6A00037F0070E0501C96FD00EC86F000164ECBA
:10B6B0003FF0012C01D003D0000E016EBED1040179
:10B6C000010148A742D01B0E0401BD6FBE6B0001F3
:10B6D0004AEC4FF0030E0401BE6FE80EBD6F00018F
:10B6E000CFEC56F001C0BCF40401BC532CE0BC51BB
:10B6F000100803E0BC51500821E1040EBD6FFA0EA2
:10B700000801116F0001D9EC26F00401BD2FF7D715
:10B710001B0EBD6FBE6B00014AEC4FF0030E05011E
:10B72000C96FE80EC86F000164EC3FF0012C01D036
:10B7300003D0000E016E81D105D00401000E016E10
:10B7400000017BD10401FCD001011C0E0401BD6F7E
:10B75000BE6B00014AEC4FF0030E0401BE6FE80E11
:10B76000BD6F0001CFEC56F001C0BCF40401BC5326
:10B770002BE0BC51100803E0BC51500821E1040E3D
:10B78000BD6FFA0E0801116F0001D9EC26F004011B
:10B79000BD2FF7D71C0EBD6FBE6B00014AEC4FF0FA
:10B7A000030E0501C96FE80EC86F000164EC3FF09D
:10B7B000012C01D003D0000E016E3FD105D0040151
:10B7C000000E016E000139D1010151390401BD6F34
:10B7D000BE6B0F0EBD17BD510F0B006E036ABF6F1E
:10B7E000E8CF10F80001D6EC3AF001C095F451C151
:10B7F000BDF40401BE6BBD510F0B006E036ABF6F39
:10B80000E8CF10F80001D6EC3AF001C096F401013F
:10B8100051310401BE6F010150310401BD6FBE33CF
:10B82000BD33BE33BD33BE33BD330F0EBE17BD5166
:10B830000F0B006E036ABF6FE8CF10F80001D6EC63
:10B840003AF001C097F4010150510F0B006E036AEA
:10B85000E8CFBDF4E8CF10F80001D6EC3AF001C013
:10B8600098F4040E08010E6F8F0E0D6F0001ECECC2
:10B8700037F0070E0401BE6FD00EBD6F0001CFEC94
:10B8800056F001C0BCF40401BC535AE0BC5110088E
:10B8900003E0BC5150084FE1080EBD6FFA0E0801DD
:10B8A000116F0001D9EC26F00401BD2FF7D7040E6B
:10B8B00008010E6F8F0E0D6F0001ECEC37F0070ED4
:10B8C0000401BE6FD00EBD6F0001CFEC56F001C079
:10B8D000BCF40401BC532EE0BC51100803E0BC5181
:10B8E000500823E1080EBD6FFA0E0801116F000128
:10B8F000D9EC26F00401BD2FF7D7040E08010E6F16
:10B900008F0E0D6F0001ECEC37F0070E0501C96FCB
:10B91000D00EC86F000164EC3FF0012C01D003D0C1
:10B92000000E016E8AD005D00401000E016E0001E8
:10B9300084D0040105D0000E016E00017ED0040108
:10B94000010148A309D0110E0401BD6F010EBE6FA5
:10B9500000014AEC4FF008D0130E0401BD6F010E38
:10B96000BE6F00014AEC4FF0640E0801116F000138
:10B97000D9EC26F0010148B10AD0100E0401BD6FC8
:10B98000010EBE6F00014AEC4FF009D001010F0E0D
:10B990000401BD6F010EBE6F00014AEC4FF0640E52
:10B9A0000801116F0001D9EC26F0010148A52FD044
:10B9B000536B480E526FD8908535036A350F016E70
:10B9C000000E03220150380FE96E010E0320EA6ECB
:10B9D00053C1ECFFED5252C1EFFF140E0401C06FD2
:10B9E000010EC16F00016DEC40F0180E0401C06F34
:10B9F000010EC16F00016DEC40F0150E0401C06F27
:10BA0000010EC16F00016DEC40F011D00101140E68
:10BA10000401C06F010EC16F00016DEC40F0180E03
:10BA20000401C06F010EC16F00016DEC40F0640EA7
:10BA30000801116F0001D9EC26F044EF5DF001011F
:10BA40004839006E0F0E00160050020A000115E082
:10BA5000010A13E0060A11E00D0A0FE0010A0DE0E9
:10BA60000E0A0BE0030A09E0050A07E0070A05E0F1
:10BA70000C0A03E0060A06E00AD082EF54F00150F7
:10BA80000AD009D022EF58F0015005D004D0000EA2
:10BA9000016E01D000D0000C60C4E2F7CFEC53F08F
:10BAA0000101DB3D2AD060C475F40C0E0401766FF1
:10BAB000000181EC34F0012C1FD0040EEA6E610EFF
:10BAC000E96EF2CF75F4F29E000ED3EC1DF00A0081
:10BAD0000900F550EE6E0009FBE1040175BFF28E1E
:10BAE000040E0701E36F610EE26F0001F0EC30F02D
:10BAF000A6DF010E016E2BD00101040EEA6E610E6D
:10BB0000E96EF2CF75F4F29E000E0001EBEC1DF031
:10BB10000A000900F550EE6E0009FBE1040175BF53
:10BB2000F28E040E0701E36F610EE26F0001F0EC8C
:10BB300030F0080E0401756FFA0E0701CE6F000198
:10BB4000C4EC26F00401752FF7D7000E016E00013A
:10BB5000000C04017E51390805E2370E7E5D016E4E
:10BB600005D004D0300E7E5D016E00D00001000CC7
:10BB70000401756B766B776B020E786F900E796FA0
:10BB800063C4E9FF64C4EAFFEC6AED52EF6A040E95
:10BB9000EA6E650EE96E08010A6B0C6B100E0B6FF6
:10BBA000000186EC28F001014839006E0F0E0016E6
:10BBB00000500C0805E1050E0401786FFE0E796F48
:10BBC000020E04017A6FC80E0801116F0001D9EC52
:10BBD00026F004017A2FF7D70001A8B13CD0040168
:10BBE00075510F08D8B002D0000135D00001F3EC38
:10BBF00036F001C076F40A0E0801116F0001D9EC8D
:10BC000026F0010139A50ED076C412F8570E0801AE
:10BC1000136F00011BEC37F0200E9EA8FED7AD6E0F
:10BC200007D001010A0E0801116F0001D9EC26F0BE
:10BC300004017951765D04E1756B76C465F40AD030
:10BC4000752B036A7551650FE96E040E0320EA6EC9
:10BC500076C4EFFFC1D7030E04017825755D03E2BA
:10BC6000000E016E6DD001014839006E0F0E0016F6
:10BC700000500C0829E178C477F4030E04017825FC
:10BC8000775D01E022E2036A7751650F016E040ED1
:10BC9000032201C07AF403C07BF4036A7751650F75
:10BCA000E96E040E0320EA6EEFCF7CF47CC47EF4D0
:10BCB00000014FDF7BC4EAFF7AC4E9FF01C0EFFF58
:10BCC0000401772B0101D9D70401776B7751030861
:10BCD00035E363C4E9FF64C4EAFFEF34026EEC3479
:10BCE000036E023603360236033602360336F00E92
:10BCF00002160250ED52EF6E03C0ECFF64C403F075
:10BD000064C4EAFF63C4E9FFECCF7DF4ED52EFCFEA
:10BD10007CF477517825036A650FE96E040E0320E1
:10BD2000EA6EEF500F0B7C1164C4EAFF63C4E9FFB5
:10BD30007DC4ECFFED52EF6E772BC8D7010E016E7C
:10BD40000001000C0401756B766B020E776F900E8C
:10BD5000786F63C4E9FF64C4EAFFEF6A040EEA6E19
:10BD6000650EE96E08010A6B0C6B100E0B6F00017B
:10BD700086EC28F001014839006E0F0E00160050C5
:10BD80000C0805E1050E0401776FFE0E786F020EB8
:10BD90000401796FC80E0801116F0001D9EC26F07B
:10BDA0000401792FF7D70001A8B13CD004017551E7
:10BDB0000F08D8B002D0000135D00001F3EC36F006
:10BDC00001C076F40A0E0801116F0001D9EC26F0CB
:10BDD000010139A50ED076C412F8570E0801136F71
:10BDE00000011BEC37F0200E9EA8FED7AD6E07D0E9
:10BDF00001010A0E0801116F0001D9EC26F00401BF
:10BE00007851765D04E1756B76C465F40AD0752BC4
:10BE1000036A7551650FE96E040E0320EA6E76C45D
:10BE2000EFFFC1D7020E04017725755D03E2000E16
:10BE3000016E7CD001014839006E0F0E00160050D3
:10BE40000C083EE1036A04017751650F016E040E90
:10BE5000032201C079F403C07AF4036A7751650FB5
:10BE6000E96E040E0320EA6EEFCF7BF47BC47EF410
:10BE700000016FDE7AC4EAFF79C4E9FF01C0EFFF79
:10BE8000010E04017725036A650F016E040E03227B
:10BE900001C07AF403C07BF4010E7725036A650FB5
:10BEA000E96E040E0320EA6EEFCF7DF47DC47EF4CC
:10BEB00000014FDE7BC4EAFF7AC4E9FF01C0EFFF57
:10BEC00064C403F00401036A7751650FE96E040E40
:10BED0000320EA6EEFCF7BF464C4EAFF63C4E9FF9A
:10BEE0007BC4EFFF63C4E9FF64C4EAFFEF38006E70
:10BEF000F00E001600C0EFFF64C403F064C4EAFF54
:10BF000063C4E9FFEFCF7BF4010E7725036A650F69
:10BF1000E96E040E0320EA6EEF500F0B7B1164C430
:10BF2000EAFF63C4E9FFEF6E010E016E0001000C31
:10BF30000401606B616B626B0001EFEC39F0010191
:10BF40004839006E0F0E001600500C0816E0080E5F
:10BF50000401C06FC16B000191EC49F0040E0401B3
:10BF6000646F610E636F000103DE012C04D062C4B4
:10BF700053F161C452F116D00101080E0401C06FE3
:10BF8000C16B00016DEC40F0040E0401646F600EA3
:10BF9000636F0001D7DE012C05D00401605101015F
:10BFA000536B526F0001000C04014B510608D8A4DA
:10BFB0007AD00001A8992FEF3FF001C0D6F3EFEC43
:10BFC00039F00301D63D01D05CD0010139A511D073
:10BFD0000401606B60510001C8EC0DF00401602B9E
:10BFE000006E00509EA8FED7AD6E160E605DF2E1A9
:10BFF0000101040EEA6E4C0EE96EF2CF60F4F29E7F
:10C00000000E0001E3EC0DF00A000900F550EE6EA1
:10C010000009FBE1040160BFF28E040E0701E36F2B
:10C020004C0EE26F0001F0EC30F0A8890301D6510C
:10C03000300A000103E0010A08E00ED0010138B720
:10C0400003D038953887448E0001010138B503D0FC
:10C0500038973885448E06D0010138510C0B02E127
:10C060003885448E040E0401606FFA0E0801116FCA
:10C070000001D9EC26F00401602FF7D767D109D071
:10C080000301010138510C0B05E00001A8890401EE
:10C090005DD10101330E0401C06F010EC16F0001BB
:10C0A0006DEC40F00401040EEA6E4C0EE96E0801DE
:10C0B0000A6B0C6B140E0B6F000186EC28F0330E2C
:10C0C0000401C06FC16B00016DEC40F040EF46F021
:10C0D0000152D8A47DD00401C06BC16B000191EC6A
:10C0E00049F0070E0501A56FD00EA46F000103EC07
:10C0F00047F001523CE10401C06BC16B000191ECBF
:10C1000049F0070E0501A56FD00EA46F000103ECE6
:10C1100047F001522CE1040EEA6E4C0EE96EF2CFAC
:10C1200060F4F29E000EFBEC0DF00A000900F550E1
:10C13000EE6E0009FBE1040160BFF28E4B51300945
:10C140005C6F040E0701E36F4C0EE26F0001F0EC30
:10C1500030F0040E0401606FFA0E0801116F000147
:10C16000D9EC26F00401602FF7D7F0D000014BC4C2
:10C1700060F48EEF4FF00101485302E10401E6D074
:10C180000D0E0401C06FC16B000191EC49F04E0E21
:10C190000501A56F200EA46F000103EC47F001011B
:10C1A00038A306D04BC460F4000176DC10D0010146
:10C1B000310E0401C06FC16B000191EC49F04E0ECD
:10C1C0000501A56F200EA46F000103EC47F071D0AC
:10C1D0000101486BC00E4813040EEA6E4C0EE96E66
:10C1E000F2CF60F4F29E000E000113EC0EF00A0094
:10C1F0000900F550EE6E0009FBE1040160BFF28E0C
:10C200004B5130095C6F040E0701E36F4C0EE26F77
:10C210000001F0EC30F0010139A510D00401606B91
:10C22000605100012BEC0EF00401602B006E0050F9
:10C230009EA8FED7AD6E100E605DF2E10001EFEC3E
:10C2400039F00D0E0401C06FC16B00016DEC40F0C0
:10C250001F0E0501C96F400EC86F000164EC3FF06E
:10C26000EFEC39F01A0E0401BD6FBE6B00014AEC11
:10C270004FF0030E0501C96FE80EC86F000164ECB2
:10C280003FF0010138A306D04BC460F4000104DC88
:10C2900010D00101310E0401C06FC16B00016DECC3
:10C2A00040F0170E0501C96F700EC86F000164ECF5
:10C2B0003FF001014883110E0401BD6F010EBE6FF6
:10C2C00000014AEC4FF0010148871B0E0401BD6FCD
:10C2D000010EBE6F00014AEC4FF001014885150EBA
:10C2E0000401BD6F010EBE6F00014AEC4FF0010169
:10C2F0004891100E0401BD6F010EBE6F00014AECA3
:10C300004FF0036A01018551200F016E000E0322D8
:10C310000150380FE96E010E0320EA6E48C1EFFFAD
:10C32000000106DED89001018535036A350F016EE4
:10C33000000E03220150380FE96E010E0320EA6E51
:10C3400053C1ECFFED5252C1EFFF040100010CEFAD
:10C3500062F0010EEA6E580EE96E08010A6B0C6B72
:10C36000070E0B6F000186EC28F03EEC37F0010160
:10C3700039A510D004014B6B4B51000193EC0DF02B
:10C3800004014B2B006E00509EA8FED7AD6E200E10
:10C390004B5DF2E1010E04014A6F4A5106083FE38A
:10C3A000010139A526D004014B6B4B510001B3ECC0
:10C3B0000DF004014B2B006E00509EA8FED7AD6E11
:10C3C000050E4B5DF2E14AC4E9F71F0E0701EA6F63
:10C3D00000016EEC37F03A0E9EA8FED7AD6E200E2F
:10C3E0009EA8FED7AD6E200E9EA8FED7AD6E07D0DC
:10C3F0000101320E0801116F0001D9EC26F04AC488
:10C4000069F4F5EC3CF00A0E0801116F0001D9EC5B
:10C4100026F04AC44BF4C8D504014A2BBED700010C
:10C42000000C040EEA6E6B0EE96E08010A6B0C6BD1
:10C43000130E0B6F000186EC28F0040EEA6E7E0EE0
:10C44000E96E08010A6B0C6B130E0B6F000186EC92
:10C4500028F00D013D6B69C43CFD3F6B120E3E6F31
:10C460000001A2EC29F002C003F00150DC0F016EC4
:10C47000010E032201C091F403C092F4040E0801DE
:10C480000B6F6B0E0A6F03C00DF801C00CF8120E93
:10C490000E6F0001B1EC30F00C0E04016B6F036AFB
:10C4A00003013251330FE96E030E0320EA6EEF2CC5
:10C4B00003D03E0E04016C6F040E08010B6F6B0E6F
:10C4C0000A6F0001DDEC27F0050E0801116F000175
:10C4D000D9EC26F00D013D6B6AC43CFD3F6B120E9A
:10C4E0003E6F0001A2EC29F002C003F00150DC0F06
:10C4F000016E010E032201C091F403C092F4040EF8
:10C5000008010B6F7E0E0A6F03C00DF801C00CF816
:10C51000120E0E6F0001B1EC30F00A0E04017E6FB6
:10C52000036A03013251330FE96E030E0320EA6EF2
:10C53000EF50020803E13E0E04017F6F040E080174
:10C540000B6F7E0E0A6F0001DDEC27F0000C04017A
:10C550004A6B4A6B4A51020821E3036A4A51330F7E
:10C56000E96E030E0320EA6EEF6A036A4A51370F41
:10C57000016E030E032203C04CF4036A4A513F0FBD
:10C58000E96E030E0320EA6EEFCF4DF44CC4EAFFD0
:10C5900001C0E9FF4DC4EFFF4A2BDCD70301326B2A
:10C5A0000001A893A895A8970301D36BD3C3D5F333
:10C5B000D5C3D4F3036A3251370FE96E030E03205B
:10C5C000EA6EEFCF4BF4036A3251370FE96E030E78
:10C5D0000320EA6E010EEF2404014D6F4BC469F491
:10C5E0006A6F00011EDF000C036A6451680FE96E78
:10C5F000000E0320EA6EEFCFB8F40401010E000133
:10C6000064253F0B646F6451615D01E15B8E040141
:10C61000B8C401F00001000C036A6351680FE96EB1
:10C62000000E0320EA6EEFCF4BF40401010E00016F
:10C6300063253F0B636F6351615D01E15B8C040116
:10C640004BC401F00001000C04014A6B5BBE06D034
:10C650000001CADF01C04AF40401F8D70001666B8B
:10C660005BBC04D0D9DF01C04AF4FAD7000E9EBAF1
:10C67000010E000A06E09EAAFED7AECF4AF40001E2
:10C68000F5D7666B9D8A0A0E0701CE6F0001C4ECD8
:10C6900026F0C00EF21275EF65F00401476B486B8F
:10C6A000496BFA0E0701CE6F0001C4EC26F0FF0EB5
:10C6B0000401186F176F196F1C6B1B6F1A6F5B905B
:10C6C000589E456A446A476A466A4C6A5B925B9424
:10C6D0005B965C6A5D6A5E6A5F6A496B49510C08E9
:10C6E0000AE3036A4951CF0FE96E010E0320EA6E97
:10C6F000EF6A492BF3D7010EEA6E380EE96E080196
:10C700000A6B0C6B570E0B6F000186EC28F00401CE
:10C71000496B49510108D8A086D04951040DF35006
:10C720004B6B4A6FDB0E4A25E96E030E4B21EA6E16
:10C73000FF0EEC6EED52EF6E4951040DF3504B6B52
:10C740004A6F020E4A25016E000E4B21036E015006
:10C75000DB0FE96E030E0320EA6EEF6A4951040D08
:10C76000F3504B6B4A6FE70E4A25E96E030E4B21DF
:10C77000EA6EFF0EEC6EED52EF6E4951040DF35070
:10C780004B6B4A6F020E4A25016E000E4B21036E61
:10C790000150E70FE96E030E0320EA6EEF6A49517C
:10C7A000040DF3504B6B4A6FF30E4A25E96E030EEE
:10C7B0004B21EA6EFF0EEC6EED52EF6E4951040D07
:10C7C000F3504B6B4A6F020E4A25016E000E4B214F
:10C7D000036E0150F30FE96E030E0320EA6EEF6A59
:10C7E0004951040DF3504B6B4A6FFF0E4A25E96E19
:10C7F000030E4B21EA6EFF0EEC6EED52EF6E4951C7
:10C80000040DF3504B6B4A6F020E4A25016E000E69
:10C810004B21036E0150FF0FE96E030E0320EA6EF9
:10C82000EF6A492B76D70001666B0D0E676FEA6AD7
:10C83000680EE96E08010A6B0C6B400E0B6F00016D
:10C8400086EC28F0636B63C064F064C061F05B8EBB
:10C850005B8CEA6AA90EE96E08010A6B0C6B780E14
:10C860000B6F000186EC28F0656B65C062F0A88153
:10C87000040EEA6E330EE96EF2CF4AF4F29E000E19
:10C880009DEC21F00A000900F550EE6E0009FBE175
:10C8900004014ABFF28E040E0701E36F330EE26F0C
:10C8A0000001F0EC30F0FAEF35F0040E04014A6FAD
:10C8B000FA0E0701CE6F0001C4EC26F004014A2FE6
:10C8C000F7D794948B940C0EBD6EC150C00B0C091D
:10C8D000C16EC090C082C084C09EC280B098D1900A
:10C8E000840ED56E950ECD6EB150480BB509B16E64
:10C8F000000E766E000E776E9D80F28A070EB46E83
:10C9000097500D0E006E002EFED7B450A19CB56A54
:10C91000F19EFA0E0701CE6F0001C4EC26F0B5ECD3
:10C920002BF0F19CF288F19AF086F198F088F1965C
:10C93000F08AA38AC00EF212196AF2BE198EF29E14
:10C94000400E0D01436F446B000158EC22F019BEFC
:10C95000F28E02C088F101C087F188C1DCF387C183
:10C96000DBF388C1E0F387C1DFF3196AF2BE198EE9
:10C97000F29E400E0D01436F446B000158EC22F013
:10C9800019BEF28E02C048F401C047F4196AF2BE23
:10C99000198EF29E440E0D01436F446B000158EC5A
:10C9A00022F019BEF28E02C048F401C047F4196AA1
:10C9B000F2BE198EF29E420E0D01436F446B0001D0
:10C9C00058EC22F019BEF28E02C048F401C047F4C0
:10C9D000196AF2BE198EF29E460E0D01436F446B2A
:10C9E000000158EC22F019BEF28E02C048F401C0DA
:10C9F00047F4040EEA6E330EE96EF2CF4AF4F29E6B
:10CA0000000E13EC21F00A000900F550EE6E00094B
:10CA1000FBE104014ABFF28E040E0701E36F330EFF
:10CA2000E26F0001F0EC30F094DC01013AAB02D08F
:10CA30009D8A01D09D9A00018ADD050E0701CE6F07
:10CA40000001C4EC26F0010139A105D0FA0E040161
:10CA5000191704D00101FC0E04011917199F196A56
:10CA6000F2BE198EF29E480E0D014E6F010E4F6FF1
:10CA700019C450FD0001EBEC23F019BEF28E448A7C
:10CA80003BC189F1498A49840101856B866B036A40
:10CA90003B51200F016E000E03220150380FE96E4A
:10CAA000010E0320EA6EEF50F00B06E03BC18BF164
:10CAB0004A803CC18CF14A82010E04014A6F000198
:10CAC00027EC29F0012C03D00101B48302D001012D
:10CAD000B493050E0701CE6F0001C4EC26F00101EE
:10CAE0003ABB01D09D9A0001AFD5C4EFE8F0010137
:10CAF00086530CE00701D4517F0B06E1D2517F0B26
:10CB000003E1D3517F0B01E0468C01014839006EEF
:10CB10000F0E00160050FF0FF40F19E20C0F00016A
:10CB2000A9EF65F0D2C7D5F7D3C7D6F7D4C7D7F7E3
:10CB3000F9EC39F001010BD0D2C7D5F7D3C7D6F73E
:10CB4000D4C7D7F7E5EC3AF0010101D001010001AB
:10CB5000000CF2CF0EF0F29EE824F76AF7367D0F54
:10CB6000F66ECB0EF722000EF86EFB6E0A00F55043
:10CB7000FA6E0800F5500EBEF28EF96E24CB24CB6F
:10CB800024CB24CB24CB24CB24CB24CB24CB24CB2D
:10CB90004CCB38CB0401336B346B356B140E366FD2
:10CBA000180E376F070E386F396B050E3A6F060E89
:10CBB0003B6F120E3C6F01014839006E0F0E0016DC
:10CBC0000050020A000117E0070A1EE0010A24E0F3
:10CBD0000E0A2BE0020A29E0010A27E00E0A25E0EE
:10CBE0000B0A2CE0020A33E00F0A3AE0070A38E0A9
:10CBF000050A40E049D0120E0401376F0D0E366F62
:10CC0000070E386F396B42D0080E0401376F070EDC
:10CC1000366F386F396B3AD0100E0401376F0C0E37
:10CC2000366F070E386F396B31D0180E0401376F2D
:10CC3000140E366F070E386F396B28D0180E0401AA
:10CC4000376F080E366F070E386F396B1FD0140E12
:10CC50000401376F0C0E366F070E386F396B16D024
:10CC6000180E0401376F140E366F070E386F020E60
:10CC7000396F0CD0100E0401376F0A0E366F070E95
:10CC8000386F396B03D00001C8D10401375101015D
:10CC9000455D02E245C137F4040136510101465DAC
:10CCA00002E246C136F4196AF2BE198EF29E7F0E78
:10CCB0000D01436F37C444FD0001BFEC22F019BEE3
:10CCC000F28E01C03AF4196AF2BE198EF29E7F0EFE
:10CCD0000D01436F36C444FD0001BFEC22F019BEC4
:10CCE000F28E01C03BF4196AF2BE198EF29E7F0EDD
:10CCF0000D01436F38C444FD0001BFEC22F019BEA2
:10CD0000F28E01C03CF401014839006E0F0E00168E
:10CD100000500A08D8B4F2D0D8904731FF0A800FEB
:10CD200037533AE1365D38E2800ED880365504013B
:10CD30003D6FD8900101473104013D5D3F6F196A95
:10CD4000F2BE198EF29EE8CF43FD3AC444FD0001C5
:10CD5000BFEC22F019BEF28E01C034F4040134514C
:10CD6000375D03E237C434F404D0345302E1010EDA
:10CD7000346F3FC100F001018551016E04E0D8908D
:10CD80000032012EFCD700A003D00401349F02D052
:10CD90000401348F3ED00101D89047317F0F3753C3
:10CDA00003E1365D37E036E3800E365D04013D6F0A
:10CDB000D8900101473104013D5D3F6F196AF2BE11
:10CDC000198EF29EE8CF43FD3AC444FD0001BFEC4A
:10CDD00022F019BEF28E01C034F404013451375DE3
:10CDE00003E237C434F404D0345302E1010E346F4B
:10CDF0003FC100F001018551016E04E0D89000327E
:10CE0000012EFCD700A003D00401348F02D004010E
:10CE1000349F01017F0ED8804755355336E1345D8C
:10CE200034E2800ED8803455D880475504013F6FD6
:10CE3000196AF2BE198EF29EE8CF43FD3BC444FD51
:10CE40000001BFEC22F019BEF28E01C033F40401E0
:10CE50003351365D03E236C433F404D0335302E178
:10CE6000010E336F40C100F001018551016E04E0F5
:10CE7000D8900032012EFCD700A003D00401338FDC
:10CE800002D00401339F39D001017F0E472535536D
:10CE900003E1345D33E032E3800E345DD8804755E2
:10CEA00004013F6F196AF2BE198EF29EE8CF43FD6E
:10CEB0003BC444FD0001BFEC22F019BEF28E01C05C
:10CEC00033F404013351365D03E236C433F404D045
:10CED000335302E1010E336F40C100F0010185516F
:10CEE000016E04E0D8900032012EFCD700A003D0E0
:10CEF0000401339F02D00401338F0101D8904731E0
:10CF0000FF0A800F335333E1325D31E2800ED88067
:10CF1000325504013D6FD8900101473104013D5D58
:10CF20003F6F196AF2BE198EF29EE8CF43FD3CC4F2
:10CF300044FD0001BFEC22F019BEF28E01C035F4B1
:10CF400004013551385D03E238C435F405D035515C
:10CF5000395D02E339C435F4358701013AA503D0C0
:10CF60000401358F02D00401359F37D00101D890DC
:10CF700047317F0F335303E1325D30E02FE3800E02
:10CF8000325D04013D6FD8900101473104013D5DE0
:10CF90003F6F196AF2BE198EF29EE8CF43FD3CC482
:10CFA00044FD0001BFEC22F019BEF28E01C035F441
:10CFB00004013551385D03E238C435F405D03551EC
:10CFC000395D02E339C435F4358701013AA503D050
:10CFD0000401359F02D00401358F01012251040163
:10CFE000355D0DE1010123510401345D08E10101CA
:10CFF00024510401335D03E100010FD0040135C465
:10D0000022F134C423F133C424F134C4D2F733C43D
:10D01000D3F735C4D4F700016ADDCBEFE8F00401A3
:10D02000356B36913693196AF2BE198EF29E460E12
:10D030000D01436F446B000158EC22F019BEF28ED3
:10D0400002C034F401C033F4FF0E0401331B341B5F
:10D0500034C404F433C403F419A107D03351800855
:10D06000D8A4C4D03453D8A4C1D033C400F03451B0
:10D07000036E05E100520001D8B479D004010350D9
:10D0800006E1010E005C0001D8B474D00401200E4A
:10D09000035C05E100520001D8B475D004010350CF
:10D0A00006E1020E005C0001D8B476D00401020E45
:10D0B000035C05E100520001D8B46ED00401040EF7
:10D0C000035C05E100520001D8B466D00401080EEB
:10D0D000035C05E100520001D8B45ED00401400EAB
:10D0E000035C05E100520001D8B456D00401800E63
:10D0F000035C04E1005200014FE00401035005E12C
:10D10000400E005C000150E00401035005E1200ED8
:10D11000005C00014FE00401035005E1800E005C5B
:10D12000000150E00401035005E1040E005C000121
:10D1300049E00401035005E1080E005C000142E0F3
:10D140000401035005E1100E005C00013BE0040106
:10D15000010E035C04E10052000134E00401100EF2
:10D16000035C04E1005200012DE004012DD05B942A
:10D170005B963BD0040119B303D036815B8401D0A8
:10D180003683000132D0040119B303D036815B86A7
:10D1900001D03683000129D0040119B302D03681B1
:10D1A00001D03683000121D0606B5B980401368189
:10D1B00000011BD001018A6B8B6B8C6B04013681E3
:10D1C000000113D00401368158B406D045BA04D00A
:10D1D00058BE02D05BA007D05B90589E459A58A4D9
:10D1E00002D044805886000100D0040136A105D049
:10D1F00035C405F4058F5B9A04D000C404F4FFC362
:10D2000003F4000142EF9EF0040E04015B5F0AE3A9
:10D21000040EEA6E5B0EE96EEF5004E001D00000F0
:10D22000EF2EFDD70001000C080E04016D6F00C049
:10D230006EF4978E0A0E006E002EFED7978C85AC8A
:10D24000FED785BED88085AED89001360A0E006E16
:10D25000002EFED7979C8E9C6D2FEBD7978E0A0ED3
:10D26000006E002EFED78E9E6E51D8A4979E0000B1
:10D27000978C85ACFED70A0E006E002EFED78E9CD2
:10D28000979C0A0E006E002EFED78E9E979E000180
:10D2900087EF69F004016B6B978E0A0E006E002E0B
:10D2A000FED7978C0A0E006E002EFED78E9E979E9C
:10D2B0000A0E006E002EFED78E9C979C6951FE0BC5
:10D2C0006C6F6F6F0001B3EC29F06AC46FF4B3ECBC
:10D2D00029F0978E0A0E006E002EFED7978C0A0E4C
:10D2E000006E002EFED785ACFED78E9E979E0A0E4E
:10D2F000006E002EFED78E9C979C04016951010997
:10D300006C6F6F6F0001B3EC29F0006A8DD701C01C
:10D310006BF4979E0000978C85ACFED70A0E006ECA
:10D32000002EFED700D00000978E0A0E006E002E51
:10D33000FED71D0E006E002EFED700D004016BC478
:10D3400001F00001A9EF69F067C469F468C46AF4E8
:10D35000A1D70150000C0401506B516B400E526F6D
:10D36000536B546B556B566B576B586B599119AF88
:10D3700091D14F510008D8B08DD14F510608D8A097
:10D3800089D14E0E676F010E686F000195EC28F091
:10D3900001C054F4F60E04015417010E4F5D020F44
:10D3A000536F4E0E676F686B000195EC28F001C05B
:10D3B00055F404014F51010A00010CE0030A1EE07C
:10D3C000010A30E0070A42E0010A54E0030AD8B437
:10D3D00066D07BD055C400F004015351016E04E0C7
:10D3E000D8900032012EFCD700A003D0C00E506FA1
:10D3F00004D0C60E506FC00E526F6AD055C400F0F4
:10D4000004015351016E04E0D8900032012EFCD784
:10D4100000A003D0C10E506F04D0C70E506FC00ED5
:10D42000526F56D055C400F004015351016E04E010
:10D43000D8900032012EFCD700A003D0CE0E506F42
:10D4400004D0CA0E506FC00E526F42D055C400F0C7
:10D4500004015351016E04E0D8900032012EFCD734
:10D4600000A003D0CF0E506F04D0CB0E506FC00E73
:10D47000526F2ED055C400F004015351016E04E0E8
:10D48000D8900032012EFCD700A003D0D00E506FF0
:10D4900004D0D60E506FC00E526F548119D055C4AF
:10D4A00000F004015351016E04E0D8900032012EC7
:10D4B000FCD700A003D0D10E506F04D0D70E506F10
:10D4C000C00E526F548704D00001E4D0040100D094
:10D4D0009784599185B45981586B576B9784000E86
:10D4E00085B4010E5A6F000E59B1010E5A5D16E156
:10D4F000030E5A6F6E0E5B6F000186DE04015A2F19
:10D50000F9D7572BD8B4582B5851000806E2FF0A18
:10D5100003E157512B0801E201D0E0D797845991DC
:10D5200085B45981586B576B9784000E85B4010EF2
:10D530005A6F000E59B1010E5A5D16E1030E5A6F73
:10D540006E0E5B6F000160DE04015A2FF9D7572B76
:10D55000D8B4582B5851000806E2FF0A03E157518E
:10D560002B0801E201D0E0D7586B576B9784599193
:10D5700085B4598159B120D09784000E85B4010E2D
:10D580005A6F000E59B1010E5A5D16E1030E5A6F23
:10D590006E0E5B6F000138DE04015A2FF9D7572B4E
:10D5A000D8B4582B5851000806E2FF0A03E157513E
:10D5B0002B0801E201D0E0D78E849794420E676F6A
:10D5C000860E686F6A6B050E696F000124EC2AF005
:10D5D000420E0401676F020E686F6A6B50C469F4F3
:10D5E000000124EC2AF0630E0701CE6F0001C4ECA9
:10D5F00026F08E949794420E0401676F860E686F32
:10D600006A6B450E696F000124EC2AF04E0E04018E
:10D61000676F010E686F6A6B54C469F40001E6EC31
:10D620002AF0420E0401676F090E686F6A6B52C4DC
:10D6300069F4000124EC2AF0880E0401676F610E82
:10D64000686F000195EC28F001C056F40401569D66
:10D65000880E676F610E686F6A6B56C469F40001CB
:10D66000E6EC2AF0030E04015A6F6E0E5B6F0001A8
:10D67000CBDD04015A2FF9D7420E676F1E0E686F7B
:10D68000000162DE01C051F4040151AD02D04782B5
:10D6900001D047840001000C0401506B4F531DE181
:10D6A000880E676F610E686F000195EC28F001C06D
:10D6B00050F40401509D880E676F610E686F6A6BAD
:10D6C00050C469F40001E6EC2AF0110E0701CE6F98
:10D6D0000001C4EC26F052D004014E0E676F010E1B
:10D6E000686F000195EC28F001C050F4F60E0401BB
:10D6F00050174E0E676F010E686F6A6B50C469F465
:10D700000001E6EC2AF0110E0701CE6F0001C4EC17
:10D7100026F0880E0401676F3A0E686F000195ECE1
:10D7200028F001C050F404015051800B12E0509FCA
:10D73000880E676F3A0E686F6A6B50C469F4000117
:10D74000E6EC2AF0110E0701CE6F0001C4EC26F0C2
:10D750000401880E676F610E686F000195EC28F078
:10D7600001C050F40401508D880E676F610E686F20
:10D770006A6B50C469F40001E6EC2AF0000C040165
:10D78000686B010E686F685106081BE368C469F492
:10D790000001F5EC3CF00401672D09D00E0EBD6FC1
:10D7A000010EBE6F00014AEC4FF008D004010D0ECF
:10D7B000BD6F010EBE6F00014AEC4FF00401682BF3
:10D7C000E2D7000132EF6DF00401676B676B6751C0
:10D7D000020821E3036A6751330FE96E030E032049
:10D7E000EA6EEF6A036A6751370F016E030E032278
:10D7F00003C069F4036A67513F0FE96E030E03200B
:10D80000EA6EEFCF6AF469C4EAFF01C0E9FF6AC4B7
:10D81000EFFF672BDCD7686B000133EC2DF00301C1
:10D82000326B0001A893A895A8970301D36BD3C3CB
:10D83000D5F3D5C3D4F3036A3251370FE96E030E23
:10D840000320EA6EEFCF68F468C469F4120E040195
:10D850006A6F000111EC62F033EF6DF00401506B60
:10D86000516B526B4F2D21D019A11ED0040EEA6EC0
:10D87000530EE96EF2CF67F4F29E000E0001B5EC94
:10D8800021F00A000900F550EE6E0009FBE10401E9
:10D8900067BFF28E040E0701E36F530EE26F0001C3
:10D8A000F0EC30F0FF000401DFD04F53D8A4DCD0FF
:10D8B00019B1DAD00301326B040EEA6E530EE96E31
:10D8C000200E08010A6F0C6B140E0B6F000186EC22
:10D8D00028F0036A03013251330FE96E030E03206F
:10D8E000EA6E010EEF6E040EEA6E530EE96EF2CF91
:10D8F00067F4F29E000E0001CDEC21F00A00090051
:10D90000F550EE6E0009FBE1040167BFF28E040ED4
:10D9100008010B6F530E0A6F0001DDEC27F0040EB7
:10D92000EA6E530EE96EF2CF67F4F29E000EE4EC5D
:10D9300021F00A000900F550EE6E0009FBE1040138
:10D9400067BFF28E040E08010B6F530E0A6F0001C1
:10D95000DDEC27F04E0E0401676F010E686F0001C9
:10D9600095EC28F001C050F4F60E04015017F90EA2
:10D9700050174E0E676F010E686F6A6B50C469F4E2
:10D980000001E6EC2AF0880E0401676F610E686FF3
:10D99000000195EC28F00401526B01C051F4518D47
:10D9A000880E676F610E686F52C46AF451C469F4DF
:10D9B0000001E6EC2AF0880E0401676F610E686FC3
:10D9C0000001C2DC0401526B01C051F4518D880E7C
:10D9D000676F610E686F52C46AF451C469F4000144
:10D9E00024EC2AF0FF0E0401186F176F196F1B6FDC
:10D9F0001A6F196AF2BE198EF29E480E0D014E6F13
:10DA0000010E4F6F19C450FD0001EBEC23F019BE5D
:10DA1000F28E196AF2BE198EF29E4C0E0D01456F00
:10DA2000466B18C448FD17C447FD000114EC24F0F0
:10DA300019BEF28E196AF2BE198EF29E4A0E0D01BF
:10DA4000456F466B1BC448FD1AC447FD000114EC2A
:10DA500024F019BEF28EBE6A9D90010E0401676F1C
:10DA600000018DD6B1D604010001000C020E0301A5
:10DA7000375DF10FD8B0C8D00F0F000107EF6EF07F
:10DA80000301D3530BE1448C3FC337F3036A325194
:10DA9000330FE96E030E0320EA6EEF6AB5D003017F
:10DAA000D35101013B5D03E0D3C33BF1448E03013D
:10DAB000ABD00301D35101013C5D03E0D3C33CF182
:10DAC000448E0301A1D00301D3510101435D03E062
:10DAD000D3C343F1448E030197D00301D351010115
:10DAE0003E5D03E0D3C33EF1448E03018DD00301BC
:10DAF000D35305E101013A97448E06D00301D32D9B
:10DB000004D001013A87448E03017ED00301D35132
:10DB100001013D5D03E0D3C33DF1448E030174D0A8
:10DB20000301D35305E101013A93448E06D003016A
:10DB3000D32D04D001013A83448E030165D0030143
:10DB4000D3510101445D04E0D3C344F1448E07D0B6
:10DB50004451030DF3CF4FF404014FC4BEFF030142
:10DB600053D00301D35305E101013A95448E06D009
:10DB70000301D32D04D001013A85448E030144D022
:10DB80000301D32D05D001013A81448E06D0030153
:10DB9000D35304E101013A91448E030135D00301CE
:10DBA000D35306E101013A99448A448E07D0030118
:10DBB000D32D05D001013A89448A448E030124D033
:10DBC0000301D3510101455D03E0D3C345F1448E08
:10DBD00003011AD00301D3510101465D03E0D3C311
:10DBE00046F1448E030110D00301D35305E1010136
:10DBF0003A8F448E06D00301D32D04D001013A9F01
:10DC0000448E030101D003010301FEEF6FF0F2CF58
:10DC10000EF0F29EE824F76AF736390FF66EDC0E46
:10DC2000F722000EF86EFB6E0A00F550FA6E08003F
:10DC3000F5500EBEF28EF96E80DA9EDAB2DAC0DBF3
:10DC4000D4DBC6DADADAEEDA0CDB20DB62DB80DB8F
:10DC50009EDBE8DB3EDB0A0E04014F6F200E506FA7
:10DC6000516F526F430E536F6C0E546F650E556FAC
:10DC7000610E566F720E576F690E586F6E0E596FA8
:10DC8000670E5A6F200E5B6F5C6F5D6B5E6B5F6B38
:10DC9000010E0301385DF70FD8B080D0090F0001E5
:10DCA000D1EF6EF00301D35305E101013A8B458EAC
:10DCB00006D00301D32D04D001013A9B458E030108
:10DCC000448E6CD00301D35304E101013A8D05D099
:10DCD0000301D32D03D001013A9D0301448E5ED090
:10DCE0000301D35301E1458259D00301D3530BE122
:10DCF000040E08010B6F4F0E0A6F0001DDEC27F0D8
:10DD00006CEC32F003014AD00301D32D03D00101A2
:10DD1000398702D001013997448E03013FD00301B6
:10DD2000D32D04D00101398903D0030101013999B0
:10DD3000448E030133D00301D32D03D00101388376
:10DD400002D001013893448E030128D00301D32D62
:10DD500003D00101388902D001013899448E0301B2
:10DD60001DD00301D32D07D001013885389700015C
:10DD7000A88910D00301D351020807E101013895A9
:10DD800038870001A88906D003010101389538972A
:10DD90000001A899448E030101D003010301FEEFA5
:10DDA0006FF0F2CF0EF0F29EE824F76AF736CD0F4F
:10DDB000F66EDD0EF722000EF86EFB6E0A00F550CF
:10DDC000FA6E0800F5500EBEF28EF96EA4DCC4DCCB
:10DDD000E0DCEADC08DD1EDD36DD4CDD62DD040161
:10DDE0004F6B036A03013251370FE96E030E0320B4
:10DDF000EA6E010EEF5CF90FD8B077D0070F000183
:10DE000078EF6FF004014F2B000104014F2B00014C
:10DE100004014F2B000104014F2B000104014F2B83
:10DE2000000104014F2B00010301D3532EE13251B5
:10DE3000020815E104014F5304E101013F6B0ED0CC
:10DE40000401010E006E4F51016E04E0D8900036BF
:10DE5000012EFCD70050FF0A01013F1714D0040126
:10DE60004F5304E10101406B0ED00401010E006E1E
:10DE70004F51016E04E0D8900036012EFCD70050BF
:10DE8000FF0A010140172DD003013251020815E1AC
:10DE900004014F5305E1FF0E01013F6F0DD0040156
:10DEA000010E006E4F51016E04E0D8900036012E35
:10DEB000FCD7005001013F1314D004014F5305E17A
:10DEC000FF0E0101406F0DD00401010E006E4F5195
:10DED000016E04E0D8900036012EFCD700500101FD
:10DEE0004013448E030101D003010301FEEF6FF0E4
:10DEF000F2CF0EF0F29EE824F76AF7361B0FF66EAB
:10DF0000DF0EF722000EF86EFB6E0A00F550FA6E77
:10DF10000800F5500EBEF28EF96E28DE22DE1CDE01
:10DF200016DE10DE0ADE04DE036A03013251330F0F
:10DF3000E96E030E0320EA6EEF5002081EE1036A49
:10DF40003251370FE96E030E0320EA6E010EEF5CCB
:10DF50000401516F036A03013251370FE96E030E5A
:10DF60000320EA6EEFCF52F451C469F452C46AF44C
:10DF7000000111EC62F01BD00301036A3251370F2C
:10DF8000E96E030E0320EA6EEFCF50F4036A3251BC
:10DF9000370FE96E030E0320EA6E010EEF24040131
:10DFA000526F50C469F46A6F000111EC62F0000C0A
:10DFB000A893A895A8970301D36BD3C3D5F3D5C372
:10DFC000D4F3FF0ED36F32530BE13751100808E141
:10DFD00001014451030DF3CF50F4040150C4BEFFBE
:10DFE0000001A2DF000C03013251FC0F07E2040F15
:10DFF000000102EF70F03AD52ED6F1D60001D8DF3D
:10E00000C5EF76F0F2CF0EF0F29EE824F76AF7360D
:10E010002F0FF66EE00EF722000EF86EFB6E0A0070
:10E02000F550FA6E0800F5500EBEF28EF96EF6DF6E
:10E03000F8DFFADFFADFA8B33CD00301325324E162
:10E04000036A3251330FE96E030E0320EA6EEF6A62
:10E05000036A3251370F016E030E0322040103C01D
:10E0600050F4036A030132513F0FE96E030E03209F
:10E07000EA6EEFCF51F4040150C4EAFF01C0E9FF9A
:10E0800051C4EFFF13D00301036A3251330FE96E1D
:10E09000030E0320EA6E020EEF6E036A3251370F51
:10E0A000E96E030E0320EA6E010EEF6E00013CDF05
:10E0B00001D07EDF000C03013751110A00012CE072
:10E0C000130A46E00D0A5EE0060AD8B490D0020AB0
:10E0D000D8B4A9D0070AD8B4C2D0020AD8B4F4D0B0
:10E0E0000B0AD8B426D1030AD8B423D1050AD8B470
:10E0F00034D1070AD8B43BD1030AD8B442D10F0AAD
:10E10000D8B448D1020AD8B44FD11A0AD8B456D1DB
:10E110001D0AD8B45CD190D1010E0401686F0001D2
:10E1200033EC2DF0036A03013251370FE96E030E11
:10E130000320EA6E010EEF6E036A3251330FE96E6F
:10E14000030E0320EA6E020EEF6E000174DF78D139
:10E15000030EEA6E430EE96EF2CF4FF4F29E000E0C
:10E1600045EC0BF00A000900F550EE6E0009FBE1EA
:10E1700004014FBFF28E0301D46BD36BD3C3D5F32D
:10E1800000015ED1030EEA6E430EE96EF2CF4FF44A
:10E19000F29E000E5AEC0BF00A000900F550EE6EEC
:10E1A0000009FBE104014FBFF28E030EEA6E550E2B
:10E1B000E96EF2CF4FF4F29E000E00016FEC0BF00F
:10E1C0000A000900F550EE6E0009FBE104014FBFA3
:10E1D000F28E0301D36B01013ABF03D00301D32BAD
:10E1E0000101010E0301D46FD56B000129D1020E8C
:10E1F0000401686F000133EC2DF0036A0301325112
:10E20000370FE96E030E0320EA6E010EEF6E036A0C
:10E210003251330FE96E030E0320EA6E020EEF6EE9
:10E22000000109DF0DD1030E0401686F000133EC1A
:10E230002DF0036A03013251370FE96E030E0320FC
:10E24000EA6E010EEF6E036A3251330FE96E030E70
:10E250000320EA6E020EEF6E0001EDDEF1D0030E38
:10E26000EA6E430EE96EF2CF4FF4F29E000E84EC9C
:10E270000BF00A000900F550EE6E0009FBE1040105
:10E280004FBFF28E030EEA6E550EE96EF2CF4FF4D9
:10E29000F29E000E00019AEC0BF00A000900F55006
:10E2A000EE6E0009FBE104014FBFF28E0301D36B58
:10E2B00001013AA503D00301D32B0101010E030193
:10E2C000D46FD56B0001BCD0030EEA6E430EE96E2D
:10E2D000F2CF4FF4F29E000EB0EC0BF00A000900F2
:10E2E000F550EE6E0009FBE104014FBFF28E030E04
:10E2F000EA6E550EE96EF2CF4FF4F29E000E000169
:10E30000C6EC0BF00A000900F550EE6E0009FBE1C7
:10E3100004014FBFF28E010E0301D46FD36B0101D4
:10E320003AA903D00301D32B01010301D56B0001EE
:10E3300087D0A885180E0301D46F010ED56F375111
:10E34000050A000103E0030A04E006D045C1D3F347
:10E3500003D046C1D3F300D073D0A885060E0301C5
:10E36000D46F3BC1D3F3010ED56F000169D0A885EE
:10E370000C0E0301D46F3CC1D3F3010ED56F000125
:10E380005FD0A8853C0E0301D46F43C1D3F3D56B96
:10E39000000156D0A885180E0301D46F010ED56F69
:10E3A0003EC1D3F300014CD0A885140E0301D46FF5
:10E3B000010ED56F3DC1D3F3000142D0A885320EC6
:10E3C0000301D46FD56B44C1D3F3000139D0030EE0
:10E3D000EA6E430EE96EF2CF4FF4F29E000EDCECD3
:10E3E0000BF00A000900F550EE6E0009FBE1040194
:10E3F0004FBFF28E030EEA6E550EE96EF2CF4FF468
:10E40000F29E000E0001F3EC0BF00A000900F5503B
:10E41000EE6E0009FBE104014FBFF28E010E030115
:10E42000D46FD36B01013AA103D00301D32B0101B7
:10E430000301D56B000104D0A893A895A89700D03C
:10E44000D9EF76F003013851030A000119E0070AF9
:10E4500017E0010A2EE0030A60E0070AD8B491D061
:10E46000030AD8B48ED0050AD8B4DCD00F0AD8B4C9
:10E470000DD1010AD8B43ED1030AD8B48BD190D1C2
:10E48000030EEA6E430EE96EF2CF4FF4F29E000ED9
:10E4900045EC0BF00A000900F550EE6E0009FBE1B7
:10E4A00004014FBFF28E0301D46BD36BD3C3D5F3FA
:10E4B0007CD1030EEA6E430EE96EF2CF4FF4F29E6A
:10E4C000000E0AEC0CF00A000900F550EE6E00098F
:10E4D000FBE104014FBFF28E030EEA6E550EE96EAA
:10E4E000F2CF4FF4F29E000E00011FEC0CF00A0078
:10E4F0000900F550EE6E0009FBE104014FBFF28EFA
:10E50000010E0301D46FD56BD36B010139A703D082
:10E510000301D32B0101030148D1030EEA6E430E20
:10E52000E96EF2CF4FF4F29E000E34EC0CF00A00CC
:10E530000900F550EE6E0009FBE104014FBFF28EB9
:10E54000030EEA6E550EE96EF2CF4FF4F29E000E06
:10E5500000014BEC0CF00A000900F550EE6E0009CA
:10E56000FBE104014FBFF28E010E0301D46FD56BA6
:10E57000D36B010139A903D00301D32B010103019E
:10E5800014D1030EEA6E430EE96EF2CF4FF4F29E01
:10E59000000E5AEC0BF00A000900F550EE6E00096F
:10E5A000FBE104014FBFF28E030EEA6E550EE96ED9
:10E5B000F2CF4FF4F29E000E00016FEC0BF00A0058
:10E5C0000900F550EE6E0009FBE104014FBFF28E29
:10E5D000036A03013251370FE96E030E0320EA6E1E
:10E5E000EF50010A000103E0030A0AE012D0030120
:10E5F000D36B01013ABB03D00301D32B01010DD032
:10E600000301D36B01013ABD03D00301D32B0101F8
:10E6100004D00301D36B010100D0010E0301D46FBC
:10E62000D56BC3D0030EEA6E430EE96EF2CF4FF402
:10E63000F29E000E62EC0CF00A000900F550EE6E3E
:10E640000009FBE104014FBFF28E030EEA6E550E86
:10E65000E96EF2CF4FF4F29E000E00017AEC0CF05E
:10E660000A000900F550EE6E0009FBE104014FBFFE
:10E67000F28E010E0301D46FD56BD36B010138A369
:10E6800003D00301D32B010103018FD0030EEA6EE7
:10E69000430EE96EF2CF4FF4F29E000E92EC0CF0B6
:10E6A0000A000900F550EE6E0009FBE104014FBFBE
:10E6B000F28E030EEA6E550EE96EF2CF4FF4F29E23
:10E6C000000E0001AAEC0CF00A000900F550EE6EF5
:10E6D0000009FBE104014FBFF28E010E0301D46F6C
:10E6E000D56BD36B010138A903D00301D32B0101F2
:10E6F00003015BD0030EEA6E430EE96EF2CF4FF4D6
:10E70000F29E000EC2EC0CF00A000900F550EE6E0D
:10E710000009FBE104014FBFF28E030EEA6E550EB5
:10E72000E96EF2CF4FF4F29E000E0001DAEC0CF02D
:10E730000A000900F550EE6E0009FBE104014FBF2D
:10E74000F28E030EEA6E670EE96EF2CF4FF4F29E80
:10E75000000E0001F2EC0CF00A000900F550EE6E1C
:10E760000009FBE104014FBFF28E020E0301D46FDA
:10E77000D56B010138A505D0010E0301D36F09D077
:10E78000010138A704D0020E0301D36F02D00301A8
:10E79000D36B0BD00401686B000133EC2DF008DC67
:10E7A000A893A895A897030100D00001D9EF76F0AF
:10E7B00004014F6B030EEA6E430EE96EF2CF50F484
:10E7C000F29E000E000184EC0BF00A000900F550E7
:10E7D000EE6E0009FBE1040150BFF28E030EEA6EFB
:10E7E000550EE96EF2CF50F4F29E000E00019AEC45
:10E7F0000BF00A000900F550EE6E0009FBE1040180
:10E8000050BFF28E010E0301D46FD56B036A3251F3
:10E81000370FE96E030E0320EA6EEF50070A00017E
:10E820000FE0010A10E0030A11E0010A12E0070AF2
:10E8300013E0010A14E0030A15E0090A3EE044D09F
:10E8400004014F2B000104014F2B000104014F2B49
:10E85000000104014F2B000104014F2B00010401B2
:10E860004F2B000104014F5301E14F2B03013251A3
:10E8700002080FE13FC100F004014F51016E04E0B6
:10E88000D8900032012EFCD70301D36B00B0D32BFC
:10E8900011D0325103080EE140C100F004014F5184
:10E8A000016E04E0D8900032012EFCD70301D36B37
:10E8B00000B0D32B0001A8830BD00401686B0001CA
:10E8C00033EC2DF0D8EC6FF0A893A895A89700D062
:10E8D000D9EF76F004017951F00B006E003A0F0E7B
:10E8E0000016005000010FE0010A41E0030AD8B40D
:10E8F0008DD0010AD8B4BFD0070AD8B407D1010A15
:10E90000D8B435D165D1040179510F0B090815E34D
:10E91000010E7A5D036A7B25E96E7C510320EA6E65
:10E92000300EEF6E036A7A517B25E96E7C5103202D
:10E93000EA6E79513009EF6E19D079510F0B0F083B
:10E9400015E3010E7A5D036A7B25E96E7C51032095
:10E95000EA6E310EEF6E036A7A517B25E96E7C51C7
:10E960000320EA6E0A0E795D3009EF6E46D104018C
:10E9700079510F0B030816E3010E7A5D036A7B25BC
:10E98000E96E7C510320EA6E310EEF6E036A7A5114
:10E990007B25E96E7C510320EA6E0A0E795D300911
:10E9A000EF6E33D079510F0B0D0816E3010E7A5D2F
:10E9B000036A7B25E96E7C510320EA6E320EEF6E0E
:10E9C000036A7A517B25E96E7C510320EA6E140EAE
:10E9D000795D3009EF6E19D079510F0B0F0815E3EF
:10E9E000010E7A5D036A7B25E96E7C510320EA6E95
:10E9F000330EEF6E036A7A517B25E96E7C5103205A
:10EA0000EA6E1E0E795D3009EF6EF7D00401795180
:10EA10000F0B070816E3010E7A5D036A7B25E96E8A
:10EA20007C510320EA6E330EEF6E036A7A517B2528
:10EA3000E96E7C510320EA6E1E0E795D3009EF6E9F
:10EA400019D079510F0B0F0815E3010E7A5D036A97
:10EA50007B25E96E7C510320EA6E340EEF6E036A6B
:10EA60007A517B25E96E7C510320EA6E280E795D90
:10EA70003009EF6EC2D0040179510F0B010816E383
:10EA8000010E7A5D036A7B25E96E7C510320EA6EF4
:10EA9000340EEF6E036A7A517B25E96E7C510320B8
:10EAA000EA6E280E795D3009EF6E2FD079510F0B89
:10EAB0000B0816E3010E7A5D036A7B25E96E7C5133
:10EAC0000320EA6E350EEF6E036A7A517B25E96EFC
:10EAD0007C510320EA6E320E795D3009EF6E15D05D
:10EAE000010E7A5D036A7B25E96E7C510320EA6E94
:10EAF000360EEF6E036A7A517B25E96E7C51032056
:10EB0000EA6E3C0E795D3009EF6E77D004017951E1
:10EB10000F0B050816E3010E7A5D036A7B25E96E8B
:10EB20007C510320EA6E360EEF6E036A7A517B2524
:10EB3000E96E7C510320EA6E3C0E795D3009EF6E80
:10EB400015D0010E7A5D036A7B25E96E7C510320A6
:10EB5000EA6E370EEF6E036A7A517B25E96E7C51BF
:10EB60000320EA6E460E795D3009EF6E46D004014F
:10EB700079510F0B090816E3010E7A5D036A7B25B4
:10EB8000E96E7C510320EA6E380EEF6E036A7A510B
:10EB90007B25E96E7C510320EA6E500E795D3009C9
:10EBA000EF6E15D0010E7A5D036A7B25E96E7C510C
:10EBB0000320EA6E390EEF6E036A7A517B25E96E07
:10EBC0007C510320EA6E5A0E795D3009EF6E15D044
:10EBD000010E04017A5D036A7B25E96E7C510320F6
:10EBE000EA6E450EEF6E036A7A517B25E96E7C5121
:10EBF0000320EA6E450EEF6E00D00001000C040EFB
:10EC0000EA6E530EE96E08010A6B0C6B130E0B6F64
:10EC1000000186EC28F0040EEA6E660EE96E08012B
:10EC20000A6B0C6B130E0B6F000186EC28F0036A65
:10EC300003013251370FE96E030E0320EA6E0D0116
:10EC40003D6BEFCF3CFD3F6B120E3E6F0001A2EC1F
:10EC500029F002C003F00150DC0F016E010E032207
:10EC600001C07AF403C07BF4040E08010B6F530E4D
:10EC70000A6F03C00DF801C00CF8120E0E6F0001F0
:10EC8000B1EC30F00C0E0401536F040E08010B6F51
:10EC9000530E0A6F0001DDEC27F0050E0801116F1D
:10ECA0000001D9EC26F0A8B51CD004015251120D78
:10ECB000F350036A430F016E030E032201C079F47F
:10ECC00003C07AF4040E08010B6F660E0A6F03C0CE
:10ECD0000DF801C00CF8120E0E6F0001B1EC30F00F
:10ECE00042D0A8B71CD0040EEA6E660EE96E200E64
:10ECF00008010A6F0C6B090E0B6F000186EC28F0FF
:10ED000052C479F4090E04017A6F040E7C6F660E0A
:10ED10007B6F0001DFDD0401706B25D00001040E64
:10ED2000EA6E660EE96E200E08010A6F0C6B090E82
:10ED30000B6F000186EC28F052C479F4090E04012F
:10ED40007A6F040E7C6F660E7B6F0001C3DD730E5D
:10ED50000401716F650E726F630E736F746B6FC415
:10ED600070F42E0E6F6F0A0E0401666F3E0E676F11
:10ED7000040E08010B6F660E0A6F0001DDEC27F030
:10ED8000000CA8A303D0F3EF6FF018D0A883030101
:10ED90003251000107E0010A07E0030A07E0010A17
:10EDA00005E005D05BEF70F022EF72F001D5A8937B
:10EDB00000D0A8A303D0D3C352F421DF6CEF84F0BA
:10EDC0000301D551D35D03E1010ED425D36FD307E1
:10EDD00032530AE13751100807E1D351030DF3CF45
:10EDE00052F4040152C4BEFFD3C352F4000107DF42
:10EDF00009EF77F0040EEA6E4F0EE96E08010A6B18
:10EE00000C6B030E0B6F000186EC28F0A8A302D058
:10EE1000D7D7FFD0036A03013251330FE96E030ED7
:10EE20000320EA6EEF50000105E0010A31E0030A19
:10EE30004EE0EFD0036A03013251370FE96E030E43
:10EE40000320EA6E020EEF6E036A3251330FE96E51
:10EE5000030E0320EA6E010EEF6E036A3251370F84
:10EE6000E96E030E0320EA6EEFCF52F4036A3251CB
:10EE7000370FE96E030E0320EA6E010EEF24040142
:10EE8000546F52C469F46A6F000111EC62F0C1D092
:10EE9000036A03013251370FE96E030E0320EA6E55
:10EEA000EF2A036A3251330FE96E030E0320EA6E34
:10EEB000020EEF6E030E04014F6F506B040E08013B
:10EEC0000B6F4F0E0A6F0001DDEC27F0A2D0036A32
:10EED00003013251370FE96E030E0320EA6EEF2A69
:10EEE000036A3251370FE96E030E0320EA6EEFCF4B
:10EEF00052F4036A32513B0FE96E030E0320EA6EAF
:10EF0000EF500401525D67E066E30301325324E1F0
:10EF1000036A3251330FE96E030E0320EA6EEF6A83
:10EF2000036A3251370F016E030E0322040103C03E
:10EF300053F4036A030132513F0FE96E030E0320BD
:10EF4000EA6EEFCF54F4040153C4EAFF01C0E9FFB5
:10EF500054C4EFFF23D00301036A3251330FE96E2B
:10EF6000030E0320EA6E020EEF6E036A3251370F72
:10EF7000016E030E0322040103C053F4036A03016C
:10EF800032513F0FE96E030E0320EA6E010EEF24AB
:10EF9000040153C4EAFF01C0E9FFEF6E036A0301F5
:10EFA00032513F0FE96E030E0320EA6EEFCF52F4A9
:10EFB000036A32513F0FE96E030E0320EA6E010E21
:10EFC000EF240401546F52C469F46A6F000111EC1C
:10EFD00062F01ED00401036A03013251370FE96E5B
:10EFE000030E0320EA6E010EEF5C0401536F036A07
:10EFF00003013251370FE96E030E0320EA6EEFCFA3
:10F0000054F453C469F454C46AF4000111EC62F07E
:10F0100000D071EF84F00301D451D35D03E1010E00
:10F02000D55DD36FD32B32530AE13751100807E176
:10F03000D351030DF3CF52F4040152C4BEFFD3C326
:10F0400052F40001DCDD34EF78F0040EEA6E4F0E6E
:10F05000E96E08010A6B0C6B030E0B6F000186EC66
:10F0600028F0A8A302D0D7D772D1036A0301325186
:10F07000330FE96E030E0320EA6EEF500208D8A4A6
:10F0800096D0036A3251370FE96E030E0320EA6E01
:10F09000EF52D8B48CD0036A3251370FE96E030EA9
:10F0A0000320EA6EEF0632534BE0036A3251370F0A
:10F0B000E96E030E0320EA6EEF5242E1036A325119
:10F0C000330FE96E030E0320EA6E020EEF6E036A41
:10F0D00032513B0FE96E030E0320EA6E010EEF5C26
:10F0E0000401536F036A030132513B0FE96E030EB3
:10F0F0000320EA6EEFCF54F453C469F454C46AF4A5
:10F10000000111EC62F0036A03013251370F016E06
:10F11000030E0322040103C053F4036A03013251B6
:10F120003B0FE96E030E0320EA6EEFCF54F40401A7
:10F1300053C4EAFF01C0E9FF54C4EFFF36D0030116
:10F14000036A3251370FE96E030E0320EA6EEF5265
:10F1500016E1036A3251370FE96E030E0320EA6E9F
:10F16000EF2A036A3251330FE96E030E0320EA6E71
:10F17000EF6A010E04014F6F506B0ED00301036A5A
:10F180003251330FE96E030E0320EA6E010EEF6E6B
:10F19000020E04014F6F506B040E08010B6F4F0EEF
:10F1A0000A6F0001DDEC27F00401D1D00301036AEE
:10F1B0003251370FE96E030E0320EA6EEFCF52F49F
:10F1C000036A32513F0FE96E030E0320EA6EEF50DF
:10F1D0000401525DD8B47AD0D8A078D0036A030174
:10F1E0003251370FE96E030E0320EA6EEF06036A11
:10F1F0003251370FE96E030E0320EA6EEF5001081B
:10F2000049E3036A3251370FE96E030E0320EA6EB9
:10F21000EF06325311E1036A3251330FE96E030EE8
:10F220000320EA6EEF6A036A3251370FE96E030E6C
:10F230000320EA6EEF6A12D0036A3251370FE96E8B
:10F24000030E0320EA6E010EEF6E036A3251330F94
:10F25000E96E030E0320EA6E020EEF6E036A32516E
:10F260003F0FE96E030E0320EA6EEFCF52F4036AFC
:10F2700032513F0FE96E030E0320EA6E010EEF24B8
:10F280000401546F52C469F46A6F000111EC62F01A
:10F290001BD00301036A3251370FE96E030E0320BE
:10F2A000EA6EEFCF52F4036A3251370FE96E030E64
:10F2B0000320EA6E010EEF240401546F52C469F476
:10F2C0006A6F000111EC62F042D00401036A03018D
:10F2D0003251330FE96E030E0320EA6E020EEF6E19
:10F2E000036A32513B0FE96E030E0320EA6E010EF2
:10F2F000EF5C0401536F036A030132513B0FE96E67
:10F30000030E0320EA6EEFCF54F453C469F454C4DF
:10F310006AF4000111EC62F0036A03013251370F05
:10F32000016E030E0322040103C053F4036A0301B8
:10F3300032513B0FE96E030E0320EA6EEFCF54F417
:10F34000040153C4EAFF01C0E9FF54C4EFFF040104
:10F3500078EF89F00401356B3691196AF2BE198E87
:10F36000F29E400E0D01436F446B000158EC22F0F9
:10F3700019BEF28E02C034F401C033F4010187518A
:10F380000401331B010188510401341B34C4E0F330
:10F3900033C4DFF358B40CD019B102D019B308D07C
:10F3A0000301E16BDCC3E0F3DBC3DFF3CDD0040189
:10F3B00033C400F03451036E05E100520001D8B4AB
:10F3C0007AD00401035006E1010E005C0001D8B4BC
:10F3D0008ED00401035006E1020E005C0001D8B497
:10F3E00086D00401035006E1040E005C0001D8B48D
:10F3F0007ED00401035006E1080E005C0001D8B481
:10F4000076D00401035006E1100E005C0001D8B470
:10F410006ED00401035006E1200E005C0001D8B458
:10F4200066D00401035006E1400E005C0001D8B430
:10F430005ED00401035006E1800E005C0001D8B4E8
:10F4400056D00401010E035C04E1005200014FE0BC
:10F450000401020E035C04E10052000148E00401D3
:10F46000040E035C04E10052000141E00401080EB7
:10F47000035C04E1005200013AE00401100E035C59
:10F4800004E10052000133E00401200E035C04E1BA
:10F49000005200012CE00401400E035C04E1005224
:10F4A000000125E00401800E035C04E1005200012C
:10F4B0001EE0040137D00101435318E0040119B3E1
:10F4C00002D0010113D043C160F05B88376B375124
:10F4D00000019FEC1DF00401372B006E00509EA828
:10F4E000FED7AD6E190E375DF2E101011DD05B98BC
:10F4F0000401368134C412F8570E0801136F00015D
:10F500001BEC37F033C412F8570E0801136F0001DB
:10F510001BEC37F00D0E9EA8FED7AD6E0A0E9EA80E
:10F52000FED7AD6E010100D0040136A107D035C46D
:10F53000E1F30301E18F5B9A07D00401DCC3E0F340
:10F54000DBC3DFF30301E16B000160EF9EF0040118
:10F55000356B020E366F376B386B010139A554D00D
:10F56000040133C4E9FF34C4EAFFECCF3AF4ED52AE
:10F57000EFCF39F433C4E9FF34C4EAFFECCF3CF4F5
:10F58000ED52EFCF3BF43B51FF0A3D6F3C51FF0A78
:10F590003E6F3F6B3F510001AFEC17F004013F2B72
:10F5A000006E00509EA8FED7AD6E0C0E3F5DF2E1DE
:10F5B0003AC412F8370E0801136F00011BEC37F044
:10F5C00039C412F8370E0801136F00011BEC37F035
:10F5D000200E9EA8FED7AD6E3EC412F8370E08016D
:10F5E000136F00011BEC37F03DC412F8370E080111
:10F5F000136F00011BEC37F00A0E9EA8FED7AD6E0C
:10F600000D0E9EA8FED7AD6E040133C4E9FF34C4CD
:10F61000EAFFECCF03F0ED52EFCF37F403C038F43C
:10F6200037C400F03851036E06E1010E005C0001A2
:10F63000D8B477D00401035006E1020E005C00014B
:10F64000D8B472D00401035006E1040E005C00013E
:10F65000D8B46DD00401035006E1080E005C00012F
:10F66000D8B468D00401035006E1100E005C00011C
:10F67000D8B463D00401035006E1200E005C000101
:10F68000D8B45ED00401010E035C05E10052000114
:10F69000D8B46DD00401020E035C05E100520001F4
:10F6A000D8B468D00401040E035C05E100520001E7
:10F6B000D8B463D00401080E035C04E100520001D9
:10F6C0005FE00401100E035C04E1005200015BE006
:10F6D0000401200E035C04E10052000157E0040124
:10F6E000035006E1800E005C0001D8B481D0040113
:10F6F000035006E1400E005C0001D8B47CD0040148
:10F70000400E035C05E100520001D8B477D004013B
:10F71000800E035C05E100520001D8B472D00401F0
:10F7200088D00401352B00010401352B00010401B0
:10F73000352B00010401352B00010401352B00019C
:10F740000401352B01018B2D08D004013551010135
:10F750008C5D03E18A2D01D008D0010E8B6F4A80A9
:10F7600035C48CF14A828A6F498C040162D004014D
:10F77000352B00010401352B00010401352B00015C
:10F780000401352B00010401352B00010401352B48
:10F7900001013AB114D08B51020808E1040135513E
:10F7A00001018C5D03E18A51020808E0020E8B6FB3
:10F7B0004A8035C48CF14A828A6F498C17D08B2DD0
:10F7C00009D0060E0401352501018C5D03E18A2D67
:10F7D00001D00CD0010E8B6F4A80060E0401352536
:10F7E00001018C6F4A82010E8A6F498C040121D07D
:10F7F0000401362B00010401362B00010401362BD5
:10F8000000010401362B365101018B5D07E18C2D7F
:10F8100005D00401365101018A5D09E036C48BF13F
:10F820004A80010E8C6F4A8236C48AF1498C0401E9
:10F8300000D000016DEF9EF004013A6B392D1AD013
:10F840003A6B3751F00B006E036A035005E1800EEE
:10F85000005C000109E00401035005E1400E005C7A
:10F86000000105E0040105D004013A2B0001040168
:10F870003A2B2DD0020E3A6F37C400F03851036E88
:10F8800005E1800E005C000117E00401035005E172
:10F89000400E005C000113E00401800E035C04E1F3
:10F8A000005200010FE00401400E035C04E100522D
:10F8B00000010BE004010BD004013A2B000104010C
:10F8C0003A2B000104013A2B000104013A2B3AC4FF
:10F8D00001F00001000C0401356B36913693196A72
:10F8E000F2BE198EF29E440E0D01436F446B00016F
:10F8F00058EC22F019BEF28E02C034F401C033F489
:10F90000FF0E0401331B341B34C4ECF333C4EBF39C
:10F9100019A105D0E8C3ECF3E7C3EBF3E9D033C496
:10F9200000F03451036E05E100520001D8B47FD0DD
:10F930000401800E035C05E100520001D8B487D0B9
:10F940000401400E035C05E100520001D8B47FD0F1
:10F950000401035006E1400E005C0001D8B477D0EA
:10F960000401035006E1800E005C0001D8B46FD0A2
:10F970000401035006E1010E005C0001D8B4A1D0DF
:10F980000401035006E1020E005C0001D8B499D0D6
:10F990000401035006E1040E005C0001D8B491D0CC
:10F9A0000401035006E1080E005C0001D8B489D0C0
:10F9B0000401035006E1100E005C0001D8B481D0B0
:10F9C0000401035006E1200E005C0001D8B479D098
:10F9D0000401010E035C05E100520001D8B471D0AE
:10F9E0000401020E035C05E100520001D8B469D0A5
:10F9F0000401040E035C05E100520001D8B461D09B
:10FA00000401080E035C04E1005200015AE0040105
:10FA1000100E035C04E10052000153E00401200ECB
:10FA2000035C04E1005200014CE004014CD00401ED
:10FA300019B309D058B406D058AE04D05E500308AC
:10FA400001E2458A01D036835B90589E44D0040180
:10FA500019B335D0368158BE28D05BB026D058B403
:10FA600024D034C438F433C437F4396B0001E4DEF5
:10FA7000036A0150200F016E000E03220150380F5F
:10FA8000E96E010E0320EA6EEF38006E0F0E0016CD
:10FA9000005009E0588E5E6A030E0401356FF28A49
:10FAA000D76AD66A000108D004015B90589E459A37
:10FAB00058A402D0448058860401358B01D0368387
:10FAC0000AD0040136815B90589E459A58A402D012
:10FAD0004480588600D036A107D035C4EDF3030129
:10FAE000ED8F5B9A06D00401E8C3ECF3E7C3EBF3B8
:10FAF000030100017FEF9EF004014F6B506B400E3D
:10FB0000516F526B536B546B556B566B576B5891CF
:10FB10004E510008D8B092D14E510608D8A08ED1CF
:10FB20004E0E676F010E686F000195EC28F001C062
:10FB300053F4F90E04015317010E4E5D020F526F7C
:10FB40004E0E676F686B000195EC28F001C054F40D
:10FB500004014E51010A00010CE0030A1EE0010AF3
:10FB600030E0070A42E0010A54E0030AD8B466D044
:10FB70007BD054C400F004015251016E04E0D890CF
:10FB80000032012EFCD700A003D0C00E4F6F04D06E
:10FB9000C60E4F6FC00E516F6AD054C400F00401FE
:10FBA0005251016E04E0D8900032012EFCD700A023
:10FBB00003D0C10E4F6F04D0C70E4F6FC00E516FF0
:10FBC00056D054C400F004015251016E04E0D890A4
:10FBD0000032012EFCD700A003D0CE0E4F6F04D010
:10FBE000CA0E4F6FC00E516F42D054C400F00401D2
:10FBF0005251016E04E0D8900032012EFCD700A0D3
:10FC000003D0CF0E4F6F04D0CB0E4F6FC00E516F8D
:10FC10002ED054C400F004015251016E04E0D8907B
:10FC20000032012EFCD700A003D0D00E4F6F04D0BD
:10FC3000D60E4F6FC00E516F538319D054C400F0CD
:10FC400004015251016E04E0D8900032012EFCD71D
:10FC500000A003D0D10E4F6F04D0D70E4F6FC00E4F
:10FC6000516F538504D00001E9D0040100D097887A
:10FC7000589185B85881576B566B9788000E85B898
:10FC8000010E596F000E58B1010E595D17E1030EB8
:10FC9000596F6E0E5B6F000104EC69F00401592F7F
:10FCA000F8D7562BD8B4572B5751000806E2FF0A55
:10FCB00003E156512B0801E201D0DFD79788589114
:10FCC00085B85881576B566B9788000E85B8010E22
:10FCD000596F000E58B1010E595D17E1030E596FAF
:10FCE0006E0E5B6F000104EC69F00401592FF8D728
:10FCF000562BD8B4572B5751000806E2FF0A03E1F0
:10FD000056512B0801E201D0DFD7576B566B97880D
:10FD1000589185B8588158B121D09788000E85B880
:10FD2000010E596F000E58B1010E595D17E1030E17
:10FD3000596F6E0E5B6F000104EC69F00401592FDE
:10FD4000F8D7562BD8B4572B5751000806E2FF0AB4
:10FD500003E156512B0801E201D0DFD78E8A979A32
:10FD6000400E676F860E686F6A6B050E696F000143
:10FD700024EC2AF0400E0401676F020E686F6A6B74
:10FD80004FC469F4000124EC2AF0630E0701CE6F22
:10FD90000001C4EC26F08E9A979A400E0401676F1A
:10FDA000860E686F6A6B450E696F000124EC2AF0BD
:10FDB0004E0E0401676F010E686F6A6B53C469F4DD
:10FDC0000001E6EC2AF0400E0401676F090E686F2F
:10FDD0006A6B51C469F4000124EC2AF0880E040116
:10FDE000676F610E686F0001A4EC69F001C055F403
:10FDF0000401559D880E676F610E686F6A6B55C46C
:10FE000069F4000124EC2AF0030E0401596F6E0E10
:10FE10005B6F000104EC69F00401592FF8D7400E24
:10FE2000676F1E0E686F0001A4EC69F001C050F40A
:10FE3000040150AD02D0478A01D047880001DFEFAE
:10FE40008AF004014F6B506B4E51010A000107E02C
:10FE5000030A0BE0010A0FE0070A13E018D07F0E37
:10FE60000401506FFF0E4F6F17D0BF0E0401506F8B
:10FE7000FF0E4F6F11D0FF0E0401506FBF0E4F6F7A
:10FE80000BD0FF0E0401506F7F0E4F6F05D0FF0E99
:10FE90000401506F4F6F00D0196AF2BE198EF29EA6
:10FEA000400E0D01456F466B50C448FD4FC447FDE1
:10FEB000000114EC24F019BEF28E7FEF8CF0780E66
:10FEC00004011913010148A503D004011997010188
:10FED00048A103D004011999010148A303D00401EA
:10FEE000199B010148A703D00401199D0101196A5A
:10FEF000F2BE198EF29E480E0D014E6F010E4F6F2D
:10FF000019C450FD0001EBEC23F019BEF28E000C79
:10FF100004014F6B4E0E676F010E686F000195EC88
:10FF200028F001C04FF404014D5302E14F9901D074
:10FF30004F894E0E676F010E686F6A6B4FC469F48C
:10FF40000001E6EC2AF004014E2D03D08E8097903C
:10FF500002D08E9097900001000C0401346B356B39
:10FF6000010E335D016E010E006E015204E0D89067
:10FF70000036012EFCD700C035F4346B34C401F0D8
:10FF800035C402F0000120EFA0F00401346B356BA2
:10FF9000010E335D006E010E346F356B005205E0CB
:10FFA000D89034373537002EFBD734C401F035C430
:10FFB00002F000013EEFA0F058A40AD0588658A4E1
:10FFC00007D0010E0701CE6F0001C4EC26F0F7D771
:02FFD000000C23
:020000040001F9
:100000000401496B4A6B4B6B4C6B4D6B4E91040E6C
:10001000EA6E350EE96E08010A6B0C6B140E0B6F5D
:10002000000186EC28F0010139A571EF80F0040190
:1000300033C4E9FF34C4EAFFECCF50F4ED52EFCF04
:100040004FF433C4E9FF34C4EAFFECCF52F4ED526D
:10005000EFCF51F45151FF0A536F5251FF0A546FC1
:10006000556B55510001A6EC1AF00401552B006E9A
:1000700000509EA839EF80F0AD6E0C0E555DD8A4EF
:1000800031EF80F050C412F8370E0801136F0001F1
:100090001BEC37F04FC412F8370E0801136F000144
:1000A0001BEC37F0200E9EA853EF80F0AD6E54C4C9
:1000B00012F8370E0801136F00011BEC37F053C420
:1000C00012F8370E0801136F00011BEC37F00A0E0F
:1000D0009EA868EF80F0AD6E0D0E9EA86DEF80F0CB
:1000E000AD6E040133C4E9FF34C4EAFFECCF03F082
:1000F000ED52EFCF49F403C04AF433C4E9FF34C4EE
:10010000EAFFEFCF00F0E92AEF50E906036E035053
:10011000D8A492EF80F0020E005C0001D8B439EF51
:1001200081F004010350D8A49DEF80F0040E005C20
:100130000001D8B4DEEF81F004010350D8A4A8EF89
:1001400080F0200E005C0001D8B4BFEF82F0040103
:100150000350D8A4B3EF80F0400E005C0001D8B487
:1001600046EF83F004010350D8A4BEEF80F0800E68
:10017000005C0001D8B4CDEF83F00401010E035CF4
:10018000D8A4C9EF80F000520001D8B46AEF84F01F
:1001900004010350D8A4D4EF80F0080E005C0001E5
:1001A000D8B46FEF84F004010350D8A4DFEF80F0DF
:1001B000100E005C0001D8B474EF84F00401100E3E
:1001C000035CD8A4EAEF80F000520001D8B476EFC7
:1001D00084F00401020E035CD8A4F5EF80F0005215
:1001E0000001D8B47BEF84F00401040E035CD8A4B2
:1001F00000EF81F000520001D8B442EF85F0040115
:10020000080E035CD8A40BEF81F000520001D8B4B3
:1002100008EF86F004010350D8A416EF81F0010E18
:10022000005C0001D8B4ADEF86F00401200E035C41
:10023000D8A421EF81F000520001D8B470EF87F00C
:100240000401400E035CD8A42CEF81F000520001A1
:10025000D8B435EF88F00401800E035CD8A437EFE2
:1002600081F000520001D8B4D3EF88F0040178EF98
:1002700089F001014851F00BD8B4DBEF81F058B0A0
:1002800045EF81F058A453EF81F0588AA09258AC02
:1002900053EF81F0010E0701CE6F0001C4EC26F090
:1002A000010147EF81F0040119B98AEF81F0198942
:1002B000040EEA6E350EE96EF2CF4FF4F29E000E98
:1002C0000001C0EC1AF00A000900F550EE6E0009BA
:1002D000D8A464EF81F004014FBFF28E0101489170
:1002E00039A787EF81F004014F6B4F510001D8EC23
:1002F0001AF004014F2B006E00509EA87DEF81F094
:10030000AD6E0A0E4F5DD8A475EF81F00101BAEF12
:1003100081F004011999040EEA6E350EE96EF2CFF0
:100320004FF4F29E000E0001EDEC1AF00A000900F5
:10033000F550EE6E0009D8A497EF81F004014FBF8D
:10034000F28E0101488139A7BAEF81F004014F6BA9
:100350004F51000105EC1BF004014F2B006E0050C3
:100360009EA8B0EF81F0AD6E090E4F5DD8A4A8EF46
:1003700081F00101196AF2BE198EF29E480E0D013C
:100380004E6F010E4F6F19C450FD0001EBEC23F0CE
:1003900019BEF28E040E0701E36F350EE26F000105
:1003A000F0EC30F0468058B0D9EF81F058A4DBEF84
:1003B00081F0589AA082040178EF89F0040119BFF6
:1003C0006CEF82F001018453D8B462EF82F0040133
:1003D000198F196AF2BE198EF29E480E0D014E6FEA
:1003E000010E4F6F19C450FD0001EBEC23F019BE54
:1003F000F28E040EEA6E350EE96EF2CF4FF4F29EE5
:10040000000E19EC1BF00A000900F550EE6E000911
:10041000D8A404EF82F004014FBFF28E040E07014E
:10042000E36F350EE26F0001F0EC30F0A8A928EF81
:1004300082F0010184510608D8B403D0000128EFEE
:1004400082F0D7C34FF40001ABEC69F02CEF82F0DF
:1004500084C14FF4ABEC69F004014F6B00014CEC2C
:100460006BF0010139A760EF82F004014F6B4F512F
:10047000000159EC18F004014F2B006E00509EA8AB
:100480003FEF82F0AD6E070E4F5DD8A437EF82F0DC
:1004900084C1E9F71F0E0701EA6F00016EEC37F027
:1004A0000A0E9EA851EF82F0AD6E0D0E9EA856EF7B
:1004B00082F0AD6E3E0E9EA85BEF82F0AD6E010144
:1004C00069EF82F0010E04014F6F00014CEC6BF0FC
:1004D0000101BCEF82F00401199F196AF2BE198E66
:1004E000F29E480E0D014E6F010E4F6F19C450FD64
:1004F0000001EBEC23F019BEF28E040EEA6E350E0D
:10050000E96EF2CF4FF4F29E000E31EC1BF00A00C0
:100510000900F550EE6E0009D8A488EF82F00401BE
:100520004FBFF28E040E0701E36F350EE26F00013C
:10053000F0EC30F084C14FF4ABEC69F0010E040133
:100540004F6F00014CEC6BF0010139A7BCEF82F05A
:1005500004014F6B4F51000149EC1BF004014F2B7C
:10056000006E00509EA8B2EF82F0AD6E0B0E4F5D94
:10057000D8A4AAEF82F00101040178EF89F0040108
:1005800019B5F8EF82F0060E19131993040EEA6EEE
:10059000350EE96EF2CF4FF4F29E000E00015EECD4
:1005A0001BF00A000900F550EE6E0009D8A4D2EF46
:1005B00082F004014FBFF28E0101399139A7F5EFA6
:1005C00082F004014F6B4F51000176EC1BF00401E7
:1005D0004F2B006E00509EA8EBEF82F0AD6E110E17
:1005E0004F5DD8A4E3EF82F001012AEF83F004010C
:1005F000060E19131995040EEA6E350EE96EF2CF48
:100600004FF4F29E000E00018EEC1BF00A00090070
:10061000F550EE6E0009D8A407EF83F004014FBF38
:10062000F28E0101398139A72AEF83F004014F6B63
:100630004F510001A6EC1BF004014F2B006E00503F
:100640009EA820EF83F0AD6E0F0E4F5DD8A418EF7B
:1006500083F00101196AF2BE198EF29E480E0D0157
:100660004E6F010E4F6F19C450FD0001EBEC23F0EB
:1006700019BEF28E040E0701E36F350EE26F000122
:10068000F0EC30F0448E040178EF89F0040119B3E6
:100690007FEF83F0060E19131995040EEA6E350EDE
:1006A000E96EF2CF4FF4F29E000E00018EEC1BF0CB
:1006B0000A000900F550EE6E0009D8A459EF83F046
:1006C00004014FBFF28E0101398139A77CEF83F01D
:1006D00004014F6B4F510001A6EC1BF004014F2B9E
:1006E000006E00509EA872EF83F0AD6E0F0E4F5D4E
:1006F000D8A46AEF83F00101B1EF83F00401060E84
:1007000019131993040EEA6E350EE96EF2CF4FF409
:10071000F29E000E00015EEC1BF00A000900F5508D
:10072000EE6E0009D8A48EEF83F004014FBFF28E65
:100730000101399139A7B1EF83F004014F6B4F519B
:10074000000176EC1BF004014F2B006E00509EA8B8
:10075000A7EF83F0AD6E110E4F5DD8A49FEF83F02D
:100760000101196AF2BE198EF29E480E0D014E6FFC
:10077000010E4F6F19C450FD0001EBEC23F019BEC0
:10078000F28E040E0701E36F350EE26F0001F0EC0C
:1007900030F0448E040178EF89F0040119B148EF7C
:1007A00084F0020E3325E96E000E3421EA6EEFCF9D
:1007B0004FF4000E4FBD010E000AD8A425EF84F0BF
:1007C000196AF2BE198EF29E460E0D01436F446BFC
:1007D000000158EC22F019BEF28E02C04CF401C0A8
:1007E0004BF4010E04014D6F4D516308D8A025EF65
:1007F00084F04B51FF0A4F6F4C51FF0A506F4F511D
:100800008008D8A408EF84F05053D8B40AEF84F0DD
:1008100078EF89F00A0E0701CE6F0001C4EC26F0D4
:10082000196AF2BE198EF29E460E0D01436F446B9B
:10083000000158EC22F019BEF28E02C04CF401C047
:100840004BF404014D2BF4EF83F0010139A73CEF89
:1008500084F004014F6B4F510001BDEC1BF004010B
:100860004F2B006E00509EA833EF84F0AD6E0C0E3F
:100870004F5DD8A42BEF84F004014F6B00012EECE8
:100880006CF08E909790040178EF89F068EF84F017
:10089000010139A75FEF84F004014F6B4F51000154
:1008A000D3EC1BF004014F2B006E00509EA856EFB6
:1008B00084F0AD6E0B0E4F5DD8A44EEF84F0010EA8
:1008C00004014F6F00012EEC6CF0040178EF89F009
:1008D00078EF89F0C1EF76F0040178EF89F0FAEF54
:1008E00076F0040178EF89F025EF78F01BEC70F0DA
:1008F000040178EF89F001014851F00BD8B43FEFC3
:1009000085F058B087EF84F058A495EF84F0588AAA
:10091000A09258AC95EF84F0010E0701CE6F000154
:10092000C4EC26F0010189EF84F0040119B7B3EF9C
:1009300084F0140EBD6F010EBE6F00014AEC4FF043
:1009400001014895036A8551200F016E000E0322B4
:100950000150380F016E010E032201C0E9FF03C0F0
:10096000EAFFEF9404011987196AF2BE198EF29E0C
:10097000480E0D014E6F010E4F6F19C450FD00015E
:10098000EBEC23F019BEF28E040EEA6E350EE96E22
:10099000F2CF4FF4F29E000EE8EC1BF00A000900C3
:1009A000F550EE6E0009D8A4CFEF84F004014FBFDC
:1009B000F28E040E0701E36F350EE26F0001F0ECDA
:1009C00030F0010139A7F8EF84F004014F6B4F516B
:1009D000000100EC1CF004014F2B006E00509EA89B
:1009E000EFEF84F0AD6E0C0E4F5DD8A4E7EF84F00E
:1009F00004014E91000198EC5FF0160E0401BD6FEA
:100A0000010EBE6F00014AEC4FF004014EB137EF0A
:100A100085F0196AF2BE198EF29E460E0D01436FE3
:100A2000446B000158EC22F019BEF28E02C04CF467
:100A300001C04BF404014B51FF0A4F6F4C51FF0AA8
:100A4000506F4F53D8A42AEF85F050510208D8B404
:100A50002DEF85F04E8135EF85F0160EBD6F010E3E
:100A6000BE6F00014AEC4FF0040106EF85F058B06C
:100A70003DEF85F058A43FEF85F0589AA08204011D
:100A800078EF89F001014851F00BD8B405EF86F0FA
:100A900058B04EEF85F058A45CEF85F0588AA092CC
:100AA00058AC5CEF85F0010E0701CE6F0001C4EC7D
:100AB00026F0010150EF85F0040119B77AEF85F0B7
:100AC000140EBD6F010EBE6F00014AEC4FF0010124
:100AD0004895036A8551200F016E000E03220150D4
:100AE000380F016E010E032201C0E9FF03C0EAFFC7
:100AF000EF9404011987196AF2BE198EF29E480E0E
:100B00000D014E6F010E4F6F19C450FD0001EBEC4B
:100B100023F019BEF28E040EEA6E350EE96EF2CFA6
:100B20004FF4F29E000E16EC1CF00A000900F5507E
:100B3000EE6E0009D8A496EF85F004014FBFF28E47
:100B4000040E0701E36F350EE26F0001F0EC30F0A8
:100B5000010139A7BFEF85F004014F6B4F51000130
:100B60002EEC1CF004014F2B006E00509EA8B6EF37
:100B700085F0AD6E0E0E4F5DD8A4AEEF85F000018E
:100B800098EC5FF0170E0401BD6F010EBE6F0001FF
:100B90004AEC4FF004014E914EB1FDEF85F0196A19
:100BA000F2BE198EF29E460E0D01436F446B00019A
:100BB00058EC22F019BEF28E02C04CF401C04BF486
:100BC00004014B51FF0A4F6F4C51FF0A506F4F53B6
:100BD000D8A4F0EF85F050510408D8B4F3EF85F0B5
:100BE0004E81FBEF85F0170EBD6F010EBE6F000149
:100BF0004AEC4FF00401CCEF85F058B003EF86F0DB
:100C000058A405EF86F0589AA082040178EF89F085
:100C100001014851F00BD8B4AAEF86F058B014EF98
:100C200086F058A422EF86F0588AA09258AC22EFA2
:100C300086F0010E0701CE6F0001C4EC26F0010121
:100C400016EF86F0040119A759EF86F01997040EE4
:100C5000EA6E350EE96EF2CF4FF4F29E000E0001FF
:100C600045EC1CF00A000900F550EE6E0009D8A40E
:100C700033EF86F004014FBFF28E0101488539A79A
:100C800056EF86F004014F6B4F5100015DEC1CF0F4
:100C900004014F2B006E00509EA84CEF86F0AD6E05
:100CA0000E0E4F5DD8A444EF86F0010189EF86F067
:100CB00004011987040EEA6E350EE96EF2CF4FF487
:100CC000F29E000E000174EC1CF00A000900F550C1
:100CD000EE6E0009D8A466EF86F004014FBFF28ED5
:100CE0000101489539A789EF86F004014F6B4F51F8
:100CF00000018CEC1CF004014F2B006E00509EA8EC
:100D00007FEF86F0AD6E100E4F5DD8A477EF86F0C2
:100D10000101040E0701E36F350EE26F0001F0ECF4
:100D200030F0196AF2BE198EF29E480E0D014E6F18
:100D3000010E4F6F19C450FD0001EBEC23F019BEFA
:100D4000F28E468058B0A8EF86F058A4AAEF86F03D
:100D5000589AA082040178EF89F001014851F00B04
:100D6000D8B46DEF87F058B0B9EF86F058A4C7EF4C
:100D700086F0588AA09258ACC7EF86F0010E0701A2
:100D8000CE6F0001C4EC26F00101BBEF86F0040138
:100D900019BDE5EF86F01C0EBD6F010EBE6F0001A0
:100DA0004AEC4FF001014897036A8551200F016E0C
:100DB000000E03220150380F016E010E032201C004
:100DC000E9FF03C0EAFFEF960401198D196AF2BE2C
:100DD000198EF29E480E0D014E6F010E4F6F19C411
:100DE00050FD0001EBEC23F019BEF28E040EEA6E0A
:100DF000350EE96EF2CF4FF4F29E000EA4EC1CF01B
:100E00000A000900F550EE6E0009D8A401EF87F042
:100E100004014FBFF28E040E0701E36F350EE26F3F
:100E20000001F0EC30F0010139A72AEF87F004014E
:100E30004F6B4F510001BCEC1CF004014F2B006EB6
:100E400000509EA821EF87F0AD6E0D0E4F5DD8A427
:100E500019EF87F01E0E0401BD6F010EBE6F000179
:100E60004AEC4FF004014E914EB15EEF87F0420E16
:100E7000006E002EFED70000196AF2BE198EF29E97
:100E8000460E0D01436F446B000158EC22F019BE71
:100E9000F28E02C04CF401C04BF404014B51FF0A26
:100EA0004F6F4C51FF0A506F4F2D5BEF87F050533F
:100EB000D8B45CEF87F04E8134EF87F01F0EBD6F22
:100EC000010EBE6F00014AEC4FF058B06BEF87F097
:100ED00058A46DEF87F0589AA082040178EF89F04A
:100EE00001014851F00BD8B432EF88F058B07CEFD4
:100EF00087F058A48AEF87F0588AA09258AC8AEFFE
:100F000087F0010E0701CE6F0001C4EC26F001014D
:100F10007EEF87F0040119BDA8EF87F01C0EBD6FAE
:100F2000010EBE6F00014AEC4FF001014897036AC1
:100F30008551200F016E000E03220150380F016E03
:100F4000010E032201C0E9FF03C0EAFFEF9604018E
:100F5000198D196AF2BE198EF29E480E0D014E6F60
:100F6000010E4F6F19C450FD0001EBEC23F019BEC8
:100F7000F28E040EEA6E350EE96EF2CF4FF4F29E59
:100F8000000ED2EC1CF00A000900F550EE6E0009CC
:100F9000D8A4C4EF87F004014FBFF28E040E0701FE
:100FA000E36F350EE26F0001F0EC30F0010139A77C
:100FB000EDEF87F004014F6B4F510001EAEC1CF09C
:100FC00004014F2B006E00509EA8E4EF87F0AD6E39
:100FD0000C0E4F5DD8A4DCEF87F01D0E0401BD6F31
:100FE000010EBE6F00014AEC4FF004014E914EB16C
:100FF00023EF88F0420E006E002EFED70000196A23
:10100000F2BE198EF29E460E0D01436F446B000135
:1010100058EC22F019BEF28E02C04CF401C04BF421
:1010200004014B51FF0A4F6F4C51FF0A506F4F5351
:10103000D8A420EF88F050512008D8B421EF88F0D0
:101040004E81F7EF87F01F0EBD6F010EBE6F0001DE
:101050004AEC4FF058B030EF88F058A432EF88F0E7
:10106000589AA082040178EF89F001014851F00BF1
:10107000D8B4D0EF88F058B041EF88F058A44FEFC3
:1010800088F0588AA09258AC4FEF88F0010E070103
:10109000CE6F0001C4EC26F0010143EF88F004019B
:1010A00019AD6FEF88F0199D040EEA6E350EE96EEA
:1010B000F2CF4FF4F29E000E000100EC1DF00A008A
:1010C0000900F550EE6E0009D8A460EF88F0040125
:1010D0004FBFF28E0101488797EF88F00401198D08
:1010E000196AF2BE198EF29E480E0D014E6F010E66
:1010F0004F6F19C450FD0001EBEC23F019BEF28EC6
:10110000040EEA6E350EE96EF2CF4FF4F29E000E39
:1011100018EC1DF00A000900F550EE6E0009D8A485
:101120008BEF88F004014FBFF28E01014897196AD6
:10113000F2BE198EF29E480E0D014E6F010E4F6FDA
:1011400019C450FD0001EBEC23F019BEF28E040E21
:101150000701E36F350EE26F0001F0EC30F04680DE
:10116000010139A7C8EF88F004014F6B4F5100010E
:1011700030EC1DF004014F2B006E00509EA8BEEF16
:1011800088F0AD6E0D0E4F5DD8A4B6EF88F001016A
:1011900058B0CEEF88F058A4D0EF88F0589AA082CB
:1011A000040178EF89F001014851F00BD8B475EFD4
:1011B00089F058B0DFEF88F058A4EDEF88F0588A36
:1011C000A09258ACEDEF88F0010E0701CE6F000140
:1011D000C4EC26F00101E1EF88F0040119BB24EF13
:1011E00089F0198B040EEA6E350EE96EF2CF4FF4DA
:1011F000F29E000E000146EC1DF00A000900F550B9
:10120000EE6E0009D8A4FEEF88F004014FBFF28E05
:101210000101489339A721EF89F004014F6B4F5129
:1012200000015EEC1DF004014F2B006E00509EA8E3
:1012300017EF89F0AD6E0A0E4F5DD8A40FEF89F05D
:10124000010154EF89F00401199B040EEA6E350E7A
:10125000E96EF2CF4FF4F29E000E000173EC1DF028
:101260000A000900F550EE6E0009D8A431EF89F0AC
:1012700004014FBFF28E0101488339A754EF89F072
:1012800004014F6B4F5100018BEC1DF004014F2BFB
:10129000006E00509EA84AEF89F0AD6E090E4F5DBA
:1012A000D8A442EF89F00101040E0701E36F350E67
:1012B000E26F0001F0EC30F0196AF2BE198EF29E76
:1012C000480E0D014E6F010E4F6F19C450FD000105
:1012D000EBEC23F019BEF28E468058B073EF89F024
:1012E00058A475EF89F0589AA082040178EF89F02C
:1012F0000001000C0401356B366B020E376F4C6B2E
:101300004D6B040EEA6E380EE96E08010A6B0C6B29
:10131000140E0B6F000186EC28F0010139A5EBEFEC
:1013200089F0040133C4E9FF34C4EAFFECCF4FF481
:10133000ED52EFCF4EF433C4E9FF34C4EAFFECCFF3
:1013400051F4ED52EFCF50F45051FF0A526F51510A
:10135000FF0A536F546B54510001C9EC17F004019C
:10136000542B006E00509EA8B3EF89F0AD6E0C0EAA
:10137000545DD8A4ABEF89F04FC412F8370E0801C2
:10138000136F00011BEC37F04EC412F8370E080142
:10139000136F00011BEC37F0200E9EA8CDEF89F0F3
:1013A000AD6E53C412F8370E0801136F00011BEC29
:1013B00037F052C412F8370E0801136F00011BEC0E
:1013C00037F00A0E9EA8E2EF89F0AD6E0D0E9EA8D2
:1013D000E7EF89F0AD6E040133C4E9FF34C4EAFFDE
:1013E000ECCF03F0ED52EFCF35F403C036F435C443
:1013F00000F036C403F0200E365DD8A406EF8AF064
:1014000000520001D8B4ADEF8AF00401100E035C65
:10141000D8A411EF8AF000520001D8B4B0EF8AF0DE
:101420000401080E035CD8A41CEF8AF000520001EE
:10143000D8B4B3EF8AF00401040E035CD8A427EFFC
:101440008AF000520001D8B4B6EF8AF00401020E0F
:10145000035CD8A432EF8AF000520001D8B4B9EF8F
:101460008AF00401010E035CD8A43DEF8AF000521B
:101470000001D8B4BCEF8AF004010350D8A448EFAF
:101480008AF0200E005C0001D8B478EF8BF00401E4
:101490000350D8A453EF8AF0100E005C0001D8B4BA
:1014A0007BEF8BF004010350D8A45EEF8AF0080EA6
:1014B000005C0001D8B47EEF8BF004010350D8A487
:1014C00069EF8AF0040E005C0001D8B481EF8BF064
:1014D00004010350D8A474EF8AF0020E005C0001EE
:1014E000D8B484EF8BF004010350D8A47FEF8AF0C6
:1014F000010E005C0001D8B487EF8BF004010350AB
:10150000D8A48AEF8AF0800E005C0001D8B482EF84
:101510008CF004010350D8A495EF8AF0400E005CD3
:101520000001D8B485EF8CF00401800E035CD8A4D0
:10153000A0EF8AF000520001D8B488EF8CF00401CB
:10154000400E035CD8A4ABEF8AF000520001D8B47F
:101550008BEF8CF004016CEF8DF004014C2B00013B
:1015600004014C2B000104014C2B000104014C2B05
:10157000000104014C2B000104014C2B3F0E1B13F6
:101580003551FF0A006E3651FF0A036E00501A17DC
:1015900003501B17196AF2BE198EF29E4A0E0D01F6
:1015A000456F466B1BC448FD1AC447FD000114EC8F
:1015B00024F019BEF28E4CC44EF47CEF7DF04CC486
:1015C00083F1A8A905EF8BF004014C510608D8B4AB
:1015D00003D0000105EF8BF0040EEA6E380EE96EC1
:1015E000F2CF4EF4F29E000E0001E3EC17F00A0079
:1015F0000900F550EE6E0009D8A4F8EF8AF0040156
:101600004EBFF28E1DEF8BF00001040EEA6E380E15
:10161000E96EF2CF4EF4F29E000EFBEC17F00A00DA
:101620000900F550EE6E0009D8A410EF8BF004010C
:101630004EBFF28E4C513009456F5BBA28EF8BF0EC
:10164000040E0701E36F380EE26F0001F0EC30F09A
:10165000010139A757EF8BF004014E6B4E51000189
:1016600012EC18F004014E2B006E00509EA836EFCD
:101670008BF0AD6E0A0E4E5DD8A42EEF8BF04CC4ED
:10168000E9F71F0E0701EA6F00016EEC37F00A0E52
:101690009EA848EF8BF0AD6E0D0E9EA84DEF8BF01F
:1016A000AD6E3E0E9EA852EF8BF0AD6E01013AAFCB
:1016B00075EF8BF0036A04014C51200F016E000E90
:1016C00003220150380FE96E010E0320EA6EEF503D
:1016D000F00BD8B476EF8BF04C510101855DD8B496
:1016E00075EF8BF04CC48BF14A8004016CEF8DF0E8
:1016F00004014D2B000104014D2B000104014D2B71
:10170000000104014D2B000104014D2B00010401D7
:101710004D2B3F0E1A133551FF0A006E3651FF0A4A
:10172000036E00501A1703501B17196AF2BE198E68
:10173000F29E4A0E0D01456F466B1BC448FD1AC44C
:1017400047FD000114EC24F019BEF28E0401198F3C
:10175000196AF2BE198EF29E480E0D014E6F010EEF
:101760004F6F19C450FD0001EBEC23F019BEF28E4F
:10177000A8A9F3EF8BF004014D510608D8B4D7EFB8
:101780008BF0010184510608D8B403D00401D7EFCF
:101790008BF04DC44FF40001ABEC69F0010E040175
:1017A000696F0001DDEC3DF0F3EF8BF004014D516A
:1017B0000608D8A4EEEF8BF0010184510608D8A4E6
:1017C00003D00401EEEF8BF084C1D7F30401696B01
:1017D0000001DDEC3DF0F3EF8BF004014DC44FF45C
:1017E0000001ABEC69F0A8B9FAEF8BF04DC44FF4EF
:1017F000ABEC69F04DC484F104014F6B00014CEC7B
:101800006BF0A8A925EF8CF0010184510608D8B42B
:1018100003D0000125EF8CF0040EEA6E380EE96E5D
:10182000F2CF4EF4F29E000E000129EC18F00A00EF
:101830000900F550EE6E0009D8A418EF8CF00401F1
:101840004EBFF28E3DEF8CF00001040EEA6E380EB2
:10185000E96EF2CF4EF4F29E000E41EC18F00A0051
:101860000900F550EE6E0009D8A430EF8CF00401A9
:101870004EBFF28E4D513009446F5BBA48EF8CF089
:10188000040E0701E36F380EE26F0001F0EC30F058
:10189000010139A777EF8CF004014E6B4E51000126
:1018A00059EC18F004014E2B006E00509EA856EF24
:1018B0008CF0AD6E070E4E5DD8A44EEF8CF04DC48B
:1018C000E9F71F0E0701EA6F00016EEC37F00A0E10
:1018D0009EA868EF8CF0AD6E0D0E9EA86DEF8CF09B
:1018E000AD6E3E0E9EA872EF8CF0AD6E01013AA96E
:1018F0007FEF8CF04DC44EF4000121EF7FF0040126
:101900006CEF8DF00401372B00010401372B00012F
:101910000401372B00010401372B036A3751200FD4
:10192000016E000E03220150380FE96E010E0320F4
:10193000EA6EEF50F00BD8A4ADEF8CF0020E332519
:10194000E96E000E3421EA6EEFCF50F4000E50BB6A
:10195000010E000AD8A448EF8DF0C00E1A131B1315
:101960003551FF0A006E3651FF0A036E00501A17F8
:1019700003501B17196AF2BE198EF29E4A0E0D0112
:10198000456F466B1BC448FD1AC447FD000114ECAB
:1019900024F019BEF28ECF0E04011713FF0E181398
:1019A000196AF2BE198EF29E4C0E0D01456F466B00
:1019B00018C448FD17C447FD000114EC24F019BEFB
:1019C000F28E37C4E2F7CFEC53F037C469F4F5EC8C
:1019D0003CF0050E0701CE6F0001C4EC26F05FEC71
:1019E0007FF0040EEA6E380EE96EF2CF4EF4F29EEE
:1019F000000E6FEC18F00A000900F550EE6E0009B9
:101A0000D8A4FCEF8CF004014EBFF28E37513009A0
:101A1000456F5BBA15EF8DF0040E0701E36F380ECA
:101A2000E26F0001F0EC30F004014680010139A7BB
:101A300045EF8DF004014E6B4E51000187EC18F01C
:101A400004014E2B006E00509EA824EF8DF0AD6E69
:101A5000070E4E5DD8A41CEF8DF037C4E9F71F0EBA
:101A60000701EA6F00016EEC37F00A0E9EA836EF10
:101A70008DF0AD6E0D0E9EA83BEF8DF0AD6E3E0E5F
:101A80009EA840EF8DF0AD6E010169EF8DF004016D
:101A9000040EEA6E380EE96EF2CF4EF4F29E000E9E
:101AA00000019DEC18F00A000900F550EE6E0009E7
:101AB000D8A454EF8DF004014EBFF28E3751300997
:101AC000416F040E0701E36F380EE26F0001F0EC86
:101AD00030F004016CEF8DF00001000C0401336B59
:101AE000346B356B36913693196AF2BE198EF29EBD
:101AF000420E0D01436F446B000158EC22F019BEF9
:101B0000F28E02C034F401C033F4FF0E0401331B23
:101B1000341B34C4F8F333C4F7F319A196EF8DF0F6
:101B2000F4C3F8F3F3C3F7F3D6EF8EF033C400F049
:101B30003451036ED8A4A3EF8DF000520001D8B445
:101B400055EF8EF004010350D8A4AEEF8DF0400E97
:101B5000005C0001D8B469EF8EF004010350D8A4F2
:101B6000B9EF8DF0800E005C0001D8B469EF8EF003
:101B700004010350D8A4C4EF8DF0010E005C0001F5
:101B8000D8B4AFEF8EF004010350D8A4CFEF8DF09E
:101B9000020E005C0001D8B4AFEF8EF004010350D8
:101BA000D8A4DAEF8DF0040E005C0001D8B4AFEFDA
:101BB0008EF004010350D8A4E5EF8DF0080E005C10
:101BC0000001D8B4AFEF8EF00401010E035CD8A47D
:101BD000F0EF8DF000520001D8B4AFEF8EF00401A9
:101BE000020E035CD8A4FBEF8DF000520001D8B4C4
:101BF000AFEF8EF00401040E035CD8A406EF8EF064
:101C000000520001D8B4AFEF8EF00401080E035C5F
:101C1000D8A411EF8EF000520001D8B4AFEF8EF0CF
:101C20000401100E035CD8A41CEF8EF000520001DA
:101C3000D8B4AFEF8EF00401200E035CD8A427EFD8
:101C40008EF000520001D8B4AFEF8EF00401400EC8
:101C5000035CD8A432EF8EF000520001D8B4AFEF8D
:101C60008EF00401800E035CD8A43DEF8EF000528C
:101C70000001D8B4AFEF8EF004010350D8A448EFB0
:101C80008EF0200E005C0001D8B4BBEF8EF0040192
:101C90000350D8A453EF8EF0100E005C0001D8B4AE
:101CA000BBEF8EF00401BDEF8EF0040119B365EFB8
:101CB0008EF058B465EF8EF05BA065EF8EF05E504D
:101CC0000208D8B065EF8EF0458A5B90589EC7EF4A
:101CD0008EF0040119B3ACEF8EF0368158BEA0EF40
:101CE0008EF05BB0A0EF8EF058B4A0EF8EF034C44D
:101CF00038F433C437F4010E396F00011CEC7CF06A
:101D0000036A0150200F016E000E03220150380FAC
:101D1000E96E010E0320EA6EEF38006E0F0E00161A
:101D20000050D8B49DEF8EF05B805E6A030E040114
:101D3000356FF28AD76AD66A0001A8EF8EF00401E7
:101D40005B90589E459A58A4A8EF8EF04480588620
:101D50000401358BADEF8EF03683C7EF8EF00401B2
:101D600019B3B6EF8EF03681B7EF8EF036835B9005
:101D7000589EC7EF8EF0040136815B90589E459ABD
:101D800058A4C5EF8EF044805886C7EF8EF036A178
:101D9000D2EF8EF035C4F9F30301F98F5B9AD7EFD8
:101DA0008EF00401F4C3F8F3F3C3F7F30301000169
:101DB0009EEF9EF00401696B6A6B6B6B020E6C6F99
:101DC000900E6D6F040EEA6E590EE96E08010A6BF3
:101DD0000C6B100E0B6F000186EC28F0040155C44B
:101DE000E9FF56C4EAFFEE52EE52EC6AED52EF6A9A
:101DF000ED52EF6AED52EF6A57C4E9FF58C4EAFFAB
:101E0000EC6AED52EF6AFA0E0801116F0001D9EC8D
:101E100026F0A8B151EF8FF0040169510F08D8B036
:101E200003D0000151EF8FF00001F3EC36F001C058
:101E30006BF40A0E0801116F0001D9EC26F00101C4
:101E400039A533EF8FF06BC412F8570E0801136FEA
:101E500000011BEC37F0200E9EA82CEF8FF0AD6E2A
:101E600039EF8FF00101320E0801116F0001D9EC3A
:101E700026F004016D516B5DD8A444EF8FF0696BBF
:101E80006BC459F44EEF8FF0692B036A6951590FF7
:101E9000E96E040E0320EA6E6BC4EFFF000109EF48
:101EA0008FF0080E04016C25695DD8B05CEF8FF0EF
:101EB000000E016E15EF90F0036A6C51590FE96E38
:101EC000040E0320EA6EEFCF6EF4000E6EB7010E23
:101ED0000108D8A477EF8FF055C4E9FF56C4EAFF94
:101EE000FF0EEF6EEC6EEC6EEC6E84EF8FF055C46F
:101EF000E9FF56C4EAFFEE52EE52EC6AED52EF6A89
:101F0000ED52EF6AED52EF6A6A6B6A510408D8A08D
:101F1000D6EF8FF055C4E9FF56C4EAFFEF34006EE8
:101F2000EC34016EEC34026EEC34036E0036013694
:101F300002360336003601360236033600360136E5
:101F400002360336F00E0016ED52ED52ED5200C08F
:101F5000EFFF01C0ECFF02C0ECFF03C0ECFF56C472
:101F600003F056C4EAFF55C4E9FFEFCF70F4ECCF9D
:101F700071F4ECCF72F4ECCF73F46A516C25036A00
:101F8000590FE96E040E0320EA6EEF500F0B70112B
:101F900056C4EAFF55C4E9FFEF6E71C4ECFF72C48A
:101FA000ECFF73C4ECFF6A2B85EF8FF0050E6A6FB0
:101FB0006A510808D8A013EF90F057C4E9FF58C43D
:101FC000EAFFEF34026EEC34036E0236033602365B
:101FD000033602360336F00E02160250ED52EF6E53
:101FE00003C0ECFF58C403F058C4EAFF57C4E9FF2C
:101FF000ECCF71F4ED52EFCF70F46A516C25036AA7
:10200000590FE96E040E0320EA6EEF500F0B7011AA
:1020100058C4EAFF57C4E9FF71C4ECFFED52EF6EFC
:102020006A2BD8EF8FF0010E016E000181EF91F065
:102030000401676B686B696B020E6A6F900E6B6FC1
:1020400055C4E9FF56C4EAFFEE52EE52EC6AED5277
:10205000EF6AED52EF6AED52EF6A01014839006E06
:102060000F0E001600500C08D8A43DEF90F0050E9E
:1020700004016A6FFE0E6B6F0101040EEA6E570ECB
:10208000E96E08010A6B0C6B100E0B6F000186ECF9
:1020900028F0FA0E0801116F0001D9EC26F0A8B162
:1020A00097EF90F0040167510F08D8B003D00001FA
:1020B00097EF90F00001F3EC36F001C068F40A0EDF
:1020C0000801116F0001D9EC26F0010139A579EF63
:1020D00090F068C412F8570E0801136F00011BEC52
:1020E00037F0200E9EA872EF90F0AD6E7FEF90F06B
:1020F00001010A0E0801116F0001D9EC26F004015C
:102100006B51685DD8A48AEF90F0676B68C457F490
:1021100094EF90F0672B036A6751570FE96E040E36
:102120000320EA6E68C4EFFF00014FEF90F0070E46
:1021300004016A25675DD8B0A2EF90F0000E016E31
:1021400030EF91F001014839006E0F0E001600507B
:102150000C08D8A4DBEF90F06AC469F4070E040100
:102160006A25695DD8B4B8EF90F0D8B0DCEF90F094
:10217000036A6951570F016E040E032201C06CF40B
:1021800003C06DF4036A6951570FE96E040E032012
:10219000EA6EEFCF6EF46EC47EF40001A9EC5DF040
:1021A0006DC4EAFF6CC4E9FF01C0EFFF0401692BB5
:1021B0000101AEEF90F00401696B69510708D8A0E6
:1021C0002EEF91F055C4E9FF56C4EAFFEF34006EDC
:1021D000EC34016EEC34026EEC34036E00360136E2
:1021E0000236033600360136023603360036013633
:1021F00002360336F00E0016ED52ED52ED5200C0DD
:10220000EFFF01C0ECFF02C0ECFF03C0ECFF56C4BF
:1022100003F056C4EAFF55C4E9FFEFCF6EF4ECCFEC
:102220006FF4ECCF70F4ECCF71F469516A25036A56
:10223000570FE96E040E0320EA6EEF500F0B6E117C
:1022400056C4EAFF55C4E9FFEF6E6FC4ECFF70C4DB
:10225000ECFF71C4ECFF692BDDEF90F0010E016E15
:102260000001A3EF91F004014D6B4E6B4F6B506B6F
:10227000516B526B536B54810001EFEC39F0040148
:10228000BD6B010EBE6F00014AEC4FF001014839F1
:10229000006E0F0E001600500A08D8B4B3EF91F08C
:1022A0000001EFEC39F00A0E0401BD6FBE6B0001B6
:1022B0004AEC4FF001014839006E0F0E0016005035
:1022C0000808D8B476EF91F04839006E0F0E00166A
:1022D00000500708D8B476EF91F04839006E0F0E21
:1022E000001600500908D8A49CEF91F0040E0401D8
:1022F000566F4D0E556F040E586F510E576F0001FB
:1023000059D5012C94EF91F004014F510F0BE8CFF8
:1023100049F14EC44BF14DC44AF152C44DF151C480
:102320004CF199EF91F00001000E016E3BEF92F03D
